:10000000003C0120157C02009199020091990200A8
:100010009199020091990200919902009199020030
:100020009199020091990200919902009199020020
:0C0030009199020091990200CD18010086
:10003C002DE9F047A8B004460078A0F1A0015C2996
:10004C0000F26780DFE811F0BC00DF005D005D00AE
:10005C00F70024015E015D0083018C01A801E5011C
:10006C0014023B024E025A02680273027C028502A1
:10007C008B0294029A02C802DF02EA02F60206031D
:10008C001103B900B900B9001B032503B900B9006D
:10009C003003B900B900B900B900B900B900B90012
:1000AC00B9003B034103B900B900B900B900B9006C
:1000BC00B900B900B9004A035303B900B900B9003B
:1000CC00B900B900B900B900B9005C03B900B900B6
:1000DC006303B9008503B900B900B900B9008F03F7
:1000EC00B900B900B900B900B900B900B900B9003C
:1000FC00B900B900B900B900B9009803A6035D00B6
:10010C00B90060681221002808BF0221617001F05B
:10011C0083BA4D2800F25180A678DFE810F04B032B
:10012C004E005B03650345044E004E006E047F04D5
:10013C00CD044E004E004E004E004E004E00D60434
:10014C00E00408054E002D05350643064E004E060C
:10015C005D064E00680682064E00AB06CF06D20640
:10016C00DF0603074E004E004E004E004E004D07BA
:10017C004E005B076C077D074E004E004E004E0094
:10018C004E004E004E004E004E004E004E004E00F3
:10019C004E009607B107CB074E004E004E004E00A6
:1001AC00E5074E0047084E0058084E004E004E0022
:1001BC004E0078088F089C08A608122001F02BBA74
:1001CC006068002801F02682A168002901F02282D3
:1001DC0001783A20002908BF3B200BAD00211122E9
:1001EC002B462BF033FE0028607041F01582D4E9C9
:1001FC0001109DF82C204270097800F8021B691C34
:10020C00102200F034BE6168002901F003820878E6
:10021C004A783A258B788DF82C20002808BF3B258E
:10022C000BA80130002B01F03680033110222BF08B
:10023C00EFFF01F032B86168002901F0EB81A06892
:10024C00002801F0E78111F8012B00F8012B2CF0AC
:10025C00EAFC60680178002901F0AD81DFF8DC0E62
:10026C000BAE002506F108080788AF4201F0D081DB
:10027C00A9B2042000221423009628F06BFE6070B3
:10028C0020B92CF003FA002801F023820135ECE7A9
:10029C006068002801F0BE810178002901F003801C
:1002AC00DFF8980E0DF12C0A00250DF11C08002624
:1002BC000AF10809CDE90955CDE907550788B74278
:1002CC0001F0D781B1B2042000221423CDF800A094
:1002DC0028F040FE607098B96068494608220430E6
:1002EC002AF0F6FD002801F0C2814DB96068414644
:1002FC00082204302AF0ECFD0025002808BF354602
:10030C000136DCE76068002801F08481017800295F
:10031C0000F0E387DFF8240E0DF12C09002709F11A
:10032C0008080588BD4201F07781BEB20420002286
:10033C001423CDF80090314628F00CFE607020B9E3
:10034C002CF0A4F9002801F0A6810137EAE7DFF8C8
:10035C00F00D4FF4807100781FF098FF01F058B940
:10036C006068002801F056814188008828F0EAF87E
:10037C0068B9606801224188008823F095FA6068AA
:10038C004188008828F0DEF8002801F09B81616824
:10039C000979417001F03CB96168002900F070875F
:1003AC00DFF8A05D087885F8260095F8722048885B
:1003BC00E882087A2876488968834868A862888920
:1003CC00A884887B85F83800C87B6871087CE87045
:1003DC004869286388696863087F824202D024F0E8
:1003EC00FDF9616805F139001D312CF067FC95F8B9
:1003FC002600082840F04C87DFF8482D2120742176
:10040C002CF046FA00200221002525F0CDFF00F04B
:10041C0040BF6068002800F03587007824F0DEF9D2
:10042C006168DFF8205D287E4978884212D02976F1
:10043C000BA9E12028F0C0FB606841789DF82C00E6
:10044C00884207D08DF82C100BA9E12024F03CFB3E
:10045C0060684078012101FA00F0A8622AF028FABD
:10046C0000260120A5F870601EF02CFD00F00BBFDB
:10047C006068002801F0CE8001884088ADF81C002F
:10048C00ADF82C100BA9532024F01EFB07A950200B
:10049C0024F01AFB0DF11B01E12028F08DFB6068A4
:1004AC009DF81B100079814201F0B2808DF81B0081
:1004BC000DF11B01E12024F007FB01F0A9B86168E4
:1004CC00002901F0A780DFF8800C2CF0ACFB6068F1
:1004DC00DFF8782C0189807A1180DFF8741C0870A1
:1004EC0001F096B86068002801F0948000216170DA
:1004FC008178008821F0F0F901F08EB8A06800280E
:10050C0001F088800020607023F03CFE002800F091
:10051C00E886A16800F08FBE6068002801F07A8040
:10052C000021617000780AF08DF801F075B86068F0
:10053C00002801F06F80007824F00AFB01F06BB802
:10054C00A068002801F06680002060702CF0FEF896
:10055C00B2E00020607026F055FB01F05DB8A06899
:10056C00002801F05780002060702CF0CDF9A3E03A
:10057C000020607026F07EFB01F04EB86068002809
:10058C0001F0488000216170017D19B1C17CDFF858
:10059C00C42B5174817D19B1417DDFF8B82B917456
:1005AC00017C19B1C189DFF8AC2B1181017B19B128
:1005BC008168DFF8A02B5160817C19B1417CDFF898
:1005CC00942B51730179002901F026800068DFF823
:1005DC00841B086001F020B8A068002801F01A8084
:1005EC00DFF8701BD1F80D20C0F80D2091E82C001D
:1005FC0085600D7BC0E900230573B1F81110A0F8DC
:10060C00111001F005B8A068002801F0038000214A
:10061C006170411C24F07AFA00F0FEBF606800287B
:10062C0000F0F8870021617022F092FEA16808802A
:10063C0000F0F2BF6568002D00F0EC87EB88AA880B
:10064C00698828782E890A35CDE9006516F0FAFC00
:10065C0000F0E1BF6068002800F0DC8782884188E8
:10066C00007806F07DFF00F0D6BF6068002800F02F
:10067C00D18700F1120125F06BF900F0CCBF606856
:10068C00002800F0C7874168007822F01FFF00F0B7
:10069C00C2BF6068002800F0BD870021617000783F
:1006AC0026F0F4FF00F0B8BFA068002800F0B28775
:1006BC00002060702AF06CF9A16800F0BDBD00202C
:1006CC00607021F08FFD00F0A7BF6068002800F07B
:1006DC00A187006826F0B2FA00F09DBF6068002880
:1006EC0000F09887006805F0A5FB00F094BF6068E7
:1006FC00002800F08F8700680DF03CFE00F08BBFE7
:10070C000020DFF8541A6070E07800F095BD616845
:10071C00002900F081870820ADF82C000888ADF87E
:10072C002E00081D0BAC90E86800221D68C2087CE6
:10073C00D1E905231C31CDE910238DF83C0004F1DF
:10074C001C0010222BF064FD204628F045FC00F024
:10075C0063BF6068002800F05F87817A008824F00E
:10076C0019FD00F059BF60680078002800F08D85F5
:10077C0026F0DCF800F050BF6068002800F04A87D3
:10078C00DFF8D819097801293FF617AD2BF096FA46
:10079C0000F041BF6068002800F03C87DFF8BC190E
:1007AC00097801293FF609AD4168008821F010F85D
:1007BC0000F031BF6068002800F02C87407818B139
:1007CC00FF20032125F0F0FD2BF024FFE848012148
:1007DC000160FEE76068002800F01C8703210171AE
:1007EC00E449016000F014BF6268002A00F012872F
:1007FC00A168002900F00E8700206070107840B1CD
:10080C0001200870DFF858090078002818BF012073
:10081C004870907840B101200871DFF848090078E1
:10082C00002818BF01204871D07848B100202BF067
:10083C00F9FAD4E90121C0F34030C8710120887164
:10084C00107950B30120087201F10C002BF0EAFA78
:10085C00A1680882DFF80409007802281DD1DFF8AE
:10086C0008090078C8B9DFF804590120A847A16825
:10087C0048610220A847A16888610420A847A168A4
:10088C00C8610820A847A16808621020A847A16881
:10089C0048622020A847A16888626068427932B11A
:1008AC00012281F82C20DFF8C8281288CA858279A9
:1008BC0032B1012281F83020DFF8B82812884A863C
:1008CC00C27932B1012281F83420DFF8AC281288C9
:1008DC00CA86027A3AB1012281F83820DFF89C28C6
:1008EC00127881F83920427A3AB1012281F83A2003
:1008FC00DFF88C28127881F83B20827A3AB10122F9
:10090C0081F83C20DFF87C28127881F83D20C27AEF
:10091C003AB1012281F83E20DFF86C28127881F878
:10092C003F20027B3AB1012281F84020DFF85C289D
:10093C00127881F84120427B3AB1012281F84220A1
:10094C00DFF84C28127881F84320827B3AB10122DF
:10095C0081F84420DFF83C28127881F84520C27BCE
:10096C00002A00F0C18601201122002681F84600E1
:10097C000BAD812000212B462BF068FA9DF82C0042
:10098C00A168002881F8470000F091862CF0F5F959
:10099C00A1680028886400F0A2869DF82C20691CB0
:1009AC002BF036FC00F09FBE254655F8040F0028AE
:1009BC0000F0308600216170017841B14078DFF899
:1009CC00A0270121107063202BF062FF28680179A9
:1009DC0041B14079DFF88C27012110706D202BF08C
:1009EC0057FF28688179002900F07D84C1794FF484
:1009FC0000500CF025FF00F08ABC6068002800F065
:100A0C00098690F9005028462AF042FBA06800287D
:100A1C0000F0FE85E9B2017000F0FABD60680028B4
:100A2C0000F0F885002161702A212BF079FADFF8AB
:100A3C0014576068DFF860670822E98A0180A98C86
:100A4C008181698BC182DFF854170978817205F1B5
:100A5C0039010E30B04767682BF0B8F80146B81C66
:100A6C000822B047606805F11C0108221830B04715
:100A7C006068297E012280F82310DFF8241780F8A3
:100A8C0021208978CB0718BF80F824208A0744BF1F
:100A9C00012280F825204A0744BF012280F8262035
:100AAC000A0744BF012280F82720490644BF0121D0
:100ABC0080F8281000F0B0BD6068002800F0AA850E
:100ACC0000782BF0F1FE00F0A3BD6068002800F068
:100ADC00A1850088002110F08FFA00F09DBD6068A0
:100AEC00002800F0978530462AF052FE0546002873
:100AFC0000F01585E888DFF8AC1640F00C00E880B3
:100B0C0002202BF0C7F8DFF8A01603202BF0C2F858
:100B1C0040F20110ADF831006068016800790B916A
:100B2C008DF830000BA820F09BFC00F074BD6068C1
:100B3C00002800F06F850BAD011D082228462BF014
:100B4C0067FB032029F0A4FE6068C07B27F01AFB2A
:100B5C00DFF84C0683786068418886890278807B50
:100B6C00CDE90060284614F05FFE00F054BD00BFD4
:100B7C007C052043010102066768002F00F04A85BE
:100B8C002BF02DFF0546002800F0DA84387828B1C8
:100B9C00E988787821F001010843E880B87830B111
:100BAC00E988F87821F0020141EA4000E8803879C0
:100BBC0030B1E988787921F0040141EA8000E880BD
:100BCC00B87930B1E988F87921F0080141EAC00020
:100BDC00E880387A30B1E988787A21F0100141EA5E
:100BEC000010E880B87A30B1E988F87A21F0200159
:100BFC0041EA4010E880387B30B1E988787B21F0FD
:100C0C00400141EA8010E880B87B28B1A968F87BE4
:100C1C0021F001010843A860387C38B1A968787CC0
:100C2C0021F00201002818BF0231A960B87C38B14C
:100C3C00A968F87C21F00401002818BF0431A960D0
:100C4C00B87D38B1A968F87D21F01001002818BFD3
:100C5C001031A960387E38B1A968787E21F0200166
:100C6C00002818BF2031A960B87E38B1A968F87E79
:100C7C0021F04001002818BF4031A96097F82200EC
:100C8C0048B1A96897F8230021F48061002818BFA7
:100C9C0001F58061A96097F8260048B1A96897F81A
:100CAC00270021F40051002818BF01F50051A9605C
:100CBC0097F8280048B1A96897F8290021F48041D9
:100CCC00002818BF01F58041A96097F82A0048B1A7
:100CDC00A96897F82B0021F40041002818BF01F5F2
:100CEC000041A96097F8340048B1A96897F835001D
:100CFC0021F48011002818BF01F58011A96097F824
:100D0C00380048B1A96897F8390021F4800100280F
:100D1C0018BF01F58001A96097F83C0048B1A9689B
:100D2C0097F83D0021F08071002818BF01F1807107
:100D3C00A96097F83E0048B1A96897F83F0021F0E8
:100D4C000071002818BF01F10071A96097F84000EC
:100D5C0048B1A96897F8410021F00061002818BF3C
:100D6C0001F10061A96097F84200002800F054845A
:100D7C0097F84310A86800290CBF20F0805040F071
:100D8C008050A86000F048BC6068002800F04284E5
:100D9C008178002900F0E783C2780321002A08BF7C
:100DAC000121E1E36168002900F0348408888A7825
:100DBC0001211CF0E7FB00F02EBC02206070606883
:100DCC00002800F029844188007825F077F8002865
:100DDC0040F01E8400F020BC6068002800F01A84EB
:100DEC0000216170007825F09DFE00F015BC606854
:100DFC00002800F00F84A168002900F00B8400216A
:100E0C00617000782AF07CF9A168087040002BF022
:100E1C00B4FF0146D4E901025160007829F01EF9B3
:100E2C00FAE36068002800F0F583A068002800F061
:100E3C00F1830026C0E9006660684188007828F0DC
:100E4C00B1FC002800F0CF8366700546A1680088CD
:100E5C000880A8780028887000F0DE832BF08DFFC6
:100E6C00A1680028486000F0D7838A78E91C2BF031
:100E7C00CFF9D1E36068002800F0CC830021CDF8D5
:100E8C003A10CDF83610CDF83210CDF82E1002797C
:100E9C004188ADF82C105AB1816849B10F2A28BF8E
:100EAC000F228DF82E200BA803302BF0B1F96068BF
:100EBC0000780BA901221EF03FFEACE32AF026FFBE
:100ECC00A9E36568002D00F0A5832F7838462AF039
:100EDC006BFC002800F05183D0209CE36068002854
:100EEC0000F0988300782AF05FFC002800F09283D1
:100EFC000546007B26F07CFB0028607040F08C835C
:100F0C00DFF8E40A4168002900F0868300220C46D1
:100F1C002346002C00F0CD83AB4200F0CA831C6842
:100F2C001A46F5E76668002E00F07483357D284676
:100F3C002AF03AFC002800F06D83307F102141EA42
:100F4C004007717F002908BF4700B07F002818BFF9
:100F5C0047F00807F07F002818BF47F0200796F8E5
:100F6C002000002818BF47F0400796F82100002801
:100F7C0018BF67F07F07D6F8188028462BF0B8F911
:100F8C00002800F0478305466068827A01788DF866
:100F9C00352082898DF83410ADF836204A1E022A8D
:100FAC0005D3032900F047840F2940F04984418878
:100FBC00ADF82C1000F044BC61680220002900F050
:100FCC002A830A888DF834004988ADF82C200BA8A8
:100FDC0002221DE061680220002900F01C838DF8BC
:100FEC003400002308880A794988ADF82C000BA836
:100FFC0028F0ECFF0FE361680220002900F00B835E
:10100C008DF83400052208884988ADF82C000BA80F
:10101C0000232AF021F8FEE265680220002D00F082
:10102C00FA828DF834002E7B00272888AB79AA88A9
:10103C006988ADF82C00A8682D69CDE90006CDE9CA
:10104C0002570BA817F028F8E5E265680220002D7E
:10105C0000F0E1828DF83400EE682F7C4FF0000C2C
:10106C002888EB8869882A79ADF82C00287A6D6974
:10107C008DE8C100CDE9035C0BA816F0B5FFCAE200
:10108C006168002900F0C68202208DF83400887B4C
:10109C000D88421E8DF82400022AADF82C5005D381
:1010AC00032800F0A2820F2840F0A482088AADF831
:1010BC001C009FE26068002800F0AC8202218DF8D1
:1010CC0034100188ADF82C10817B4A1E8DF8241049
:1010DC00022A05D3032900F0B0820F2940F0B38215
:1010EC00018AADF81C10AEE26068002800F0928214
:1010FC0002214FF6FC728DF8341001888A1A032AEB
:10110C0011D8022A0FD02BF079FAADF82C006068B8
:10111C000021837AC27A0091811C0BA824F056FE20
:10112C00607060680188ADF82C10837AC27A002157
:10113C000091811C0BA824F049FE6CE254F00200D3
:10114C00036E0020C05E002008250020062500202C
:10115C000425002080200020B32600201C25002020
:10116C00EE260020326E0020F3260020D5FC010074
:10117C009E2600209A260020A2260020E42600208D
:10118C00E1260020D6260020E2260020ED260020B5
:10119C00D7260020F02600201DC2020004230020C8
:1011AC00806C002079630200BDBE020062680220E0
:1011BC00002A00F030828DF83400002310889178DA
:1011CC00D278ADF82C000BA820F0D6FA23E2616897
:1011DC00002900F01F82CA7A887A0B7B4D7B002A8B
:1011EC0018BF40F00200002B18BF40F00400002D87
:1011FC0018BF40F008008A7B002A18BF40F040005E
:10120C00C2B208880231002325F01CFC03E260689E
:10121C00002800F0FF81A168002900F0FB81007814
:10122C000BA929F0EBF80020BDF82C206070D4E954
:10123C000101A1F8012000780870EDE16068002838
:10124C0000F0E881B0F80110ADF82C1000780BA973
:10125C0029F02CFFDFE16068002800F0DB81017AC7
:10126C00427A00231FF0A2F8D5E16068002800F054
:10127C00D1818178C2780088002326F0FBFFCAE177
:10128C00022506E002266670C6E129F0A6F8C3E145
:10129C0000256570C0E127F01DF80BAA2846112126
:1012AC002BF0F6FAB7E100F10C010BA810222AF092
:1012BC00AFFF6068D0E907120430CDE90F1207A91F
:1012CC0028F096FE0028607000F0FE816168488866
:1012DC0004310BAA21F041FD9DE101302AF0B7FB4E
:1012EC0099E1012097E1017A89B1C168008A42072E
:1012FC0001D064290BD315F085FA002001210CF0E4
:10130C009FFADFF8EC26352028212BF0C1FA28684B
:10131C00817C41B1808ADFF8DC26022110804420D8
:10132C002BF0B6FA2868817D41B1008BDFF8C82616
:10133C000221108046202BF0ABFA2868817E41B147
:10134C00808BDFF8B8260221108083202BF0A0FAC6
:10135C002868817F41B1C07FDFF8A426012110707D
:10136C0029202BF095FA286890F8201049B190F8B4
:10137C002100DFF89026012110702B202BF088FA29
:10138C00286890F8221049B190F82300DFF87826ED
:10139C000121107043202BF07BFA286890F8241060
:1013AC0049B190F82500DFF86426012110702E2039
:1013BC002BF06EFA286890F8261049B190F82700A7
:1013CC00DFF84C26012110702F202BF061FA2868D1
:1013DC0090F8281049B190F82900DFF8382601213F
:1013EC00107030202BF054FA286890F82A1049B16C
:1013FC0090F82B00DFF82026012110702C202BF008
:10140C0047FA286890F82C1089B190F82D20102AF2
:10141C0028BF10228DF82C20016B0BAC601C2AF01D
:10142C00F7FE8120112122462BF032FA286890F821
:10143C00341049B190F83510102928BF1021826B57
:10144C0062202BF025FA286890F83C1041B1006C12
:10145C00DFF8C8250421106084202BF019FA2868C5
:10146C0090F8441049B190F84500DFF8B4250121FB
:10147C0010704B202BF00CFA286890F8461069B1CC
:10148C00DFF8A04500F14701082220462AF0C0FEF3
:10149C004720082122462BF0FBF9286890F84F10C2
:1014AC0031B100F15002012008212BF0F1F928682C
:1014BC0090F8581041B190F859008DF82C000BA9F8
:1014CC00522023F001FB286890F85E1049B190F887
:1014DC005F00DFF854250121107033202BF0D8F970
:1014EC00286890F85C1059B190F85D00DFF83C2545
:1014FC000121107032202BF0CBF922F0DBFC286894
:10150C0090F86010002900F0878090F86100DFF8F7
:10151C00D8144870DFF8CC1481F868007CE01C20EB
:10152C002BF02BFC002877D01C2105462AF0F8FC68
:10153C0028462E7126F012F900287FF4DBAA91E0E0
:10154C001C202BF01AFC002866D01C2105462AF022
:10155C00E7FC28462E7126F001F9002800F0828065
:10156C006768FFF713BB002103794279002B18BF82
:10157C00403100880FF0CEF94DE02AF021F9DFF868
:10158C0068140978884270D22BF029FA20B1814670
:10159C00007B002800F08E811C202BF0EEFBD8B3D2
:1015AC001C2181462AF0BCFC89F804604FF001082C
:1015BC0065682F7880E1013007A928F019FD60706B
:1015CC0050BB07980021182240880BAB2AF03EFC38
:1015DC00607008BBA068DDE90F12C0E90712093082
:1015EC000BA9FEF70DBEB12015E0103107A82BF0AA
:1015FC001AFB6168DFF8EC03C08A854210D1887A47
:10160C000A7E0C310123009107A90AF0D3FC08B122
:10161C00002000E002206070012028B0BDE8F087B7
:10162C0088890A7E8B7A07AE0025CDE90006CDE9C4
:10163C0002258A1C0BA9212011E000F1100107A83A
:10164C002BF0F1FA60688189027E837A07AE00255F
:10165C00CDE90225CDE90016821C0BA922201CF035
:10166C0029FED8E728462BF086FBD120D3E7374656
:10167C003546012DD0DB60680822011D48462AF052
:10168C00C7FD60681422D0E90710CDE90B10B9B280
:10169C000BAB042008E00BAD142128462AF040FCCB
:1016AC000420314614222B4627F06AFCB3E78E64E3
:1016BC0019E0AB42B0D1A94208BF021D28681060E6
:1016CC002846E3E0C820A6E70798182140880BAA13
:1016DC00E6E5A068DDE90B12C0E907129CE70020E3
:1016EC00886481F847006068007C70B110202BF092
:1016FC0044FB0346A06803653BB10121102280F82E
:10170C004C10622000212AF0A1FB6068417C31B1B1
:10171C00A168012281F85420C04A12688A65817C34
:10172C0039B1A168012281F85C20BD4A127881F898
:10173C005D20C17C51B1A0680121082280F85E10A7
:10174C00A8495F3039312AF063FD6068017D59B1D9
:10175C00A568012085F867002AF038FA014605F1E2
:10176C0068002BF060FA6068417D79B10BA95220BA
:10177C0027F022FAA068012180F870109DF82C1037
:10178C00002918BF012180F871106068817D19B1A2
:10179C00A1680122A1F87220C17D51B1A16801227A
:1017AC0081F87420A14A1278002A18BF012281F80E
:1017BC007520017E39B1A168012281F876209A4A00
:1017CC00127881F87720417E51B1A168012281F80D
:1017DC007820854A5278002A18BF012281F8792096
:1017EC00807E00283FF418AFA068012580F87A505D
:1017FC007C4890F82600082818BF042817D0A8B9F0
:10180C0021202BF0CEF9742810D10BAB2120002114
:10181C00742200252AF01AFB48B99DF852000438AE
:10182C0020F00400B0FA80F0450900E00025A06823
:10183C0080F87B50F0E6811C0BA82BF0F4F9606863
:10184C00817B31B348002BF098FA88B36168064667
:10185C000022887B904206D00B6933F8123026F8B0
:10186C0012300132F6E78B8CCA8AD1F828C091F875
:10187C002210FFB2CDE90406CDE90271CDE900C812
:10188C000BA8294622F0BBFE607030462BF073FA91
:10189C00C2E6838CC28A816A90F82200FEB2CDE93E
:1018AC000018CDE902600BA8294608F0E9FDB2E664
:1018BC001020B0E64FF000084E4606F80C7F287A50
:1018CC0030734A48706014202BF057FA0028B0602F
:1018DC0045D014212AF024FB6268D9F81400526810
:1018EC008179927901F0F00102F00F0211448171BB
:1018FC006168D9F8140049680A780270D1F802209E
:10190C00C0F80220CA79C271097B017350002BF018
:10191C0034FAD9F81410886060B1CA7900239A425D
:10192C0008D065686D68AD6835F8135020F8135011
:10193C000133F4E7087B40002BF01FFAD9F81410A0
:10194C00086160B1097B0022914208D063685B6832
:10195C001B6933F8123020F812300132F4E73046AC
:10196C0028F06AFBB82802D00746022806D1307846
:10197C0025F03EFE304628F05FFB074637B1B8F144
:10198C00000F0FD048462BF0F6F923E0B8F1000F0A
:10199C003FF442AE484625F0E1FE00287FF43CAE11
:1019AC00484673E7D9F8140078B1816821B108462C
:1019BC002BF0E1F9D9F81400016921B108462BF09C
:1019CC00DAF9D9F814002BF0D6F90020C6E900009A
:1019DC00C6E90200B82F3FF47FAA022F3FF47CAA7D
:1019EC001AE600BFC05E0020782500207D5700203D
:1019FC00606800209E2600209A260020A226002047
:101A0C00E4260020E1260020D6260020E226002035
:101A1C00ED260020D7260020F02600208826002066
:101A2C00D3260020B0250020DB260020DC26002059
:101A3C002DE9F04F99B080466FF007000DF11C0BAB
:101A4C00063098F808105A46ADF85200D8F8040041
:101A5C0011F0D4FB002800F0B5809DF81E609DF8B5
:101A6C001F409DF82070BDF826502AF0C1FD84421D
:101A7C0040F0A88025F003004FF6F87480B2A04225
:101A8C0000F0A080012F00F29D80022E80F09A8041
:101A9C00B8F82800ADF84800B8F83200ADF82A00C4
:101AAC009DF82200D0B1D8F804109DF81D209DF8A7
:101ABC003830012029F06EFA08B1CF2083E0DFF82E
:101ACC005807C078012809D1B8F828002BF01DF868
:101ADC0020B1417901F0E701083141719DF82100F5
:101AEC0068B1BDF82610FF2027F05CFE9DF8211090
:101AFC00D8B141F001012C268DF8211016E09DF88B
:101B0C003900002864D09DF83D10FF2902D000292F
:101B1C0040F0ED80DFF80407BDF82620C18A8A4228
:101B2C0040F0EE800120222607E0082601F0030099
:101B3C00012808BF46F0110601203746B107DFF82F
:101B4C00DC9658BF67F07F07002808BF37469DF822
:101B5C00220030B999F80B0018B107F022002228A6
:101B6C0013D117F0400A58D0119899F80E2001782B
:101B7C00920718D40C291BD8012241F290438A40B9
:101B8C001A4245D1032940D012E0F8B200F04200CD
:101B9C0042287FF492AF1198007800F0FE000628DE
:101BAC007FF48BAFDDE7A1F10C0212F10C0F2AD8F8
:101BBC00B9F81600BDF82620824203D1BDF82800E2
:101BCC0026F0D8F9D32017F0D8FC19B0BDE8F08F67
:101BDC00BDF8260024F092FD0238DFF84016B0FA6A
:101BEC0080F0CA8A4109BDF82600904208BF023134
:101BFC00002900F08C809DF81E20002A00F03A810C
:101C0C0001F1400738E1032902D140780D2804D0B6
:101C1C0007A823F0AFFF0128D7D0B9F82400B8F8F3
:101C2C00441081420AD198F84620B8F84210B8F80E
:101C3C00280000230093002310F090F89DF8220058
:101C4C00E0B1B8F84210B8F8280026F07BFCB8B325
:101C5C000646D8F804009DF81D10F2780844417B24
:101C6C008A421EBF00227260F1700130042127F0FD
:101C7C008DFA71688842A8D30130706099F80E0013
:101C8C008007A2D59DF84D0058B1BDF8280029F069
:101C9C002FFC00286FD0D8F80400417801F0DF0148
:101CAC0041709DF82E00A0B3D8F804008179013959
:101CBC0081718DF82E1007F07F0009062CD12AE0D7
:101CCC009DF84D00002841D0042028F04DF8002844
:101CDC003FF47BAF01464FF4B2700880B8F828008F
:101CEC004880DFF83C0500781FF03EFC6DE7109A49
:101CFC009DF83C0022F03EFE30B1012000261CE78E
:101D0C0090F826000428F8D10026002015E70027BB
:101D1C00B2E007F07F000746390702D44FF0000A03
:101D2C0049E0F9B24A0737D4C9069DF821103DD5D0
:101D3C00C1F3820212B1072A18BF013A002A08BF68
:101D4C00074601F0E30040EA82012DE099F86C00AF
:101D5C0001287FF493AF11980078062803D1BAF1CB
:101D6C00000F7FF48BAFE01DBDF82A1080B28142CA
:101D7C003FF42BAF44E1D32017F0FFFBDFF8A404B2
:101D8C000078002800F0AD80DFF89C1451F820009A
:101D9C00C0EB00108100A6E09DF8210000F0E001EE
:101DAC0000F0E30040EAD1018DF82110D8F80400CE
:101DBC004FF4805A017299F82600092801D00428A2
:101DCC0029D1B9F81610BDF8260088420AD024F0A3
:101DDC0095FC022806D09DF8210000F00300012894
:101DEC007FF4F3AE9DF81E0000285BD011989DF88F
:101DFC0038100078042808BF02296DD0072808BFC6
:101E0C00042900F0838003287FF4DFAE07A80021AB
:101E1C0012F0FEFCD9E6FEB217F0610F49D0F007C4
:101E2C0008D0B8F8281007A816F03AFF002871D08F
:101E3C0007F09F070025FEB2B80605D529F0D0FDA6
:101E4C0007A815A906F0ACFA700640F13981B8F86C
:101E5C00281007A80DF152022B4611F04BFA00285E
:101E6C0000F08180054611980078012808BF4AF0DF
:101E7C00100A25E101F1200724F040FC0138B0FAEA
:101E8C0080F0400947EA00069DF81E0000283FF448
:101E9C0053AE1198007829F067FB012818BF07F0A2
:101EAC007E0649E629F09CFD07A815A906F078FAEC
:101EBC008BE69DF81E00012864D111980078032848
:101ECC0053D005285ED1B8F8281007A80DF152029E
:101EDC00002311F00FFA78E607A9002012F00CF994
:101EEC0073E6D1480168D1480268BDF828009047D4
:101EFC0001287FF46AAECE480168BDF828008847F7
:101F0C00CC480168BDF8280088475EE607A819F0A0
:101F1C00AFFA5AE628F06CFB9DF82E100546BDF87A
:101F2C00280021B9B8F8281088423FF484AFB9F8DA
:101F3C001610814204D1B848807800283FF47BAF5A
:101F4C00B8F8281007A82A460AF096FA002800F0DC
:101F5C009E8030074AF0040ABDF8260048BFE01DF9
:101F6C00ADF8520067E70025AAE0BDF8260029F07D
:101F7C00BFFA38B1B8F8281007A80DF152020023A7
:101F8C0011F0B8F99DF82E0088B325F087FD0028D4
:101F9C007FF41BAE9DF83900B8B3109A9DF83C0045
:101FAC009DF83D1022F0E6FC002873D09DF83D0012
:101FBC00002878D010992AF035FD9DF82430ADF822
:101FCC00520011209DF823209DF821104AF0400A60
:101FDC00002B08BF0920002A18BF0830002918BFA1
:101FEC000130D8F804100A5C013A0A5465E09DF8F7
:101FFC001E00012804D11198007803283FF4E5ADA8
:10200C0007A841461FF0C8FDDFE59DF82010BDF87C
:10201C0026000029ADF8520000F0CF804020BDF81A
:10202C0026100BF11D0200EAC7099DF820004B4653
:10203C001AF0A6FA38B1D8F804004AF0200A017850
:10204C0001F03F0101709DF8390048B1BDF8261030
:10205C000BF1200023F070FD4AF0400AADF852005D
:10206C009DF81E00012806D0BDF82810BDF82600EA
:10207C00002216F075FABDF82810BDF826004A4665
:10208C0013F010FF002818BF4AF0200A15E007F0E3
:10209C00DF07CFE6BDF82610BDF828000B22002381
:1020AC001BF07EFF91E5BDF82600ADF852002AF03A
:1020BC002CFD002808BF4AF0400A28F099FA054682
:1020CC00A01DBDF8521080B20E1A5B4818BF2E46E8
:1020DC000078012805D1E01DB8F8321080B2814299
:1020EC002ED178B2B0F1FF3F3FF76FAD002E3FF429
:1020FC006CADB8F808002AF040FE00283FF465AD3E
:10210C00B8F80820D8F8041005462AF081F89DF894
:10211C001E10002098F80830B8F8282016908DF87A
:10212C005410BDF8521015ACCDE9006ACDE902048B
:10213C00284614F08DFC68B328462AF01CFE44E5B2
:10214C00B8F828108142CCD0601CBDF8262080B293
:10215C008242C6D2BDF828008142C2D02AF0D5FCFA
:10216C000028BED0017901390129BAD84088012153
:10217C008DF85410ADF8600015AD284620F020FB0A
:10218C000028AED0281D1FF08FF80028A9D027F00A
:10219C00E7FEA6E72048407800283FF416AD002063
:1021AC008DF81860ADF81900DDF826004FEA3040C4
:1021BC00059005A829F040FE07E531073FF52EAF45
:1021CC009DF81E1001293FF429AF00211AF098F94F
:1021DC0020B1407901380228FFF420AFB8F8441040
:1021EC00BDF8520026F0AEF930B1807828F090FCA2
:1021FC0001380728FFF412AFBDF8280029F078F950
:10220C0018B104208DF8200008E7BDF82610BDF8A1
:10221C002800022243E700BFEC240020C05E00200F
:10222C00036E0020E5260020C8EA02004C220020A4
:10223C005422002050220020F12600202DE9F04FDE
:10224C008FB00C46480718D4200471D4E00400F178
:10225C00CC81200600F1EA81A00700F10082200564
:10226C0000F13482600600F13482A00400F1668231
:10227C00600400F1A782002017E2DFF8D80501788E
:10228C00062900F21082DFE811F00700C0010E02EF
:10229C000E0208020E02C501DFF8BC6596F8371075
:1022AC004A0700F1C8818A0700F1ED81090740F166
:1022BC00FA810621017096F83A00002800F0C582D8
:1022CC0021F060FF002800F0C0820546F0684068ED
:1022DC004078800740F19482287804AB03210022D7
:1022EC0023F055FB002800F0798206980188B42968
:1022FC0016D8B4214FF47A720180DFF860054FF4E0
:10230C00005100782AF0A1FCDFF85805016839B1BA
:10231C00DFF854050078FF2814BF2878FF20884781
:10232C00F06840684078C00740F0618209205BE2A9
:10233C00DFF83C05DFF82475DFF818A5DFF8445505
:10234C0048F2040848F202094FF6FE7B008802901E
:10235C0038781EF071FC002800F0448106460078A5
:10236C00D3280DD1F089404537D0484539D048F2B3
:10237C000101884240F01C81304617F041FF17E103
:10238C009AF80010884219D1012856D0032840F041
:10239C000F81DFF8CC0400780138012800F20881A5
:1023AC00B078012877D0002840F00281707800289E
:1023BC0000F0BE80002020F01BFBF9E00A2840F062
:1023CC00F780DFF8941491F837003071096A00290E
:1023DC0000F0EE80B01C8847EAE030461CF012F8A2
:1023EC00E6E0DFF894040078002800F0E1809AF829
:1023FC000000012840F0DC8029F062FE002840F04B
:10240C00D7807088002840F0D3800AAD122128466E
:10241C0029F086FD2AF098FA304629461AF01CFE5F
:10242C00BDF83400B0F5285FC0F095800120022182
:10243C0021F072F8DFF84C54BAE0DFF8240400788D
:10244C000138012800F2B4807078DFF80C2460B1F8
:10245C0092F83C0092F83D10013082F83C00C0B27A
:10246C00884202D901200021A0E09AF8010003283B
:10247C0034D002284BD0012840F09A80DFF8F803C2
:10248C000078002800F08C8029F01AFE002800F05B
:10249C009380012085E07078002851D02AF0AEF8A6
:1024AC005845DFF8D8B34FF6FE7103D1BBF81600D0
:1024BC00884207D0ABF81610ADF81010532004A9C1
:1024CC0022F002FB21F016FA28F0B2F800208BF86B
:1024DC0026001FF087FE4FF6FE7B69E0AB4604AD8D
:1024EC00AB2000212A461EF0B3FE04200A955D465F
:1024FC004FF6FE7B8DF82C000AA811F08BFD2AF00C
:10250C0023FA38784FF4805141F2883220E00120D0
:10251C0050714FF48060ADF8100004A81BF088FADD
:10252C002AF012FADFF84C034FF4805102680EE0E7
:10253C0013F04AFAC848406AD0BB1FF053FE37E08C
:10254C0002204FF4805140F6B8328AF802003878F5
:10255C002AF07BFB2CE0CA480DF10F01006804AA9D
:10256C0019F02EFA01460298C64D814213D29DF8FD
:10257C00200010B1FD208DF820000420142204ABA3
:10258C008B4626F0FDFC0BEB4B004FF6FE7B01213E
:10259C0005EB80004172B048002180F83B1003E04D
:1025AC000020AD4981F83B000120012102F078FEAA
:1025BC00304628F089FBCBE6A74991F83E0020B1C4
:1025CC00886A0028F4D08047F2E70020002102221C
:1025DC000023ADF8100002208DF8180004A828F094
:1025EC003BFD8CE784F400405FE09D4800780138A7
:1025FC00012868D89748017803295CD0012962D159
:10260C004178002020F088FF5DE00120012120F0BE
:10261C0083FF48E00021322201708F4880F8361089
:10262C008E48042100782AF010FB3CE014F03AFFAD
:10263C0084F0800039E00521017096F83810890784
:10264C0036D596F83A1099BB052101600120B0707F
:10265C00002020F015FF022027F012FD23E0804817
:10266C000078013801280BD80020CDE9040004A81B
:10267C0016F020FA20B17948022100781DF006FEF0
:10268C0084F0020011E00421017096F83810C9079B
:10269C0009D096F83A10002942D028F033FB0420D8
:1026AC00012102F0FDFD84F004000FB0BDE8F08FB5
:1026BC0005200021F5E78178022904D101218170E0
:1026CC00002021F03BFD84F48050EEE784F40060A0
:1026DC00EBE721F057FDD0B15F4F05463878013854
:1026EC003870000616D05D4E4FF48041307823F0E0
:1026FC00D7FA30B9386929F013FE10B928781FF0D1
:10270C00BFF83078402143F698222AF09EFA5248BE
:10271C00007810B90B2029F0FBFD84F04000C4E7D1
:10272C004F49097801390129BDD8032101600120E5
:10273C00B070012020F0A4FE01208DE7464EDFF89A
:10274C001C914FF0000804AD4FF0000B06F1080788
:10275C003F685FB3D7F804A09AF800000028F7D0C0
:10276C00F028F5D8032100222B4623F010F900287D
:10277C00EED00698018821B101394FF0010B018090
:10278C00E6E74FF4407086F836802AF02DF999F878
:10279C0000000AA92AF0E9F9324886F83680016867
:1027AC000029D5D09AF800008847D1E799F80000A5
:1027BC005FEACB710BD04FF400514FF47A722AF0D0
:1027CC0044FA08E012F08AFE84F480406DE74FF47E
:1027DC0000511EF003FA84F4005066E7F06840687C
:1027EC004078C0070CD10E2029F092FD08E040F291
:1027FC0009302AF0F9F8194800780AA92AF0B5F935
:10280C00F06840684078C1073FF44DAF174909683C
:10281C00C1B128781FF034F810B10E2029F078FDE2
:10282C000E4D0C20402143F69822307028782AF067
:10283C000CFA40F20A302AF0D7F828780AA92AF0C4
:10284C0094F930E780073FF52EAF0E2029F060FD9C
:10285C0029E700BF606D0020542000200A6E002084
:10286C001C2500206C260020AE260020A82200206B
:10287C0054F0020078260020C5260020C05E0020FF
:10288C00386D0020AC6800202DE9F04F89B024F0A1
:10289C00D1FADFF810158122DFF81485DFF814A5C2
:1028AC00DFF82045DFF814E50A70DFF8FC14086047
:1028BC00DFF8F804FF2101700020DFF80415A8F8F8
:1028CC0000008AF80000DFF8F0040968007891F83D
:1028DC0008B04FF6FE718EF8000059448AB2A16818
:1028EC00D1F80031DB899A4200F267810422DFF8CB
:1028FC00DC54A8F80020DFF8D02412689668330E58
:10290C00CEF80C60C6F301592B706FF0FF0303EA8D
:10291C001627B3B2D1F8B86047EA1327AEF80470A3
:10292C0036781EB9B9F1020F00F04781B9F1030FE7
:10293C0000F043811B0A03F0070316B1002B00F0D3
:10294C003C81DFF88CC4042B9CF800C008BFBCF1A0
:10295C00000F00F032813EB1DFF878643678862EB5
:10296C0002D1022B40F02981BB0416D4BBB203F078
:10297C000703022B08BFBCF1000F20D0DFF8541462
:10298C000978862909D10020764624F08BFADFF8E5
:10299C004004B64690F800C0307800284ED0BCF108
:1029AC00000F4BD1012800F0088103283FD00228EA
:1029BC0044D1BEF80400400740F0FF803EE0D1F85F
:1029CC00D40090F88300022800F080802746052070
:1029DC00147BF246A946A8F8000029F0F1FD054643
:1029EC00DFF8F003007886286DD1B868016C0968AF
:1029FC0011B9D0F84C05804760B2002100262AF0AE
:102A0C0004FAB9680A6C12685077086C006886770B
:102A1C00086C0068C47728462AF0E7F8BAF8041066
:102A2C0099F8000001F010011FF0AEFC4EE0BEF86A
:102A3C00040000F00700032840F0BF80BEF804003B
:102A4C00010700F1BA80810402D4810500F1B58040
:102A5C009EF80E20C2F38107012F00F0AE8096097C
:102A6C00012E00F0AA80B9F1010F11D840F002013B
:102A7C0001F0070103290BD117B93F2A40F29D80C1
:102A8C0037B9A168D1F8AC100978002900F095800D
:102A9C004FF6FB71B9F1020F0BEB010C19D1CF4BB7
:102AAC00D95D9B5D03EB01090023402AB7FA87F23D
:102ABC0038BF012352091A40430616D4002A08BF16
:102ACC0009F1020915E028462AF08FF828F0CEFB10
:102ADC0075E0C14B402AD95D9B5D03EB010908D31E
:102AEC00420648BFA9F1020903E0002A18BF4FF0C3
:102AFC000209C0F300205FFA89F11FFA8CF30A1A5D
:102B0C008EF801009A4258DC60440391B346401A97
:102B1C00A168AEF806007430D1F8501280B2884724
:102B2C00A6490028886048D07421CDE9019729F086
:102B3C00F7F9A24F0020B870A548007820B9387971
:102B4C0000F020008AF8000078789AF80010DFF87E
:102B5C0078C24FF000092E4600299A493DD0002832
:102B6C004FF000003AD1B88800F00700032807D0D6
:102B7C00012832D18868D0F8D40090F8820060B374
:102B8C00C8684069007818B129F016F8FE280DD0F5
:102B9C008C488068D0F84C02804738B989488068E6
:102BAC00D0F844028047002800F0F780834F0120C2
:102BBC00B870DFF814C22E4610E028F049FE29F058
:102BCC00FFFC814900240A6813681C7112680A60B2
:102BDC002AF00BF809B0BDE8F08F0020BC6804F1B6
:102BEC00740184F830B06160A1657978BB88FA888B
:102BFC000029A381029B228184F83A30337808BFE4
:102C0C00994697F80EB084F84990019DA4F85C2081
:102C1C00FF22B8F80030A273CBF301195E1A797B4E
:102C2C00A8F8006001F0780160F3820101EB090063
:102C3C002074280600F0AE80DCF8000004AF039A84
:102C4C0010FA86F000F1080138462AF00BF956FA12
:102C5C0085F0CBF38105A8F80000207C00F040083B
:102C6C00CDB3B9F1020F06D1B8F1000F03D0B4F80F
:102C7C00440004AF06E0BDF810000237A4F844008D
:102C8C00A4F84200564EF189884203D04FF6FF71EA
:102C9C0088425ED1032D11D104F1320039462AF05D
:102CAC000DF8464CF11CA068323027F0EBFB45497F
:102CBC0000284ED094F80EB008370EE037F8020B0F
:102CCC00B1898842608606D04FF6FF713B4C884232
:102CDC003C493ED101E03B49384CBBF1400F20D37D
:102CEC00B9F1020F06D16DB9B8F1000F0AD1334812
:102CFC00806803E0A068017C490603D43988023758
:102D0C00A0F84210BBF1C00F06D32C4C3946A0687A
:102D1C00283029F0D3FF03E0284C3888A1680885B7
:102D2C0028498968A088D1F8AC201278B2B1B9F1E1
:102D3C00020F13D200F00700012802D003282FD174
:102D4C001E4C6DB9264AA368D289B3F8423093421F
:102D5C0006D01BF0F6FD1BF0FDFB30E700F0070082
:102D6C00032806D0012815D1D1F8D40090F88200A0
:102D7C0080B1A068D1F848128847104A50B9002099
:102D8C00D17B9070907BC1F3011100F07800084466
:102D9C00916808740BF02EF811E7084FB87808E723
:102DAC00064CDDE71B6E0020A86D0020206E002075
:102DBC00F26D00201E6E00201D6E0020FC230020F2
:102DCC00DC6D00200C010020246D00202D6E0020F5
:102DDC002C6E0020236E002008F0020004F002008C
:102DEC00506C00202DE9F04F97B0DFF810850546A8
:102DFC00DFF80C6598F800000328307040F04C8127
:102E0C00002088F8000030700DAC204629F062FFDD
:102E1C002046002127F0A3FFDFF8E894B0603A21A8
:102E2C00484629F07DF84FF0FF30A9F81400C9F896
:102E3C001000C9F80C0025F00FFE0020294620F0E8
:102E4C0085FF06F11001F06029F0DEFED6E90502DF
:102E5C00DFF8B474B0FBF2F1C9B2032928BF032127
:102E6C0089F800103970B2F5005F40F01281B0EBB8
:102E7C00413FC0F00E81F068002800F00A814FF449
:102E8C000050FF224FF000084FF0885BA9F80600B5
:102E9C00FF2089F8032089F8058005900020089010
:102EAC0000200B9000200990002007900020069035
:102EBC0000200A9000200C90FF200290FF2004902C
:102ECC00FF200390CCB2A04580F0E9805FFA88F631
:102EDC00002116AA0423304629F05AF9DFF83044B1
:102EEC003046002115AAA0473046012114AAA0475C
:102EFC003046022113AAA04716996FF06F0050FAC2
:102F0C0081F2C8B20E2A06D8012303FA02F245F266
:102F1C0001131A4203D1A0F1FE02022A04D242F29A
:102F2C008352B2EB914F1ED0304616F0C5FEDFF83F
:102F3C00D0130028087040F0D2803046002116AA29
:102F4C00042329F025F9DFF8C8433046002115AADF
:102F5C00A0473046012114AAA0473046022113AAEB
:102F6C00A0471699C8B208EB4802CA463D4609EB81
:102F7C008209C1F30142090A4C46FD2804F8160FD8
:102F8C0061709DF85610E270A17001D9102135E0E6
:102F9C00BDF854104FF6FF7291422FD10EA823F0BA
:102FAC00C9FB304600214FF088524FF400534FF4C8
:102FBC00005729F0EDF86FF0030313FA87F7B8B256
:102FCC0050F80B104A1C01D10328F6D80122012617
:102FDC00D3B2042B06D8CBB2FF2B18BF1646013246
:102FEC00090AF5E740F80B10CA480E9900684268C8
:102FFC00C948904757FA86F081B22078A9F81C107E
:10300C009DF85210702889F81A10BDF85010A9F8C4
:10301C001E109DF84E1089F81B10BDF84C10A9F825
:10302C00201011D07828D14614D07C282F4616D0E9
:10303C007E281AD0FE281FD0FF2823D10898CDF85F
:10304C000C800130089020E00A98D1462F460130C0
:10305C000A901AE006982F460130069015E0079862
:10306C00CDF81080013007900FE0099801300990DD
:10307C001FFA88F0029008E00B98CDF8148001300C
:10308C000B9002E00C9801300C90397808F1010893
:10309C0018E7012088F8000017B0BDE8F08F0C98F5
:1030AC00974E00060BD10B98C0B2012807D80A988E
:1030BC00C0B2012803D80998C0B2012811D993488D
:1030CC00042200240270CAB2E0B2904210D216F070
:1030DC00F3FD31780134084339783070F3E7884ECA
:1030EC001BE0089BD8B2A04219D18848002202707C
:1030FC00002089F8030089F80100481E7E2189F818
:10310C000200B9F81C00A9F80600002024F01EF9F2
:10311C0099F80200FE2124F019F93078BCE70A98DE
:10312C00000624D00B98059A000603D1039A1806C2
:10313C0000F08480754802210127D5B289F802205D
:10314C00017017FA82F0B0FBF4F101FB140089F85E
:10315C000100284616F0B0FD30702846FE2124F000
:10316C00F5F889F80570002000F0D8F8D5E70B9831
:10317C00059A000621D06548012189F802200170CA
:10318C0011FA82F0049AB0FBF4F101FB140091B235
:10319C00FF2989F801001FD10299FF2919BF89F86D
:1031AC00031001EB410089F8030000EB400009EB30
:1031BC008000808BA9F80600AFE7DDE906201043FC
:1031CC0000063FF47CAF25F01BFCA04280F085800C
:1031DC004E48032101703EE0480089F8032010FAA4
:1031EC0082F009EB8000818B1829A9F8061094D382
:1031FC000739D0B20EAA89B218F066FC9DF84300CC
:10320C004007B0D5B9F80610BDF84620002399F850
:10321C00030000930323891A0EAA073989B208F018
:10322C00FDFD00287FF479AFBDF8441000293FF470
:10323C0074AF9DF848001FF0E9FE6EE725F0E0FB47
:10324C000621A042314838BF03210329017002D066
:10325C00062952D061E725F0D3FB054689F80C000E
:10326C0000EB400009EB8000408BA9F80D000FF03B
:10327C00B9F939782844B0FBF1F202FB110089F856
:10328C0002000130C2B2B2FBF1F202FB110089F86C
:10329C0001007C2024F074F8FF2812D17E2024F049
:1032AC006FF8FF280DD1FF2024F06AF8FF2808D111
:1032BC00782024F065F8014699F80100FF2918BF21
:1032CC000846C1B289F80300490051FA80F009EBB5
:1032DC008000808BA9F806001AE70898000609D030
:1032EC0099F80200FE213C46374624F02FF824784A
:1032FC00039A40E7054806210170FEE7A926002045
:10330C000822002000660020026E0020116E0020B2
:10331C00DBC30200D8010010004003402DE9F04F40
:10332C009BB00446DFF80805406818B180470028B8
:10333C0000F03C82DFF8FC04DFF8FCB40B940DF1D8
:10334C00300A4FF0F8080078411E002C099118BF84
:10335C0001218BF80F109BF802900BF118049BF8CD
:10336C000110002700250A91C0B287421FD2B9452F
:10337C0017D0FEB2002152460423304628F008FF35
:10338C000C9810F4403F40F0040018BF0135C0B257
:10339C007C2806D130460621F82227F08BFD84F8D4
:1033AC000080DFF890040C3401370078DCE7E9B2D8
:1033BC0001380022884204D19BF80500002800F057
:1033CC003282DDF82CA05046BAF1000F08BF102055
:1033DC00049013AF00200390DDE909560024280463
:1033EC0000F0E6819BF80F0010B901208BF80F005C
:1033FC00F0B200210CAA04234FF0000828F0C8FEFC
:10340C000C98BAF1000F1DD010F4403F17D04FF4B8
:10341C000050DFF820140134013DABF810009BF88C
:10342C000F00097801388BF80F00012050FA86F054
:10343C00B0FBF1F202FB11068BF80D60CFE7A04652
:10344C00CDE90956C0B20A9D0024702803D0E8B219
:10345C00702123F07BFF5FFA89F600210CAA04236C
:10346C00304628F095FE9DF83000FE2803D03046FB
:10347C00FE2123F06BFF30460621FE2227F01AFDB9
:10348C004FF400500BF116018BF80C908BF80D508B
:10349C00ABF814405A46ABF81000FF208BF80E0026
:1034AC00E8B2400050FA85F0D57B01EB8000B0F813
:1034BC0006B0DF4804707000A2F812B050FA89F020
:1034CC0001EB8003FE20194601F8020F33F8060FBA
:1034DC0002910790D7480193047812A823F02AF997
:1034EC000A980A9A089655FA80F0013890FBF4F184
:1034FC0001FB14000090D5B20A92B54200F04A814B
:10350C00A81BB0FA80F0400905900020069000201E
:10351C00C00740F093801FFA8BF0162871D9C4486D
:10352C000078002840F03C81ABF1070A28460DAA30
:10353C001FFA8AF4214618F0C7FABDF8426006F16A
:10354C001000A0421AD89DF83E00962816D19DF87E
:10355C003F00C10701D1800703D40020AAEB060B62
:10356C002CE0AAEB06009DF83D2031462B4684B298
:10357C0020461BF07EFD20B3ABF1080A1FFA8AF03F
:10358C001728C0F00D81AAF11604362828463A46B1
:10359C0088BF2024AAEB040AA3B21FFA8AF128F0F0
:1035AC00F7FD2004EAD017FA84F010F8010C9628E5
:1035BC0001D0013CF5E704EB0A0B0020DDF82CA050
:1035CC00A6E7F01D83B2079813FA80F1B1F5005FFE
:1035DC0001D90120F2E780B28B469A4918440A1AA5
:1035EC002846214628F0D4FD069801300690BBF5FC
:1035FC00005F07BF01204FF400515946002007918E
:10360C00ACE7069810B18C4928F020FF0098C0B2A6
:10361C00854200F0C2800A990120089E50FA81F080
:10362C0084490978B0FBF1F202FB1102824902EBEA
:10363C00420001EB8000B0F81CB05CE7069810B1BA
:10364C007D4928F003FF0020DDF828900590784C88
:10365C002078002840F0A48007981021C0F5005273
:10366C00103883B20898C1F2001223F07FF8217849
:10367C00084312992070714800684268704890475E
:10368C00059888B16B4800782918013991FBF0F244
:10369C0002FB101968495FFA89F0400050FA89F072
:1036AC0001EB8000B0F81CB063480799089C01231B
:1036BC00A0F814B08346018280F80E900198BBF9F3
:1036CC00122001809BF80D10204625F0AFF9BBF9B4
:1036DC0014209BF80E102046022325F0A7F9BBF806
:1036EC001000BAF1000FC0F5005004D004998842C4
:1036FC00A4BF01210391049988424FF07C01B8BF0B
:10370C007821089C204623F021FE0EF06BFF054625
:10371C009BF80F000621FC22401B8BF80F00204663
:10372C0027F0C8FB0299FC209BF80E3008709BF820
:10373C00021015FA88F00A9301443E480078B1FB58
:10374C00F0F202FB101909F101018BF80290CAB2D8
:10375C00B2FBF0F202FB10118BF8011003EB4301EA
:10376C000BEB8101898B102906D10A990131B1FB30
:10377C00F0F202FB10100A900998401BBAF1000FEE
:10378C0009903FF429AE039880F00100C0077FF444
:10379C0023AE0DE00120354658E7DDF8009056E7E2
:1037AC0026481299006842682548904700223AE062
:1037BC007C2023F0E5FD0446FF281DD17E2023F05C
:1037CC00DFFD0446FF2817D19BF8014004EB4400B1
:1037DC000BEB8000807DFF280AD016489BF8021066
:1037EC0000780144013991FBF0F202FB101403E064
:1037FC0020467E2123F0AAFDE0B2FE218BF8034087
:10380C00400050FA84F00BEB8000808BABF8060084
:10381C009BF8020023F09AFD00208BF80500BBF802
:10382C001000C0F5005210B21BB0BDE8F08F00BF05
:10383C0008220020026E002000660020D801001033
:10384C0000400340002000112DE9F84305460C46CA
:10385C00480414D4A00025D4A0075FD4600500F15F
:10386C008180200500F10881200700F13D81600076
:10387C0040F1F8801CF034F824F08044F2E028F099
:10388C009FFEDFF824140F6D3FB1D7E90A1202F046
:10389C00E04201F00A0189184BD029F0A6F924F472
:1038AC008044DFE0BB48DFF80474016841F080011C
:1038BC000160B878012804D1042023F0AFFD00206A
:1038CC00B87028F07DFE0646B348406D01680420B0
:1038DC008847DFF8E0130A68904219D12A7EBAB102
:1038EC00FA68AAB1DFF8C003806C002800F097805A
:1038FC00C16840F603020988914206D0C06840F6C0
:10390C0004010088884240F08A8005F1140088E0A8
:10391C0040F6C4120860C5E9042284E00BF078FC80
:10392C00DFF88403006C002840F09D8024F0020432
:10393C0098E0D7E90A65D7E90A12AA43B143C7E967
:10394C000A1229F052F9B8680028A8D056EA0500E6
:10395C00A5D0D7F808C03869B7F9301032462B46D5
:10396C00E0479CE728F02CFE054626F0B1FA00282B
:10397C0000F0B780CC48876B002F00F0B280DFF8E6
:10398C002C830420CC49002288F81800C64828F063
:10399C0006F829F054F9C94829F024F9C4480068FC
:1039AC00006B8047C8F810000125042088F80250ED
:1039BC0024F040FB386990F82810C8F80400490737
:1039CC0003D5436A04210022984701201DF0F8FD1D
:1039DC00D8F80400457615F011F9D8F80400816880
:1039EC000B461A465B684BB11E88A6F60306072EDB
:1039FC00F7D805FA06F616F0830FF2D0537B03F0D6
:103A0C00F003013353730023FD6853602D88A5F632
:103A1C000305012D00F28A80C8F810309FE005F1F3
:103A2C00100020F085FF304629F0DFF824F01AFB57
:103A3C0078B12E6A28466FF4807100224FF0007323
:103A4C00B0479948806B10B11BF04AFF01E044F07D
:103A5C000204EE692846002100224FF08063B04733
:103A6C0024F0005434B1984821462830BDE8F8437E
:103A7C0029F097B9BDE8F8838C4EB078012804D1B1
:103A8C00042023F0CBFC0020B07024F0EBFA38B10A
:103A9C0070686FF4807100224FF00073056AA847BC
:103AAC00306950B182480068006B80473269716898
:103ABC00801A000BC860002030617B4D81490022C8
:103ACC00284627F06CFF02203076286C20B17E4807
:103ADC000221283029F065F91BF002FF24F4006460
:103AEC00C0E729F0ACF841E028F06AFD054626F065
:103AFC00EFF9A0B1DFF8B48198F8000000070ED4FC
:103B0C0098F9000000280AD4684615F057FB08B154
:103B1C00009820B1DFF8B49199F8610048B329F00E
:103B2C008EF81BF0DDFE24F008049BE7034633F807
:103B3C00385FA5B190F8445090F8456005F0F00559
:103B4C0080F8445006F0F005013580F8455000250A
:103B5C005360C5634587507B00F0F00050735848A4
:103B6C000022C2610160012026F042FE24F4806430
:103B7C0078E700260127602E10D009EB0600817A29
:103B8C0031B18772407A07FA00F0C0B223F060FCC2
:103B9C002036F0E7CC2108408C010010032088F877
:103BAC001800464829F01EF829F049F8444F3E4DBC
:103BBC000022786900207861F968F8602846444949
:103BCC0027F0EDFE3A480068006B8047D8F80C10DF
:103BDC00D8F82020411A02EB1130B0EB113F38BF5E
:103BEC004FF0FF3098F82410C8F8200021B1D8F815
:103BFC000810B0EBC12F20D926F00AFEB8B140F660
:103C0C000900414621F83C0F002048804A7B02F015
:103C1C00F00201324A730A7B02F0F0020A73486028
:103C2C00F8613960B8F83E0010F4406FFAD000200B
:103C3C00C8F82000012088F8240020F063F82548FB
:103C4C00002101600220002126F0D2FD022023F089
:103C5C00E5FB102013F0A4FE98F8010020B9D8F869
:103C6C000400503029F099F81B48807810B90D20C9
:103C7C0013F096FE98F8250028B1002088F825004E
:103C8C00052023F0CBFB002088F818001348C8F857
:103C9C001C000220B5F85610B5F85420914208BF0C
:103CAC0007201AF0CBFF3CE7A81F0020481D00207E
:103CBC008C010010C4250020B99E0200B0630020C6
:103CCC0000100440192E0100E81E0020385F00206F
:103CDC0051F901000000046058EF020001280100B6
:103CEC002DE9F04FAFB004460020ADF8280094F851
:103CFC002400012809D1DFF8380494F828108078C2
:103D0C0031B1002800F0FD8102E0DFF82404807856
:103D1C0048B9207D00F0FE00022804D12FB0BDE888
:103D2C00F04F1BF063B8DFF808743878012806D11F
:103D3C00DFF800043979007E814240F0CD80DFF855
:103D4C0000544FF4FA60E060286828F0A9FB18B121
:103D5C00E1680844E06007E0E168286828F011FF9A
:103D6C00DFF8E00329F027F894F825008DF86C00B3
:103D7C0048B1022809D11BA804F11801082204300B
:103D8C0028F00EFB01E0E06A1C900DF12B051BA83E
:103D9C000AAA294619F0AAFC0646D0B99DF8381093
:103DAC0094F8260001F0030181420DD105F10E00BB
:103DBC0004F13401042228F0F3FABDF82810022093
:103DCC0041222B461EF006FC9DF86A0008B1DE4924
:103DDC000870B878B8B3012840F0938194F8380093
:103DEC00E3280DD1B86818B18047002800F089810C
:103DFC00F86818B18047002800F0838194F83800E7
:103E0C00E22804D194F82800002840F07A810020A0
:103E1C00002E18BF054695F80D801EAE30460021C9
:103E2C00282228F012F901A80021032228F00DF90C
:103E3C0094F83800E32840F0C3809DF8041041F05A
:103E4C000802E320ECE0207D042800F25A810121D5
:103E5C0001FA00F010F0130F00F0538101A80021BB
:103E6C0024224FF0000828F0F0F81EAF04F1180BD4
:103E7C0004F12C09BD1C07F1060AB8F1040F45D852
:103E8C005FFA88F0394623F0F2FE06460D2820D062
:103E9C000A2E00F0908094F825009DF8781041408F
:103EAC00490701D0022614E048B94846514604227D
:103EBC0027F084FA002840F0338194F8250002287A
:103ECC0007D158462946082227F078FA002840F0F6
:103EDC001B8108F10108D0E794F83800E32840F082
:103EEC001081954828F065FF00283FF428AF924CCC
:103EFC00204628F062FF9148C821006828F041FE56
:103F0C0020462FB0BDE8F04F28F055BF002E52D1FF
:103F1C000020616B102508269DF879209DF88530CE
:103F2C00069194F838108DF81C109DF8781005EA5D
:103F3C00D10506EAD101084402F00101C3F3820263
:103F4C00284440EA4110BDF8041040EA8310C0B286
:103F5C00084394F82910002918BF083202F15001C7
:103F6C0040EA0120ADF8040094F8400058B18DF8F7
:103F7C001D0028F074FF089028B194F8402004F13B
:103F8C00410128F00DFA6B48C08AADF8240094F971
:103F9C001500014610F16D0FD8BF6FF06C0128F0C1
:103FAC004EFAC8BF3B21A07D002818BF012041EA72
:103FBC00C0108DF82600E17D01A802F09BF8A0E06E
:103FCC0094F8251011F0070119D0022920D106F11F
:103FDC00080004F11801082228F0E2F994F83010D6
:103FEC0094F8380002228DF888109DF80410E3280C
:103FFC0062F302018DF804103FF421AF0AE0E16A8C
:10400C001F919DF8041021F007018DF8041001E0B8
:10401C009DF8041094F8292021F0080141EAC2020D
:10402C009DF80510022302F00F0263F3051194F8BA
:10403C002630022B16D394F82760012E17D0D6B950
:10404C004FEA980606F00706042E6DD8012707FAEA
:10405C0006F616F0160F67D0C8F3820621F017018A
:10406C00314408E0002B08BF21F0170103E041F0B8
:10407C00040121F0130163F30512237D032B03D1FB
:10408C00E36B41F0080127938DF89000606B23904F
:10409C0001F00700C9B242EA8010C1F3C00240EA45
:1040AC004220C1F30012C1F3401140EA822040EAE1
:1040BC00C120ADF8780094F8400020B18DF8910043
:1040CC0004F1410025901B482B46C08AADF898009E
:1040DC0094F91500014610F16D0FD8BF6FF06C010B
:1040EC0028F0ADF9C8BF3B21A07D002818BF0120E6
:1040FC0041EAC010E17D8DF89A001EA81BAA0AF0B7
:10410C003FFB2FB0BDE8F08F01A8594608220830BC
:10411C0028F046F994F830008DF814000220F8E6E7
:10412C00D9F800000290F3E601F0E801A3E700BF24
:10413C0058230020C05E0020C0640020906D002039
:10414C008C6D00207C640020F92400202DE9FE4FAA
:10415C008846080426D45FEAC87004BF0020BDE876
:10416C00FE8FE548056828F0D6FD044628F0D1FD01
:10417C0060434FF47A714FF6FF72B0FBF1F14FF6DA
:10418C00FF70002D00F01A812B886C88CB1A9BB223
:10419C009C4240F21C81E31A94B2A342B8BF1A4667
:1041AC00ED68EEE7DFF840A3CDF804809AF8000044
:1041BC001CF042FD002800F0FC8006460078012827
:1041CC0040F0EC80DAF8041096F83390D6F814B07E
:1041DC0096F8138021B148468847002840F0DE80CD
:1041EC00718896F83100022225F060F90546002806
:1041FC0042D0287A297CA0F10108FF2900F0BB806D
:10420C00707F4F46C00718BF0027E97C287D01440A
:10421C00B94204D8E974FF2101FA00F06874A96965
:10422C00A87C96F83020896A10FB0710F16A27F0F9
:10423C00EFFF287D697CB7FBF0F202FB10700122C6
:10424C008240D2B20A436A74C8457CD196F83010C9
:10425C00AB7C13FB0713A9698B844FF4FF7303FA30
:10426C0000F0C0B21043FF2868746CD1287C1DF09C
:10427C007BF9FF2028747FE0707FC00700F08E80F0
:10428C00B07F28F035F8002800F0888004461C2008
:10429C0028F073FD002800F081801C21054627F0D2
:1042AC003FFEB07F02A926F0A9F89DF80900022173
:1042BC002875284626F03CF9708896F8312096F837
:1042CC00301096F83330A880287DEA71FF2202FA6C
:1042DC0000F0687460680078A9742874302013FBAF
:1042EC00010080B225F040FD0028A8615DD0044695
:1042FC001A20B11C2060708CA080A01D26F0E4FE5A
:10430C00F27F04F13000B17F96F82830C4F81CB06D
:10431C0084F81980A062307CE273744A217563754D
:10432C000121A075928C2282F28EA285F28C62827F
:10433C00B6F81100A4F817009AF8000085F8089058
:10434C001BF0A4FF55E728F0E6FC044628F0E1FC3E
:10435C0060434FF47A71B0FBF1F0654928806348F3
:10436C00097800794843642148436249097800FB85
:10437C000100688000E04F46E87C297D6A7C01449E
:10438C000139B94218BFFF2A0CD186F83300708866
:10439C0006F11C0186F8342019F00FFB304626F08C
:1043AC0093FC03E7C845F9D1EFE7284626F0D0F88F
:1043BC00F4E7019880F40040BDE8FE8F92B282428F
:1043CC004BD049480121007828F03FFC45E0A87902
:1043DC00022806D1287CFF2837D0A86926F074FC67
:1043EC0033E028F098FC044628F093FC60434FF42B
:1043FC007A71B0FBF1F03F49288095F838000978C4
:10440C0088421BD295F83620FF2A06D195F8372022
:10441C00013085F8380085F8362095F8351095F878
:10442C00394082F0FF0300200126C7B2A7421DD2FB
:10443C0006FA07F71F4214D10130F6E7EA8BA87E83
:10444C0095F82A10E92321F0FDFC284626F080F887
:10445C002548012100781BF019FF88F00100BDE808
:10446C00FE8FFBB201441A4385F83620AB8F95F8CA
:10447C003440C8B204FB10339EB2A64203D2FF22D2
:10448C0085F8362002E0FF2A08D12346184A174E39
:10449C001278367972436426724302E095F83A201A
:1044AC0023466A802A8D0E0606D022F02002444351
:1044BC002A852A6C224404E042F020012A6C2985CA
:1044CC00297A85F82E10E9796A6285F82D10D9B20F
:1044DC0069840549496811B188470028B8D105F1AC
:1044EC00100005F04FFBB3E738250020C05E00201C
:1044FC00D0260020D62600200C5000202DE9F04FAD
:10450C00C3B00DF1450B884601469146584628F03C
:10451C00CFFB08F0080500260DF1040A042E39D84B
:10452C00F4B25146204623F0A2FB0D2803D00746D7
:10453C000A2801D17DE17DBB204659461CF0BEFC0A
:10454C0001360028EAD0002D51D10BF137010DF1C5
:10455C008600022227F024FFBDF886009DF83A1051
:10456C00ADF8C800C80700F083800AF1370732A9FC
:10457C000222384626F022FF9DF83A10012877D106
:10458C0001F0FE00FF2104228DF83A00384627F096
:10459C005CFD6FE001274CE10220214641225B4685
:1045AC001EF018F80746B4480BF10B0128F074F80C
:1045BC0068B90BF13701204628F029FB38B90BF10B
:1045CC003B01204628F023FB002800F032810C2010
:1045DC0028F045FC002800F0198128F00FFAB9F1F9
:1045EC00000F18BF4FF0010984F80A9005E19DF8FF
:1045FC004500400661D49DF84600C00700F0A48039
:10460C0032AF0DF14501384628F052FB0DF1860909
:10461C0001A9484628F04CFB9DF8BC00810700F12D
:10462C00288110F001054FF03B0007F1370108BF5E
:10463C0037200422484427F0B3FE0220002D08BF87
:10464C0001209DF8BC10084349468DF8BC0001A818
:10465C0028F02EFB08F060009DF805104038B0FAE9
:10466C0080F001F0FE01400908448DF805006BE074
:10467C00880733D44FF0FF300BF1220627F0C0FD32
:10468C003846314626F09AFE0AF12C05E0B338463E
:10469C0029460A2227F084FE32AE28460A223146E9
:1046AC0027F07EFE3046394628F0C0FA002800F08C
:1046BC00B98001A827F0A5FCB4E04FF0FF3027F03B
:1046CC009FFD32A8394626F079FE0BF1220930B352
:1046DC00384649460A2227F063FE27E00AF13B06DA
:1046EC0032A90222304626F069FE9DF83A100128C4
:1046FC0040F08E8001F0FD00FF2104228DF83A007D
:10470C00304627F0A2FC8DE02846314628F08EFA80
:10471C00002800F0928032A928460A2280E0384610
:10472C00494628F083FA002800F0958008F06001D3
:10473C009DF804006039B1FA81F100F0BF0049091D
:10474C0040EA81108DF804009DF84600810608D5DA
:10475C000AF10B000BF10B01022227F021FE9DF850
:10476C004600400613D59DF805000BF10D01012202
:10477C0040F040008DF805000AF10D0027F010FE06
:10478C000AF112000BF11201102227F009FE9DF81C
:10479C004500800605D59DF8040040F020008DF8FA
:1047AC0004000AF10E000BF10E01042227F0F8FDB3
:1047BC00BDF88400214641225346ADF84300022047
:1047CC001DF008FF07462C480AF10B0127F064FF87
:1047DC0058B90AF13701204628F019FA28B90AF11C
:1047EC003B01204628F013FA18B30C2028F037FBB5
:1047FC0060B128F003F90120A0722048214600780E
:10480C0028F060F9204628F0D4F912E0102710E0C7
:10481C0041F00100314604228DF83A000AF13700CC
:10482C0027F0BEFD01AB0220214641221DF0D2FE35
:10483C000746384643B0BDE8F08F32A8394628F019
:10484C00F5F90128EED132A8294628F0EFF9012814
:10485C003FF42FAFE6E70AF12C0732A80A223946BB
:10486C0026F0ACFD00287FF433AF3846494628F0DB
:10487C00DDF90C27DDE700BFC05E0020126E0020C2
:10488C002DE9F04F8FB00C46080430D4A00448D466
:10489C00A00652D4E00600F10B81600600F11A81EB
:1048AC00200600F11E81E00500F12081200500F1B9
:1048BC002281E00400F13581600400F13C81A00705
:1048CC0000F15081A00500F15E81200700F16881A4
:1048DC00600500F16B81E0034FF0000540F1F680BC
:1048EC001DF096FFBA48C57084F48035EEE0B648EA
:1048FC0000781CF0A1F988B10178B44A0546002073
:10490C00582808D0135C08308B42F9D1104450F869
:10491C00041C28468847284626F0D6F984F400451E
:10492C00D4E01FF0E3FC28B10546FDF781F82846DA
:10493C0026F0CAF984F40055C8E0A34F202138783A
:10494C0021F0AEF9DFF888820125D8F80810084369
:10495C0017D028F0E0F9054628F0DBF968434FF44E
:10496C007A71B0FBF1F0D8F80810401A4FEA5005F4
:10497C0038BF6FF00045002908BF0D46002D00F030
:10498C00AE8000200421002224F0ACFF06464FF03C
:10499C00060A4FF0FF094FF6FF780DF1080B002EB9
:1049AC004DD0304604210022374624F09BFF0646AA
:1049BC003889401B38BF002038810004EFD1B87B08
:1049CC00D0B301280AD17889400707D4386887F812
:1049DC000DA0B721407B1FF041FCE0E739685A4637
:1049EC008DF80690ADF80480086AC97F0EF006FCBD
:1049FC0001281BD1B87BB97A8DF838000907788A61
:104A0C0040F08002ADF8362006D540F4C070ADF809
:104A1C003600387B8DF83A00786910B1007BADF820
:104A2C001800584601A9002203F0BAFC387B87F81D
:104A3C000DA017F0E5FEB2E701207873AFE7DFF8C1
:104A4C009081614F25F0D8F800200121002224F03C
:104A5C0049FF18B1387820211BF018FC00200421E4
:104A6C000022002624F03EFF60B3068904210022B8
:104A7C0024F038FF28B10289B1B2914228BF164602
:104A8C00F4E7A8B2B1B2814217D9D6FA55F0202179
:104A9C0080B24200387828F0D8F828F03CF9054666
:104AAC0028F037F968434FF47A71B0FBF1F609E05E
:104ABC0009F012FF84F0100508E0387820211BF073
:104ACC00E5FB0026C8F8086084F0200528460FB0E6
:104ADC00BDE8F08F0DF012FF84F04005F6E70025DD
:104AEC00B0E726F04DFD84F08005EFE724F07EFD65
:104AFC0084F48075EAE71DF0A3FA374800780128A2
:104B0C000CD13448007848B14FF47A7100FB01F2B3
:104B1C002D484FF40061007828F094F884F4006577
:104B2C00D4E72B48017819B1002101701DF088FAE7
:104B3C0084F48055CAE72A48006880B1274909786F
:104B4C0001290CD180472748006800B180471E48D6
:104B5C004FF480414FF47A72007828F073F884F4A3
:104B6C008045B3E72048007890B102AD284627F085
:104B7C00D0FF27F031FD1D490B781D490A782946D5
:104B8C001CF09AFC09E017F0F1F984F400759DE72C
:104B9C001848418B012028F0E6F884F0020595E7CF
:104BAC000B48012184F0080581708FE712480078CA
:104BBC00022808BF16F017FC0E480121808C28F043
:104BCC00C4F884F4806581E7036E0020A0E802003D
:104BDC00EC240020DB260020DC260020DA26002036
:104BEC003C22002048220020B5260020DF26002091
:104BFC00E0260020C05E00201C25002070B586B089
:104C0C000C46080403D4600433D400203EE0C648AC
:104C1C0000781CF011F8B8B305460078A0F1D0016B
:104C2C0006292BD9A0F131010629C0F08A801A2857
:104C3C0044D0FD2857D0FE286FD1162025F094F8CB
:104C4C00002800F07E8006460230142127F068F917
:104C5C00932030802A796878A978EB883381307179
:104C6C003174012A18BF0222B271E978A878317523
:104C7C004DE022F09FFB84F4804007E00120884047
:104C8C0010F0750F04D05CE084F4004006B070BDE9
:104C9C0001294BD1A54E6878B178814251D006F8E4
:104CAC00020FA34B4FF000700021324623F0AAFCF8
:104CBC0016F8010C9F4981F8680042E0302025F07D
:104CCC0053F800283DD03021064627F029F99220D0
:104CDC00A91D3070A87B0328307169D1B01D082242
:104CEC0027F096FA66E00A2025F03EF848B306460F
:104CFC000020C6F80600C6F8020091203080A87883
:104D0C006978EA7870713171B271A988318126F0B5
:104D1C004BFD002840F084808AE02846FBF788F998
:104D2C0078B1A87829461CF01FFCADE7E889A0F5FE
:104D3C000041062913D8DFE801F0087F8A0498B0F7
:104D4C00BB00284625F0C0FF9EE728461BF0FEFA64
:104D5C000028F6D06988824B06460120B2E048F262
:104D6C003601884200F0B58048F22001884200F0FC
:104D7C00B88048F22101884200F0BB8048F2220141
:104D8C00884200F0BE8048F23401884200F0C180B5
:104D9C001328D6D100206E460290CDE9000028469B
:104DAC00314626F02FF969886E4B4FF080705AE02F
:104DBC000888F080D5F80200C6F81200E88AA6F838
:104DCC001B00E87BB073288A3082688AF082287DC9
:104DDC003076687D002818BF01207076687E002828
:104DEC0018BF0120B076287E7077E869306295F89C
:104DFC00200086F82400A88DF08495F82E0086F803
:104E0C002800A88C708527F0B8FF0028F06298D095
:104E1C00AA8CA96A27F0FCF9287D26F0C5FC20B1E4
:104E2C00007931461CF0A0FB8BE7F06A27F0A3FF5A
:104E3C00304625F049FF84E728461BF087FA002806
:104E4C003FF47FAF6988454B064602203AE06E4638
:104E5C001221304627F064F82846314618F0FCF849
:104E6C0069883D4B042032465AE06E461821304684
:104E7C0027F056F82846314626F036FC6988354B23
:104E8C001020324623F0BEFB039818B127F073FFB5
:104E9C00002003900598C8B953E7284624F0B5F9CB
:104EAC0000283FF44EAF6988294B0646202009E0C4
:104EBC00284624F0AAF900283FF443AF6988234B15
:104ECC0006464020324623F09DFB304627F053FF28
:104EDC0037E7A8696988184B27F059FD4FF4800013
:104EEC001EE0A8696988174B27F051FD4FF48040EC
:104EFC0016E0A8696988144B27F049FD4FF400505F
:104F0C000EE0A86969880E4B27F041FD4FF4004074
:104F1C0006E0A8696988094B27F039FD4FF4801029
:104F2C0023F070FB0DE700BF7D5700207825002093
:104F3C00D5A40200C05E0020BB9302009193020036
:104F4C00E5930200679302003D930200A711020053
:104F5C004D110200F1A401008572010059060200F6
:104F6C00B90602005F3B020098B0BE4C01214FF025
:104F7C000109206027F0CEFC09200DF10B05012161
:104F8C008DF80B0010202A4627F07CFC1020002105
:104F9C0001222B464FF0000826F058FF9DF90B001C
:104FAC0026F076F803AD284627F0AAFDAE4F002177
:104FBC002A468DF80C8007F11406304626F0AAF923
:104FCC007E6027F095FC07F1080579682A4622F0E7
:104FDC000BFA3870A548A0F80880A0F8008006AE3F
:104FEC00304627F075F8002031460FF0D1FDF860FF
:104FFC00012031460FF0CCFD38614068007826F076
:10500C00BDFD10B9387827F04EFD994EF868314641
:10501C0027F0E2FD3869314627F0DEFD082004F860
:10502C00040F94482146A060387817F065F804F115
:10503C00100108201FF032FA24F030FD8E488F4A00
:10504C000178082021F0D6FF8D4908201DF098FA30
:10505C0038781EF0D3FA8B48CDF818808DF82A904A
:10506C008DF824908DF81C9008908748CDF8260078
:10507C008648CDF82B00387806AC214627F018FD71
:10508C0006AE4421304626F04BFF40F2011031466B
:10509C00ADF85600387827F0EDFC7D487D4A017854
:1050AC00082022F097FD7A6838784FF480614FF42D
:1050BC000073CDE9003129464FF4807316F07CF86B
:1050CC008DF81880387806AD294627F0F6FC05F1E6
:1050DC000609724D4FF00A0A78684FF0FF310FF055
:1050EC00D3F90028F8D038781BF0A6FD002876D02C
:1050FC0006460078922815D0E5282BD0CA282DD04A
:10510C00CB2832D0E22834D0E32836D0C5285FD162
:10511C00307900285CD1387821468DF818A027F01A
:10512C00CCFC55E0D6F81200B17BCDF81A003079E2
:10513C008DF82710318AADF82810411E8DF8260005
:10514C00022903D303281CD00F281FD1F088ADF8F7
:10515C001E001BE0301D27F01CFD39E0387821467D
:10516C008DF8188027F08BFC32E0387827F08CFC17
:10517C002EE0301D16F09CFB2AE0301D21F0DFFFE5
:10518C0026E0B11D4846082227F042F8D6F8160052
:10519C00CDF82A00F07E8DF82E00B08BADF82F00E4
:1051AC00B07E8DF83100306A0D9096F824008DF8A1
:1051BC003800F08CADF8440096F828008DF84600C5
:1051CC00708DADF83C00F06A1090204602F0FEFAAB
:1051DC00304614F083F910B9304625F075FDB868E7
:1051EC00810723D4C1050BD52878012802D11BF0E7
:1051FC00ADFB01E014F0ACFAB86820F48070B86034
:10520C00810505D519F0F2FDB86820F40070B8607E
:10521C00410505D51DF014FCB86820F48060B86019
:10522C00010744BF20F00800B86055E70020CDE925
:10523C00060006A813F03EFC27F06BFD4FF47A71C4
:10524C00B1FBF0F04FF4FA61484315F0DFF9FF20A1
:10525C00032121F0A9F827F0DDF90F4801210160A5
:10526C00FEE700BFD821002074210020CC6C002068
:10527C005DA30200A823002083F0020014E50200C5
:10528C008171020000F8FF07FFFF01040301000118
:10529C0081F0020044F002007C0520435A230020D8
:1052AC007FB50138062800F2DE800C46DFE800F0FE
:1052BC000428465E7A8C9900B5480078013801289C
:1052CC0000F2D180002C00F010810020032100247A
:1052DC0021F06AF8AB4DAC4E042004213222287028
:1052EC00307827F0B2FC0820002108F0A9FA3078B9
:1052FC006C704FF4805104B0BDE870401BF06EBC74
:10530C000020002527F014F8A0480121017004208A
:10531C008DF80D0024B19A48C586072025F0B8FAFF
:10532C0098480421322205709748007827F08DFCAC
:10533C00934890F8371001F0FE0192E09448007801
:10534C000138012800F28F808F4804213222007826
:10535C0027F07BFC002C00F0E280894C894801216D
:10536C000170E069E0B321F069FCFAE701208DF8E7
:10537C000D0054B182480021874A80F836108548C8
:10538C0027F078F9072025F083FA7E480021322295
:10539C0001707D4827F0D1FB794890F8371001F067
:1053AC00FD015EE002208DF80D00754854B300211C
:1053BC00794A80F83610774827F05CF900200321F1
:1053CC0020F0F2FF072034E06D4C03208DF80D0027
:1053DC0094F8360008B90120A0712078002854D028
:1053EC007FBD00258DF80D5094B312F033FB65484A
:1053FC000D21C8220570624880F83610624827F0EB
:10540C009CFB29E0082180F83610614909780129B4
:10541C0011D890F83A0070B900200DF10A018DF8FE
:10542C000A0052201FF050FB26F084FC22F08AFD6B
:10543C00002025F02DFA53480021322201705248E9
:10544C0027F07BFB4E4890F8371001F0FB0108E089
:10545C004B48022180F83610494890F8371001F07B
:10546C00EF0180F837104648016A0029B8D090F84F
:10547C003600002203238DF80C004348007803A962
:10548C0000910A2120F045FA7FBD206926F048FFE3
:10549C000028A5D13C4D4FF48041287820F000FC29
:1054AC0000289DD1002604F11000C4E9056624F003
:1054BC00F9FD28784FF480411BF090FBA07901286E
:1054CC0006D194F836000B2804BF002084F836006F
:1054DC002C48A6710178062946D100213222017090
:1054EC002878042127F0B1FB43E0254C0720264DFA
:1054FC004FF4805184F8360001208DF80D00287887
:10550C001BF06CFB0020002624F060F928780221A7
:10551C0041F2883284F8376027F097FBA3E7184CE8
:10552C00022000218DF80B1084F83600154801700C
:10553C0094F837000DF10B0100F0FD0084F83700F2
:10554C0001208DF80D0052201FF0BEFA26F0F2FB60
:10555C0022F0F8FC002025F09BF9E06900283FF4CC
:10556C0082AF21F06BFBF8E7C178062904BF00215C
:10557C00C17094F8370000F0F70084F8370072E738
:10558C0054200020606D00200A6E0020CE260020E2
:10559C001C250020C05E0020A226002092B0DFF85F
:1055AC00B892D9F8000010B1002180F845104830AD
:1055BC0022F020FF27F004F88046072012F0BCFCF4
:1055CC0019F072FB10B1A54827F098F91CF050F8AF
:1055DC0001AD284626F074FE0427002029468DF8DC
:1055EC00047026F075FE9E4C206026F09FFA0AADE2
:1055FC00284626F03DFD002029468DF8287026F01F
:10560C003FFD984E306026F09BFA06AD284626F0FA
:10561C003FFD002029468DF8187026F041FD3168B9
:10562C00914D286019B9914827F068F9286810B98C
:10563C008F4827F063F9206810B98E4827F05EF97F
:10564C001EF0C8FCD9F800004FF0FF3438B1CDE99A
:10565C00104410A9082225F03BFC01281BD1CDE9F0
:10566C001044082027F089FB002846D00546002668
:10567C00052E04D827F0CCF9A8530236F8E74FF6DC
:10568C00200029460822E8807B4826F0C1FD2846E8
:10569C0027F071FB09E0D9F80010CDE9104400297E
:1056AC00DFD07548082226F0B3FD10AA012008218E
:1056BC0027F0E8F8092800D0D8B923F0E1FE8007DC
:1056CC0012D4CDE91044CDE90E440EAB01200021DB
:1056DC00082226F0BBFB60B90EA810A9082225F001
:1056EC00F7FB002800F0B280634A0120082127F064
:1056FC00CFF86149E2201FF0E7F914F077F8242085
:10570C0027F03BFB5D4E002830604DD05C4F5D4C6C
:10571C0007F10C0527F00DFA5B498968D1F84C1399
:10572C0088473068056007F1100527F002FA20F071
:10573C0031F83068456007F1140527F0FAF923F0C9
:10574C00D5FA3068856007F1180527F0F2F91CF0DE
:10575C0051FB3068C56007F11C0527F0EAF921F010
:10576C0059FD3068056107F1200527F0E2F921F0B9
:10577C00C1F83068456107F1240527F0DAF91FF00C
:10578C005FF93068856107F1280527F0D2F91CF024
:10579C004BF83068C56107F12C0527F0CAF9387051
:1057AC0011F016FA306805621AF0C0FA26F08DFE78
:1057BC00404627F01AFA19F04FFB27F04CF901205C
:1057CC001FF088FE1BF0F0FA31480078022808D14F
:1057DC002E480078012804D14FF40040012108F034
:1057EC002FF8274D4FF48041287826F05BFFDFF827
:1057FC00A4904FF0000868684FF0FF310EF044FEA3
:10580C003068002750F82710096821B9791C082F37
:10581C000F46F7D3EFE727F0F6F8316851F8271069
:10582C000C68C1F8008027F019FA59F827200020DD
:10583C0021469047044627F0E6F8316851F82710C6
:10584C000A6822430A6027F009FAD4E70A480EA92D
:10585C00082226F0DDFC4CE7602600205BE9020004
:10586C004C6D0020506D0020546D002079E9020031
:10587C008CE902009FE90200FC6C0020D46D002032
:10588C0000200020F57302000C010020F3260020FC
:10589C001C25002030EC02002DE9F04F89B08A461F
:1058AC0008040DD45FEACA7040F01D815FEA8A706B
:1058BC0000F12B815FEA0A7000F13381002042E194
:1058CC00A24F38781BF0B8F9DFF88892A04C064646
:1058DC004FF0000B48F21508002E00F001813078D3
:1058EC00312838D0322849D0D32840F0B380F08901
:1058FC00404573D0382840F0AD80CDF820B0CDE9CC
:10590C0006BB304606A922F085FC9DF81C10052923
:10591C0068D8307B002840F09D809DF81D00002841
:10592C0000F09880052800F29580069826F04DF836
:10593C00002840F08F80707C8749787070880880D0
:10594C009DF81D00214601388DF81D0006A890E831
:10595C002C002CC17EE0B87803287BD899F82E1047
:10596C00804826F032F8002874D1FF207C49607101
:10597C0070880880B088794908806BE06079FF28CE
:10598C0014D0002019F09EFA0246B9F870107878FD
:10599C003346CDF800B014F073FA6079002859D072
:1059AC0038780821322227F050F953E099F8181072
:1059BC00706820FA01F2D2071ABF3144097A00212B
:1059CC0006F1080200231B2B42D020FA03F5ED0749
:1059DC0002D0D55CA9421ED80133F4E7304623F03F
:1059EC007DFE37E0FF293DD0FE2956D199F8721083
:1059FC009DF81E00884202D860BBFF292AD11EF0F8
:105A0C00EDFE069900201B2859D021FA00F2D2078E
:105A1C0057D10130F7E7B9F86E004F49334608808B
:105A2C004E4802884E48018810200090002014F047
:105A3C0027FA0120F870B87840B93C2002214EF6C4
:105A4C006022B880387827F000F9B8780130B87047
:105A5C0084F805B0304625F037F938781BF0ECF8AF
:105A6C00064639E799F872109DF81E00884203D853
:105A7C000028EFD1FF29EDD11EF0B0FE069838B109
:105A8C00D9F82810814203D0C9F8280024F010FF5F
:105A9C00BDF8200025F010FEDCE7307B0028D9D1C2
:105AAC0070882D49802200230880707CCDE900BBD2
:105ABC00CDE902BBCDE904BB12F0A8FFCAE71B205D
:105ACC0000E0C0B299F818108142C3D02649087082
:105ADC0099F80700642100FB01F23878012162E794
:105AEC008AF400402FE020491A4C08782076E120F7
:105AFC001EF0EAFF24F0DCFE0020A4F87000012068
:105B0C0019F0E0F98AF001001DE010488188B1B16C
:105B1C0001394EF6602281800078022127F095F839
:105B2C000FE00B4C607938B12179206825F04DFFDE
:105B3C0010B96079013860718AF0080003E0002127
:105B4C0081708AF0020009B0BDE8F08F802300203C
:105B5C009C6C0020C05E0020E26C00209A6C00203F
:105B6C000E6C002000F8FF07066E00202DE9FE4F9A
:105B7C00074608680024B0B1D7E9018A0E4626F022
:105B8C001FFD8146D8F8E800082888BF0124B068BA
:105B9C00204202D17068204208D00320307448465D
:105BAC0027F023F800242046BDE8FE8FD8F8C0105B
:105BBC0069B198F8F8100029EFD006213174D8F8A3
:105BCC00C410C8F8C4604E6198F8FC100DE00021B8
:105BDC000522C8E93066C8E93411C8E9361198F8CD
:105BEC00FC10002908BF01223274002201297261C5
:105BFC0009D102204FF4E02188F8FC0098F8FB0052
:105C0C0022F058F9706889490138884205D8042077
:105C1C0022F010FA062022F00DFA022022F00AFAE5
:105C2C0098F8F80040B9DAF83C003168814203D2A8
:105C3C0098F8FC0000286CD0D8E9361009B118B9D6
:105C4C0000E028B326F07DFFDAF80000416941F04E
:105C5C0001014161484626F0C8FF98F8F80008B1E8
:105C6C000124A0E708F16C05D8F8EC10284626F0C2
:105C7C00E3FE0028F4D0D8F8C000032101743846A4
:105C8C000BF0DEFA28460021002426F0D5FE8AE728
:105C9C009AF8040027F04DF8654CDAF8101002223F
:105CAC00206991FAA1F1B1FA81F14368D8F8CC00DE
:105CBC004068006898472069DAF81410022243689B
:105CCC00D8F8CC0091FAA1F1B1FA81F140680068E2
:105CDC0098479AF8040024F07BFC9AF8040027F00B
:105CEC002AF826F02EFF0020C8F8E000D8F8C000F3
:105CFC000068B0F5806F01D926F023FF98F8FE00FC
:105D0C000028A1D1DAF80000416841F0020141609D
:105D1C009AE798F8F90020B1D8F8EC0001307FF43C
:105D2C008BAF484626F061FFB2683AB1D8F8E8006C
:105D3C000221092838BF0121009103E008F1F40287
:105D4C0000200090746834B1D8F8E80002270928C4
:105D5C0038BF012702E008F1F6040027DAF800004A
:105D6C00334D416841F002014160D6F800B0D9468C
:105D7C00BBF1000F40D0D8F8E800019209284FF091
:105D8C00010011D22A68B9F1000F1FD0C0071DD035
:105D9C002178DAF800009268904700281EBF3C4436
:105DAC00A9F101090120EDE72A68B9F1000F16D01D
:105DBC00C00714D02188DAF80000926890470028B8
:105DCC001EBF3C44A9F101090120EDE7DAF80000FF
:105DDC00D26802A99047DDE90120107007E0DAF8DB
:105DEC000000D26802A99047DDE9012010800098DC
:105DFC00ABF1010B0244BBE7D8F8F000DAF8001065
:105E0C00CA680240102802D1002AF9D101E0002A08
:105E1C00F6D0706824F01EFAD8F8C0100020C8F82C
:105E2C00C400C8F8C00008741AE700BFFEFFFF0FDB
:105E3C00C40100102DE9F04F8BB08246807E24F017
:105E4C0077FDA8B1DAF81C1008460691087878B1ED
:105E5C008000013026F091FF40B1044626F050FA44
:105E6C001EF024F948B1204626F085FF102600E0EC
:105E7C00022630460BB0BDE8F08F069804F1010BFA
:105E8C004FF00008049400F1050900200790002051
:105E9C0005900698007880457CD239F8035CBAF8F6
:105EAC000C609AF81A40204631462A4620F024F815
:105EBC000746204631462A4608AB1FF068FDFF2FE7
:105ECC0018BF00280FD18720079AD1B201320BF8E6
:105EDC0021000BEB810019F8041C0792417039F872
:105EEC00031C418002E019F8040C20B109F10E09E1
:105EFC0008F10108CDE719F8010C9DF8261088422D
:105F0C0005D19DF82710490703D48C20DCE78D20A0
:105F1C00DAE77449B9F800304FF6FF74B9F802208B
:105F2C000968A3424FF0160408BF002A1CD017FBC7
:105F3C0004110A81CB8023F09DFD40B369490022F6
:105F4C00086817FB0400C0F80E200868D9F8065042
:105F5C0017FB040000F10E0419F8010C25F0E4FC09
:105F6C0002462046294610E017FB041000210422AB
:105F7C00C0F80E10D0F80A10C0F806105948006886
:105F8C0017FB040101F10E00123126F041F901203A
:105F9C000590ABE70598049D012840F08280504C99
:105FAC00504F162620783A6800FB06F1562026F052
:105FBC0069FC30B920783A6800FB06F1562026F0CF
:105FCC0067FC4948802100781AF008FE474804789D
:105FDC00A00026F0D2FE002863D0454F8146224611
:105FEC0009F10101781C3AB150F8013C1430013A26
:105FFC0041F8013C0431F6E73C48069490F800B0B7
:10600C00BBF1000F33D0394E01204FF000085FFA7E
:10601C0088F159452BD2000625D0386958B1D0E902
:10602C000041396126F0A7FE387B013838732046D1
:10603C0026F0A1FEF1E730780138C1B2307089004A
:10604C0051FA80F107EB810257F821105368D2E91D
:10605C000345C7E900131189C7E9034539810021BC
:10606C001161117300E0002008F10108CFE707F07F
:10607C002BFB049D069E0024A6420FD009EB840046
:10608C004188407821F01CFBFF2805D019F824101A
:10609C0000EB800007F820100134EDE7484626F0AD
:1060AC006AFE07982870000604BF012028809AF821
:1060BC000A10BAF80C209AF81A0000260123CDE930
:1060CC0000332B46CDE902160AF10E0115F046F904
:1060DC00284626F050FE24F06BFC20F077FDC8E635
:1060EC000C6E0020646D00200A6E00200E6E0020E5
:1060FC00A05F00202DE9F04F9BB004460088894634
:10610C000B2100F00700022808BF1421002808BF4B
:10611C000F21607E01EB0008404626F0A0FE00280F
:10612C0000F09380214602220746022626F038F919
:10613C002088BD1C00F00700022811D018BB0020DD
:10614C00261D04228DF8040001A83146043026F0E7
:10615C0027F928463146042226F022F9BD1D12E00B
:10616C008DF8046001A804F10806082204303146B9
:10617C0026F016F928463146082226F011F9207C23
:10618C0007F10B05B87204F114012846042226F01D
:10619C0007F9207E2871607E68710635627E52B1E7
:1061AC00E169002951D0284626F0FAF8E069667EAC
:1061BC0026F0FFFC354404F12001284626F03CFD76
:1061CC0094F82200DFF8D0A15FFA88F23946A87063
:1061DC000AF108001FF0FEF9002800F0D98080F8C1
:1061EC000090002680464FF0FF300DF11F09ADF8EE
:1061FC006800CDE91800ADF81860CDE9046601A877
:10620C0009F1020B09F10607041D042E1FD8F0B288
:10621C00494621F02CFD05460D2814D00A2D19D025
:10622C009DF804009DF81F10484040070BD12046F4
:10623C003946042225F0C2F860B920465946082296
:10624C0025F0BCF830B90136DFE71020A1E00D2DA8
:10625C0000F09680514DF2208DF81900A88CADF805
:10626C001A009DF81F00410634D5022009F12201C5
:10627C000A228DF8180018A825F0A0F880B904ACF3
:10628C0009F12A0126F065FC26F072FB40B1E98A7F
:10629C008181014694E84C004CC198F80010817340
:1062AC0009F12C0118A80A2225F088F880B904AC51
:1062BC0009F1340126F04DFC26F05AFB40B1E98A75
:1062CC008181014694E82C002CC198F80010817350
:1062DC009DF81F0040B2B0F1FF3F22DC01208DF889
:1062EC00180001A81EF045F9ADF8100026F040FB8F
:1062FC00B8B104469DF82000800604D401A81EF015
:10630C0038F9A08105E004F10C0009F10B0126F02D
:10631C0093FC04A8214690E82C002CC198F80000AE
:10632C00A0739DF82000C0072AD001208DF818001A
:10633C009DF85500C0070FD004AC09F1370126F0C9
:10634C0008FC26F015FB38B105460C3009F1390173
:10635C0026F072FC25F01FFE9DF8550080070FD526
:10636C0004AC09F13B0126F0F4FB26F001FB38B13B
:10637C0005460C3009F13D0126F05EFC25F00BFEC4
:10638C0007483221006826F0FCFB064826F013FD76
:10639C0001201BB0BDE8F08F1C240020C05E002043
:1063AC00846D0020386400202DE9F04F87B0851CE7
:1063BC008346284626F00DFC01AC064618212046E3
:1063CC0025F0AEFD9BF801A004F10B0029460095C9
:1063DC0026F074FC6FF001009BF80A1002240122D5
:1063EC00ADF8180000208DF81A408DF80C0001F063
:1063FC000800C1F3C007890782EAD00507D400283A
:10640C0008BF0124B946A8460027002507E004244C
:10641C004FF000094FF00008002808BF03248548FE
:10642C00007850EA0A000BD0834890F82600082820
:10643C0009D125F045FE00285AD0BAF1010F57D1E9
:10644C004FF0C30901E04FF0C2090025BAF1000F6B
:10645C0010D07F48007890B9BAF1010F0FD1002EFF
:10646C0055D00020214601228DF81A0001A815F004
:10647C0007FF0AE001A81CF0F9FE86B91CE001A890
:10648C002146524615F0FCFEB6B17179BAF1020FF5
:10649C0041F04002727104BF41F0600171719BF8D0
:1064AC000A10490603D5717941F080017171B179F7
:1064BC0000240131B17100E00124B0FA80F14909E6
:1064CC000D422CD107D1002D18BF814641F201009D
:1064DC00494619F088FD14B900981AF0E5FEBDF88C
:1064EC0018004FF6FE71884218BF26F050FC16E0DB
:1064FC00DEB33279A24218BFBAF1020F12D1D01E0C
:10650C00C0B201281BD857EA050020D12AE002208E
:10651C00214601228DF81A0001A815F0B1FE07B032
:10652C00BDE8F08F4FF00009009953468DF81A9092
:10653C003088ADF8180026F00AFC012586E7501EBD
:10654C00C0B201280ED849EA0800012807D13088CA
:10655C0023F0A0F950B93088ADF8180008E0308865
:10656C0026F015FC00981AF09FFE0026BDF81800C6
:10657C004FF6FE7188421ED122F0C0FF10B1BDF85B
:10658C00180011E0BAF1000F04D02C4D288823F02C
:10659C0081F930B19BF80A0000F0020021F07AFD7D
:1065AC0000E02888ADF818004FF6FE71884202D141
:1065BC004FF0C70949E79BF80A200099534626F08B
:1065CC00C6FB10B14FF001093FE71D48016811B13E
:1065DC00BDF818008847BDF818000099224607F04E
:1065EC009FFA0646174818490A6800784FF480311C
:1065FC0026F02BFB01211548C17096B1AAF10100C0
:10660C00C0B2012807D81020BAF1020F08BF082029
:10661C007179084370714FF0000901258DF81A90BB
:10662C0014E74FF6FE7000254FF001090026ADF877
:10663C0018000BE7CC230020C05E0020942600201D
:10664C0050220020036E002038F00200EC240020C1
:10665C001C2500202DE9F04F8DB0044600209A46F1
:10666C0016460F46CDE90B00CDE909008748856831
:10667C00804616F044FA1C2803D016F040FA1B286A
:10668C001BD1308840F60201884218BFB0F5C15FBB
:10669C0003D1F07B022810D93EE043F60701884273
:1066AC000BD196F82400032807D33069784940F0C1
:1066BC00806020F0604088422ED100206FB366B31A
:1066CC00387825FA00F0C00726D03046002126F095
:1066DC004EFB7048C4E90176006880B109A80090AF
:1066EC000CA90BAA0AAB30460BF022FA0B980B2123
:1066FC004FF6FF72502323F0CBFFFF280CD025F070
:10670C005FFF654F06467878012802D840B101201A
:10671C0070E0304626F069FA00200DB0BDE8F08F2D
:10672C000BF07AF95D480DF10409016841F00201A2
:10673C0001605B48C8F80000484625F0B9FDDFF859
:10674C0064B15A494A469BF801009BF800500390EB
:10675C005548283020F0CAFE554856494A4620F084
:10676C00C5FE484625F0DCFCDFF84C81534A192164
:10677C004B46029540461FF0A3F9514A08F11C0004
:10678C001A214B461FF09CF94E484F4926F0E9F967
:10679C004E484F4926F0E5F94E48006810F4402F5A
:1067AC0006D04D4A07F128000421002323F05AFBA0
:1067BC009BF8020010B10D2011F0BEFB08F1400057
:1067CC0025F0F8F808F1380025F0F4F843490020DA
:1067DC0007223876B8843862386181F86020052148
:1067EC00C7E902103E49F96138700420002123F0FA
:1067FC00FFFF78782C4941F8204001307870304602
:10680C0026F0F3F9BAF1000F06D10DF1040A35495F
:10681C002022504626F026FBDAE90012BAF81000C6
:10682C00DAE90635002AB2FA82F608BF40F6C4123D
:10683C006261216060832563760926764FF4FA76CF
:10684C00C4E9036201226276274AC4E90722C4E93B
:10685C000923DAF80C0000B12062DAF8140000B158
:10686C006062DAF8080000B1E06104F13800C82178
:10687C0025F056FB04F15000002123F0F9FF1B49D1
:10688C0004F1B80026F06DF9204646E7CC2108400B
:10689C000F00000560250020481D00200020094045
:1068AC00110000E058EF0200E81E002069AF020062
:1068BC00886500201D6E0100A81F002051F9010001
:1068CC0081DC0100F4630020959E0200B06300207F
:1068DC0015AF0200B44F00500D290200385F0020A4
:1068EC0001280100D4EC02001B6E010075CC0200E3
:1068FC002DE9F04F87B000240293002A00F03D816F
:10690C00074603A892460E464FF0200B103001901C
:10691C00504610F8011B25290CD0002900F02A81C3
:10692C00022EC0F0D980013E002F00F0D48007F871
:10693C00011BD1E09AF801002D2806D19AF802002B
:10694C000AF103034FF0010C03E00AF102034FF0CC
:10695C00000C30280CBF13F8011B01462A2920D14A
:10696C00029D2A68111D2960D2F8009013F8011BB2
:10697C00B9F1FF3FDCBFC9F100094FF0010C2E2922
:10698C001ED11A4612F8011B2A291CD1029D2A6815
:10699C00111D29609D1C126859782B4622EAE27859
:1069AC0021E04FF00009A1F13002092AE7D809EBE8
:1069BC00890201EB4201A1F1300913F8011BF2E746
:1069CC004FF0FF380FE04FF00008A1F13003092B16
:1069DC0008D808EB880301EB4301A1F1300812F849
:1069EC00011BF2E7134630284FF0000241F0200063
:1069FC0008BF4A466C2808BF13F8011B9A46692940
:106A0C0001D064290CD1029B1868011D19609045B6
:106A1C00C8BF4246DDF8048001686FF009031EE030
:106A2C0075290AD0A1F16F00092858D8DFE800F0C9
:106A3C0005695F5F835F5F5F5F05029D2868031DCB
:106A4C002B6090454FF00803C8BF4246782908BF19
:106A5C001023752908BF0A23DDF80480016840461D
:106A6C00654617F0C7FEAC460546A8EB0001A9EB3E
:106A7C000100BCF1000F0DD109E0022E05D3013E3F
:106A8C0017B107F801BB00E00027013801340128D9
:106A9C00F3DA01380A465AB1022E06D3013E1FB171
:106AAC002B7807F8013B00E00027013A0135F2E7AB
:106ABC000C44BCF1000F3FF42BAF0128FFF628AFBC
:106ACC00022E05D3013E17B107F801BB00E00027E9
:106ADC0001380134F1E700270134824618E76329B5
:106AEC0005D1029A1068011D1160006804E0AAF13A
:106AFC000100022E3AD300788DF80C00012103AD71
:106B0C00B5E7029ADDF804801023CDF800C01068B8
:106B1C00011D11601099082200290168404617F0E8
:106B2C0069FE05464FF04000DDF800C005F8010D88
:106B3C00A8EB05019BE7029ACDF800C01068011D77
:106B4C001160109905680F480029002D08BF0546F3
:106B5C00284625F0DDFC0146804538BF414618F13A
:106B6C00010208BF0146DDF800C080E7002103AD3B
:106B7C0082467CE70FB100203870204607B0BDE894
:106B8C00F08F00BF30D402002DE9F04FA7B00DF10B
:106B9C002008814600213822404625F056FA99F803
:106BAC000720089B99F8061099F8050043EA024261
:106BBC0042EA01210843089000F00700022811D096
:106BCC0008BB08F1040009F10801042215F0D6FFF6
:106BDC0008F10800FF210822FF2425F036FA8DF871
:106BEC00304010E04FF0FF3009F108040822099002
:106BFC0008F10800214615F0C1FF08F110002146EC
:106C0C00012215F0BBFF0898C10617D4C0F3411040
:106C1C004FF6FF75032800D0E8BB09F1080408F112
:106C2C0011000822214615F0A9FF08F11A0021468F
:106C3C00022215F0A3FFADF83C503BE016AF08F173
:106C4C00110A08F1040B0024BD1CBE1D042C7DD8B8
:106C5C00E0B2394621F00BF80D2818D00A2875D06F
:106C6C00089841070AD000F0070002280FD12846E7
:106C7C005146082224F0A2FB30B908E030465946B0
:106C8C00042224F09BFB20B1384625F0BAF90134DC
:106C9C00DCE70898E7E708F11100FF21082225F04E
:106CAC00D4F908F11C0009F108010222ADF83A50A0
:106CBC0015F064FF9DF8200000070BD41E20ADF8E2
:106CCC0054508DF856004FF0FF301090FF208DF887
:106CDC003E003BE009F1080608F11E000122314696
:106CEC0015F04CFF0899480403D44FF0FF30109076
:106CFC0006E008F120003146042215F03FFF089908
:106D0C0008F12400090404D4FF21102225F09DF978
:106D1C0003E03146102215F031FF0898C10302D46C
:106D2C00ADF8545006E008F134003146022215F05B
:106D3C0025FF0898800359BF1E208DF8560008F1D6
:106D4C003600314644BF012215F018FF089800F4B4
:106D5C00C261B1F5007F55D0C1060ED410F0600FA2
:106D6C0016D008A802F042FC012845D199F804007D
:106D7C00002847D148F601100FE000F00700022868
:106D8C001DD030BB00208DF810000998059020E034
:106D9C0099F80400B0BB48F20150ADF858001C48FB
:106DAC00D9F8001000220123CDE900230078CDE9A9
:106DBC00022016ABF220212220F0F7F922E002206B
:106DCC0008F1080108228DF8100004A8043025F001
:106DDC00E7FA04A816A90DF11E0216F087FC88B973
:106DEC0016AC204625F00DF9BDF81E1002204122EC
:106DFC0023461BF0EFFB05E004484078400748BFF2
:106E0C001CF022FC27B0BDE8F08F00BF58230020F7
:106E1C00CC2600202DE9F04FA5B08B464FF0FF316A
:106E2C009146ADF89010CDE922110DF1470120F0FB
:106E3C001EFF04460A2800F023810D2C00F020814F
:106E4C000DF106070DF1470A02220226384651467B
:106E5C0025F0A6FA054601A8514625F0EAFEBDF834
:106E6C00040000F00700022807D090B90AF10601CF
:106E7C0025F07FFE054606260BE00AF102012846A6
:106E8C00082225F08DFA0AF10A0125F0C9FE054603
:106E9C000B269DF84800810608D50AF10B012846FF
:106EAC0025F0C7FE05469DF848000236410608D578
:106EBC000AF10D01284625F0B3FE05469DF8480061
:106ECC000136400603D49DF84700800612D50AF11E
:106EDC000E0125F04EFE05469DF84800400601D4F3
:106EEC00043607E00AF112012846102225F058FA60
:106EFC00054614369DF84700400601D4B04641E0E3
:106F0C0000200AF122070A228DF8020022A8394635
:106F1C0024F054FA10B106F1010811E00DF106004D
:106F2C00012101228DF8021030440DF1020125F0EF
:106F3C0037FA39460A2225F033FA054606F10B08D2
:106F4C000AF12C0722A80A22394624F037FA10B18C
:106F5C000DF1060716E09DF802000DF10601012265
:106F6C0001308DF8020088190E460DF1020125F052
:106F7C0017FA394628460A22374625F011FA0546F3
:106F8C0008F10A089DF84800C00701D1464631E0D7
:106F9C0000208DF802009DF87D00C10702D108F198
:106FAC00010613E0012157FA88F001228DF8021036
:106FBC000DF1020125F0F4F90AF13701042225F054
:106FCC00EFF905469DF87D0008F10506800711D5FF
:106FDC009DF802000DF10201012201308DF8020032
:106FEC0057FA88F025F0DCF90AF13B0125F0C1FDD8
:106FFC00054604360AF13F01284625F011FE9DF89E
:10700C0047100A0701D5C90605D40AF1400125F03D
:10701C0007FE023600E00136BBF1000F26D099F8CE
:10702C00000035460DF10201002818BF023D50FA50
:10703C0085F0ADF80200584625F0FBFDF2B2412A6E
:10704C001DD899F800000DF10601002808BF0BF1BE
:10705C00020B584425F0A4F999F800009DF8021091
:10706C00002808BFA91C89F8001009E099F8000055
:10707C00002808BF0236304489F8000000E00124E3
:10708C00204625B0BDE8F08F2DE9FC470446019061
:10709C0007789148C65D9148F840ADF80260C0078A
:1070AC0040F00A810D2F13D18D4D0DF10201A8680E
:1070BC00D0F8282453209047BDF802104FF6FD70ED
:1070CC00814214D8208990B14FF0000A25469FE0E8
:1070DC000C2F11D0072F16D0052F11D1A078012815
:1070EC0000F0EA80207C304400F1240919E0A86803
:1070FC00D0F8541301A8DEE06068C08AC0050AD439
:10710C004FF0000A09E0A07848B1A07D00EBC00068
:10711C0006EB800905E04FF0010AB14605E006F1E7
:10712C001B09ADF802904FF0000A484622F01CFEF5
:10713C0000B30546072F3CD1207828706078687022
:10714C00A078A8700028E178E970D4F8051069607F
:10715C004FD0A07D0028287241D0A16900293ED0D3
:10716C0000EBC00005F110068200304625F050F807
:10717C00EE6037E00C2F40F09F80254655F8040F49
:10718C00002800F0998025F01BFA8046544880684E
:10719C00D0F8541328468847484622F0E5FD0546AA
:1071AC00404625F022FD002D00F0868025F0EAFBFC
:1071BC002EE025F0E7FB052F2AD105F118066968AA
:1071CC002422304625F024F869692A7C05F13C001C
:1071DC006E6025F01DF868682430686118E00020A6
:1071EC002872E860A06998B125F0C5FD0020A07553
:1071FC000DE01B2005F110061B2228723046A169F8
:10720C0025F006F8EE60A06925F0B5FD0020A06120
:10721C003448016819B128468847002841D10D2F00
:10722C0025D161680A78C2F38300920746D42E4AAE
:10723C00927C904242D149783F293FD894F8301043
:10724C0002293BD195F8470005F146011FF032FCAD
:10725C0001984FF6FF72418E914217D140688079A8
:10726C00022813D328461BF00DF990BB24E00C2FF9
:10727C000CD160781A2809D0686838B1C08AC00768
:10728C0004D0287C05F10F011FF014FCBAF1000F9B
:10729C000FBF1748002028701448294600781AF0B0
:1072AC0063F90C2F08D1019850F8041F21B10C4937
:1072BC008968D1F854138847BDE8FC87032808D1A6
:1072CC00012021462070094800781AF04DF9BDE8DC
:1072DC00FC87034880680BE74CEE020019C20600DD
:1072EC000C0100205C260020C05E0020136E0020E4
:1072FC00036E00202DE9F04F8DB00646806A44786D
:10730C0074B18D4909788C4280F012818B4902301E
:10731C0022462AB130F8023B013A21F8023BF8E749
:10732C008748C18A708988422FD183480078A0424F
:10733C0040F2FE80B589814A2146284623F070FE32
:10734C00284617F09DFF064682480778BE4204D1B6
:10735C004FF6FE7017F094FF0646BE4280F0E880B0
:10736C00DFF8F48108EBC6094F4657F8040F08B153
:10737C0025F001FD002C00F0B180600025F0FDFC33
:10738C000028386040F0AC80D2E0B27C002A00F0DB
:10739C00CF806A4F0025AC4205D037F815208A42C1
:1073AC0003D00135F7E7A04600E0A846002115F010
:1073BC00A7F8002800F0AD8081464079012840F004
:1073CC00A88099F8060010F0180F00F0A280B9F808
:1073DC000210204623F03CFFA54202D3002800F007
:1073EC0098805848CDE90498B6F80C904FF6FE7A80
:1073FC0000780890544800780A90002006960B906C
:10740C0052481130099052480430079000200C90DB
:10741C00DDE909564FF0000BF6B135F8117C5745F4
:10742C0018BF4F4502D1013E1C35F5E720463946C1
:10743C0023F00EFF0028F6D1287801380528F2D861
:10744C000C980BF1010BC007EDD00B985FFA8BF188
:10745C00C0B28142E7D356E0DDE907862EB338F897
:10746C00047C574518BF4F4503D1013E08F1240851
:10747C00F4E72046394623F0EBFE0028F5D198F8C6
:10748C00050001380528F0D898F8000001380228CA
:10749C00EBD30C980BF1010BC007E6D00B985FFAFD
:1074AC008BF1C0B28142E0D32DE05FEA0B6028D0B3
:1074BC000B98000625D101205FFA8BF50B90012D5E
:1074CC004FF001000C90A3D025F0A2FAC0B2B0FB93
:1074DC00F5F101FB15000B90012098E700203860B6
:1074EC001E4989F80140A9F80250097808F83610AD
:1074FC00F4B1E8B1114962000DB0BDE8F04F24F0D1
:10750C0087BE4FF6FE770498069EDDF81480478000
:10751C000A4FB37CF47CB269B1890125581EB07452
:10752C0070895FFA88F68DE8D000039511F00AFC9B
:10753C000DB0BDE8F08F00BF73F00200306B00207F
:10754C00C05E00207EF002006CF00200E4450020DA
:10755C00B83E002072F0020004600020EC260020EF
:10756C002DE9F84F2DED085B15460E46074620F029
:10757C00A7F8FF2800F06E80824600EB80018F4850
:10758C0010F82110C90700F012810AEB8A0100EBF8
:10759C0081084FF6FF71B8F80600884200F00781A9
:1075AC0008F110000468002C54D020680188A9420E
:1075BC0001D0201DF6E700284CD004AB38463146EC
:1075CC002A4611F0DBFF012844D17D488021007848
:1075DC001EF066FB05464FF0000978B179484FF470
:1075EC007A7100884843401B28BF8146B9FBF1F0F3
:1075FC0000FB1191002918BF01308146B8F8040036
:10760C0030B1B8F8081011FA89F1814240F2CF80FC
:10761C009DF81260304622F02DFA002800F0B3805D
:10762C002068A6F120030599821C00200B2B13D88F
:10763C00DFE803F050640606BEBEBEBE767D47474B
:10764C00106809685268431A38BF0B1A934280F0CD
:10765C009A80ACE00220ABE0392E7ED03A2E40F07E
:10766C00A78092ED000B92ED018B54EC106B91ED19
:10767C00000B304621465BEC107B3A465B4603F030
:10768C001BFDCDE90210384659463246234603F01D
:10769C0013FDCDE90010304621463A465B4618F002
:1076AC00C1FC00280299009808BF01460398019A72
:1076BC0008BF104653EC182B18F0B4FC002862D10C
:1076CC0075E0106809685268431AB8BF0B1A9342E8
:1076DC0059DA6CE01378097812790020CC1A9442AC
:1076EC004FF00004A8BF012425F033F9A8BF0122F4
:1076FC008B4238BF2246012A45D059E013880988AD
:10770C0092880020CC1A94424FF00004A8BF0124A8
:10771C0025F01FF9A8BF01228B4238BF22461AE080
:10772C0092F9003091F9001092F9042005E0B2F9B9
:10773C000030B1F90010B2F90420CC1A00209442A8
:10774C004FF00004A8BF012425F003F9A8BF0122C3
:10775C008B42B8BF2246B2B92AE092ED000A91EDF5
:10776C00002A92ED011AB4EE420A30EE424A32EE91
:10777C00403AF1EE10FAB8BFB0EE434AB4EE414ACB
:10778C00F1EE10FA13DB24F0BBFD504604F03EFF83
:10779C0025B11FFA89F000211BF04CFE0A48007835
:1077AC00504584BF0020A8F808001FF00FFA0020F5
:1077BC00BDEC085B01B0BDE8F08F00BFA05F0020FE
:1077CC000A6E0020F06D00200E6E0020F0B58DB01A
:1077DC000446808C032801D2012456E0924F0025E8
:1077EC000794A16A0C95ADF82C500A957C6007A8FB
:1077FC00043018F095FBA16A0A90081AA18C084471
:10780C00ADF82C00207D24F073FDE0B38068B0B39C
:10781C009DF82020A188207D9DF8273002F00302DE
:10782C001DF0D7FB58B3A688257D2846314624F099
:10783C00A7FD07F10801096851B38A88B242FAD84A
:10784C00CA88B242F7D39DF82020530703D19DF884
:10785C0027300B2B05D0400603D5607E002800F0A6
:10786C00928090071FD08968B1B107A88847FF287C
:10787C006FD0044601284FD19DF820200CE0002049
:10788C000324786001E07D600224E0B20DB0F0BD0D
:10789C009DF82020900706D06FF07C04500758BF4D
:1078AC006FF07E0438E0500733D49DF8270016287B
:1078BC0031D85E4C24FA00F1C9072CD1BDF82C103C
:1078CC008DF810505A4DADF812100A99059155F8D3
:1078DC00301004A8884700280C9000F081809DF897
:1078EC00271024FA01F2D20706D105EBC10041683A
:1078FC0007A888470C9808B125F05BF99DF827007C
:10790C00152804D84B4921FA00F0C0076DD100248A
:10791C0002E0842400E082240799487D08B9488855
:10792C0088B1012000217960E1B20029ADD0842911
:10793C0004D10724002818BF0624A6E70924002830
:10794C0018BF0824A1E79DF82030D80604D52006DE
:10795C0002D100247C6098E79DF8270001258A88D5
:10796C008DF819409DF826C0BDF8246025EAD30394
:10797C008DF81800087D8DE86810063106AB1FF0F5
:10798C0014FC0020CEE70798417D31BB408820BB1A
:10799C0028463146002223F0F1F99DF82700079B79
:1079AC009DF820504FF0010CBDF824609DF8261076
:1079BC008DF819C08DF818009A88187D2CEAD50519
:1079CC00CDE90261991DCDE9005C06AB1FF0EDFB22
:1079DC00A188207D012223F0D1F90020052450E755
:1079EC000799487D18B101241CE000241AE048884E
:1079FC000124B8B980209DF820309DF826508A8843
:107A0C00BDF824608DF819009DF8270024EAD303F3
:107A1C008DF81800087D8DE858000395063106ABEB
:107A2C001FF0C3FB00202CE7F824002080C20100CB
:107A3C00D0DF02006D192A002DE9F04F8DB00546FC
:107A4C00002095F8241005F12504CDE90A000C90CE
:107A5C00CDE908004EB2C1F38012B6F1FF3F03929C
:107A6C000EDD002201274FF000084FF0000A0292B1
:107A7C0001F00309B9F1010F1CD10020019042E083
:107A8C002278C2F3801802F00700B8F1000F8DF8CD
:107A9C00280003D0039B002B40F0F680C2F3C10AF0
:107AAC00BAF1010F00F0F080C2F3401205F1260488
:107ABC000227DCE702280DD048B902202146042217
:107ACC0028740AA8043024F0A3FB043704340020E3
:107ADC0001900CE0032005F108010822287414F829
:107AEC00010B01900AA8043024F092FB013700200E
:107AFC000822CDE904000AA804A9043023F0E8F90F
:107B0C00002840F0C180BAF1020F11D308A8214619
:107B1C00042224F07DFB95F8230004340422C01BBE
:107B2C00A0F1080B09A854FA8BF124F071FB14E0B6
:107B3C00BAF1000F03D000244FF0000B0DE02078B9
:107B4C00E02803D10398002840F09E8095F823107C
:107B5C0095F82200A1EB070B0890B9F1010F19D190
:107B6C00002E00F191802078EF2800F28D80BAF180
:107B7C00000F40F08980039860B9454812216A686B
:107B8C00012301600020002105908DF8100004A84D
:107B9C0002F0FAFF442050FA8BF022F0E5F80028AE
:107BAC0072D00646012030750420308095F82000F4
:107BBC00297C70750329B5F8210086F82010F08215
:107BCC0006F1180004D0022907D12989018004E0AC
:107BDC000AA90822043124F01BFB039886F8249090
:107BEC00DDF80890019F86F8298086F826A04FF0D2
:107BFC00000886F828009DF8280086F8279086F85B
:107C0C00307086F825000B98F0620898706309981C
:107C1C00F063A88B7084207886F8380000201EF062
:107C2C00A7F94FF4FA613071C6E9028168683061D6
:107C3C00202022F099F820B31649054630465FFA09
:107C4C008BF824F0D5F9072021464246288030795C
:107C5C00287706F1410024F0DBFA089886F840B04A
:107C6C0085F815902F7485F814A00C22A861281D96
:107C7C000AA924F0CDFA08482946007819F074FCBA
:107C8C0002E0304623F020F80DB0BDE8F08F00BFC5
:107C9C0000260020F4250020136E00202DE9F04F63
:107CAC0087B005462C200E4625F067F8002844D0F6
:107CBC00778B044624F0A2FC0021E1840121874249
:107CCC0008BF02212170707BA0703169081A6060B6
:107CDC00204618F0DFFF3178834F01F00301387B29
:107CEC00012908BF05206070C0B224F0D1FA4FF012
:107CFC00FF316077A182217F326908440A44317DCB
:107D0C003261081A3075E070A069013017D0207C00
:107D1C00032816D8DFE800F00217020906202146D6
:107D2C006082284617F0B0FC10B304202146608214
:107D3C00284609F017FB05461BE01025CFE0A325CC
:107D4C0017E0A12515E00020B3256082F87A80B9F0
:107D5C0097F8410001280CD1A07D4FF6FF761AF060
:107D6C00F7FD0025A082B04208BF6FF05E0500E071
:107D7C0000252078022807D104F1080623F026FFFD
:107D8C000146304624F09AFF280640F0A580574F54
:107D9C003878013801281AD894F8260010B994F8CC
:107DAC002700A0B1A078E178227F08441044043069
:107DBC0024F0E3FF58B1A178E2780646207F114405
:107DCC0008446168021D304624F022FA00E00026C7
:107DDC0020460EF0DBFD05463878012802D12DB97E
:107DEC00002575E0022873D1002D71D0002E73D0C0
:107DFC000DF1080800274FF0010B4FF4D00908F1E2
:107E0C00080A94F8260018B994F8270000285FD0C7
:107E1C00A178E278207F114408443146021D606845
:107E2C0024F0F6F994F8260020B184F82670C4F8F2
:107E3C00129007E094F8270020B12D4884F82770A1
:107E4C00C4F8120020460EF0A1FD10B10021054629
:107E5C0039E04046142124F063F8608A8DF819B09B
:107E6C00F0B9A08A40F20311884216D0682817D1C5
:107E7C006068C17B052929D12A30FF21082223F013
:107E8C00C5FD18B34FF0FF306946CDE90000194825
:107E9C00006824F013FFFC2000E0FF208DF8180090
:107EAC00504669460022002513F08AFD01469DF8D4
:107EBC00000038B104201422434621F061F803215C
:107ECC00002500E0032103299BD101E00221FAE700
:107EDC0016B1304624F04FFF204624F04CFFE8B298
:107EEC0007B0BDE8F08F00BFC05E00201C2500204D
:107EFC0000000301386D00202DE9F047AEB00DF104
:107F0C00540800248246142140468DF8B740CDE930
:107F1C001A4424F005F89AF804001B94C0F3C1012C
:107F2C008DF85400012916D0E9BB00F00700022897
:107F3C0025D0A8BB08F104000AF10801042214F0B2
:107F4C001DFE08F10800FF210822FF2424F07DF813
:107F5C008DF8644024E04FF0FF30FF210822FF240D
:107F6C00169008F1080024F070F808F111000AF1DD
:107F7C00080101228DF8644014F000FE13E04FF06C
:107F8C00FF300AF108050822169008F1080029466E
:107F9C0014F0F4FD08F110002946012214F0EEFD56
:107FAC00FF208DF8650000250DF176060024042CC9
:107FBC0009D8E0B231461FF05AFE10B901358DF8E0
:107FCC0069500134F3E79DF8540000F018000828BC
:107FDC0050D19DF86570280602D0E8B2B8420FD295
:107FEC0000205B498DF86A708DF86B008B208DF842
:107FFC006800DAF800000A781AA912F0D9FD4EE0F0
:10800C0000210DF1B7060022F8B20D4605280ED856
:10801C0000213246FEF7FEFE9DF8B71048B9013735
:10802C002A464B29F0D329468DF8B75001E0294652
:10803C001546F9B1C8B224F012FF0026D8B19DF84C
:10804C00654007460DF1B7098DF86B608DF8B76088
:10805C00052C0DD8E0B239464A46FEF7DBFE38B99E
:10806C009DF8B700013601348DF86B60A842EFD350
:10807C003E4600E000269DF8540010F0180F11D079
:10808C009DF8650032491B968DF86A00DAF80000FD
:10809C000A781AA912F08CFD304624F08AFD2EB015
:1080AC00BDE8F08700F00700022807D00028E7D1D0
:1080BC0000208DF848001698139009E0022008F172
:1080CC00080108228DF8480012A8043024F068F941
:1080DC00FF200DF105010DF146028DF86A0012A882
:1080EC0015F004FBE8B18B208DF868009DF8B70003
:1080FC000028C5D024F0B3FE00260028C0D00546C9
:10810C00BDF846000DF1B7028DF86B608DF8B760C5
:10811C002946FEF77FFE10B901208DF86B002E4624
:10812C00AEE7BDF846009DF8B7400DF1B70200214F
:10813C000025FEF76FFE10B18DF8B750A0E79DF843
:10814C00B7004B2824BF8DF8B7402046D0E700BFBE
:10815C00CC2600202DE9F04F85B0884608040AD4BF
:10816C005FEAC87045D15FEA887049D45FEA08704D
:10817C0055D4002005E1DFF810A29AF8000018F0A1
:10818C005BFD002800F0FB800546807FC8B9688C39
:10819C00132816D17D486E8800F11C090020494631
:1081AC004F46002818BF071D086850B1014631F82A
:1081BC00042BB242F4D144683C6024F0DCFD204630
:1081CC00F3E7A87A05F1020B022840F0BE80DFF835
:1081DC00BC9195F83170BBF8006009F11C00006887
:1081EC00A0B10188B14202D18178B94240D00430AB
:1081FC00F5E76648406900B1804788F00100C0E0AF
:10820C0062480121017088F00200BAE0D9F81C40E4
:10821C0094B30120616889B301300C46FAE75E48DB
:10822C00DFF86891807BD9F81C6000073CD424F0FF
:10823C0072FD044624F06DFD584A60434FF47A7188
:10824C00B0FBF1F0D9F818101288411A914256D3AC
:10825C00B1FBF2FB0BFB02F2511A08444C49C9F872
:10826C0018001FFA8BF00978884288BF8B461DE0F6
:10827C0047490978C1707FE000240020454980B24D
:10828C000988884261D2082024F077FD00285CD050
:10829C0000210680877041603D490978C170D9F88A
:1082AC001C1079B360603FE04FF0010B00205FFAC7
:1082BC008BF44FF0000A071D002808BF09F11C07BA
:1082CC0096B1F078C0FA5BF1A042F17006D87568EF
:1082DC0030463D6024F04FFD2E46F1E77168304684
:1082EC000AF1010A0E46E6E75FEA0A4007D10020D0
:1082FC000821C9F818002448007818F06FFC88F0A1
:10830C0008003EE0C9F81C002348807B00070BD412
:10831C0024F001FD044624F0FCFC60434FF47A7118
:10832C00B0FBF1F0C9F818001B48807B00070CD596
:10833C009AF8000008211DF0B3FC30B91748082149
:10834C0002889AF8000024F07DFC2878022810D0CE
:10835C00012811D1297EAA89EB7C05F11C006C69DE
:10836C006E7E8DE85A0005F11003594604F074FF37
:10837C0002E0284614F0AEFE284622F0A5FC88F454
:10838C00004005B0BDE8F08F016E0020E422002013
:10839C00D52600209C260020C05E0020A0260020B0
:1083AC002DE9F04F99B012AF8B4604461C211646AE
:1083BC00384623F0B5FD204639460CF079FB9DF884
:1083CC0055009DF85C10084307D09DF84800410605
:1083DC000CD560891EF092F930B140F2351011F0D5
:1083EC00CCF819B0BDE8F08F9DF84800C0F3401AE6
:1083FC0000F00C0910F0200F18BFB9F1040F21D1B7
:10840C00E08D9DF8483010F080010CD15A060AD549
:10841C009DF84920920706D143F0040202F00C02A9
:10842C000C2A40F0C2804FF00008012213F0030325
:10843C001ED0012B4BD0022BD3D1A08912A91BF03B
:10844C0011FECEE7A58924F0D9F8854202D1E08D42
:10845C00010609D4A58924F0D1F8854200F090805A
:10846C00E08D010600F18C8000067ED4A08980E0AE
:10847C00504DEB7A012B02D1A379002B7DD0022336
:10848C00A7898DF84430ADF83C70A9BBB9F1040F45
:10849C0079D1207CDFF820918DF85E00D9F80000AE
:1084AC0000289ED024F0AAF887429AD1E08D217939
:1084BC0094F83020D9F8005043460492CDE9001AC4
:1084CC00CDE902600FA812A95A46A84789E70029EE
:1084DC0018BF012152EA010003D1A08912A915F09D
:1084EC006CFAA0890797ADF81800A0798DF81A00DE
:1084FC0006A81AF03DF974E7ADF8300016989DF80F
:10850C004A109DF84B208DF8203094F832300B90A7
:10851C0060898DF82310DDF84E108DF8222094F828
:10852C0030208DF83830ADF81800A88CCDF8261016
:10853C009DF85C108DF83720ADF82400207CADF848
:10854C002A10A17C8DF8320020798DF834109DF81A
:10855C005F108DF833009DF85D008DF836108DF8A6
:10856C00350006A801F00EFB3BE7A089ADF86200D0
:10857C00608912A91FF0DEFB10B14FF49A702EE740
:10858C004FF0010A3CE71AB912A9384615F015FA52
:10859C00A07CE17CAA8C5B46CDE9001ACDE9026097
:1085AC0012A80FA90FF018FC1BE74FF001080022CE
:1085BC003CE700BFC05E0020F42200202DE9F04F04
:1085CC0093B004461FF06AFA08B11120FAE0207F3C
:1085DC004FF6FE75D0B17D480078810041EA40101D
:1085EC0061882077FF2021F0DDF898B1E08A4FF602
:1085FC00FE7A05F1010B002640F00400E082207F9A
:10860C0040F001002077402004900AE04FF6FE7AFB
:10861C00002002E04FF6FE7A4020049001264FF62F
:10862C00FE7B678838461EF069F808B1002060763A
:10863C0094F81A80B8F1000F04D1654890F80080C6
:10864C0084F81A8094F90000C5B2B0F1FF3F07DD41
:10865C00E07E40B95F480178E1760131017002E0BB
:10866C0005F003052570207EDFF86891012805D1FF
:10867C0099F80B0010B90DB90020207699F80E006E
:10868C0080072BD576B138461EF038F830B34DB193
:10869C00206900780A2821D8012101FA00F010F491
:1086AC00836F1BD0E08A410606D5B8F1010F03D1C8
:1086BC0020F00400E08211E0A188E07E627DADF83C
:1086CC0022708DF82A80ADF824108DF82B0006A8A6
:1086DC0003F0D2FE00283FF478AF2578012D07D1A6
:1086EC0020690078022803D1E08A40F04000E08243
:1086FC00E18A86F0010001F0400140EA9110A8BB2C
:10870C0099F80E00800731D5049DA71D6188607E05
:10871C003A462B4613F034FF28B100206076E08AED
:10872C0040F02000E082387870B1618804F10800D4
:10873C001DF002FA83466088834504BF0020387020
:10874C00E08A40F04000E0822078012804D0A18823
:10875C0060882A460FF004FFA18860882A460DF035
:10876C00A1FB18B1E08A40F02000E0820DF1170166
:10877C00204607F083FB06461FFA8BF0504508BFD6
:10878C00B4F802B0EEB12078617D94F82C50B9F8B1
:10879C0016209DF8173007948DF81800608DADF8F1
:1087AC001A00E08A06ACCDE90254CDE900101FFA9C
:1087BC008BF130460EF04CF9102803D1304624F0E2
:1087CC00DAFA102013B0BDE8F08F00BFD3260020DA
:1087DC0065F00200C05E00202DE9F04F97B0044612
:1087EC0080690DF15B0200214FF0000890F800B099
:1087FC009C200CF0B1FF7B480078012808D80020A1
:10880C0004211DF0B7FE80469DF85B00404400E05B
:10881C000120C1B200258DF85B0059457DD9A0EB34
:10882C000B060221F0B2022828BF0E461A20704314
:10883C00C0B224F0A2FA0027002800F0BF800994EF
:10884C000BA907965FFA86FACDF814805FFA88F6C2
:10885C000446D8464FF000090690CDF820B00431FC
:10886C000A915FFA89F050455DD25FFA88F0B04208
:10887C0056D220F057FE00284AD05B490546888C1A
:10888C0039312080A01C24F019FA4FF60270A4F89C
:10889C00170028888DF82C706082ADF82E00A97A0C
:1088AC0061760BA812F0A0FD014604F10A00012923
:1088BC0003D10A9924F002FA03E04FF0FF31416032
:1088CC000160287948B1484991F8381001310228E3
:1088DC00217612D80221012811E04348022190F898
:1088EC0038006175298800290A4618BF01222275B3
:1088FC0018BF411E2176002008E0012103282175B4
:10890C0002D16775012001E001206075A0751A3451
:10891C0008F1010809F10109A3E7002600274DE041
:10892C000598CBFA50F830480FAD4FF0020BAE1C47
:10893C0000F139075FFA89F050453AD25FFA88F1B5
:10894C0087202A460CF008FFBDF8460039462080E7
:10895C00A01C24F0B3F904F10A00314624F0AEF95E
:10896C00BDF83C001F49204B012209F1010908F117
:10897C00010860820978022938BF022293F8383046
:10898C006275A3F1010238BF4FF0FF3202294FF09C
:10899C000001227638BF012184F817B04900A17577
:1089AC00002818BF01209DF84E10207561761A34EE
:1089BC00C0E7069FDDE908B4079E0025607CF1B294
:1089CC009DF85B300022CDE90275CDE900B1A11C08
:1089DC000AF004FE17B1384624F0CDF917B0BDE803
:1089EC00F08F00BF1C250020C05E00202DE9F04751
:1089FC008AB0DFF8C0810446D8F80000416E02A8A6
:108A0C008847DFF8B4A1DAF80800016C096811B9DD
:108A1C00D0F84C058047694801210170DAF80C0048
:108A2C00C068007830B9DAF808000021D0F8582472
:108A3C000120904723F097FF476805893878C0F3E9
:108A4C00401128460FF08EFEDFF874910790D9F88C
:108A5C00101019B123F087FF0C308847D9F80800A3
:108A6C0008B18047089057480078F0B1D9F8201029
:108A7C00B9B1884755490028554B0A4608BF023200
:108A8C0012781A708DF82420CA1C002818BF4A1CB2
:108A9C0010788DF825004C481978022908BF02304F
:108AAC0000E0494801880131018016F051FC4A4828
:108ABC00484E0078F57350B123F055FF007D30B16E
:108ACC00284623F055F920F027F900286BD0002513
:108ADC003761758023F074FD07467580059524B1C8
:108AEC00012C31D13D483E49C1613C483949027B9A
:108AFC00437BC47D416045804D6002F0F0020273FF
:108B0C0003F0F0020232427304F0F0020432C27538
:108B1C004A7B22F00F02531C4B73DAF808301B6CA3
:108B2C001C6864682478A40608D52E4C42F0020216
:108B3C004C601B685B689B784A73A3732A4E706009
:108B4C00707B00F0F00070732848D8F800100822F1
:108B5C00274B0C6D00210068CDE9002102AA31469B
:108B6C00A0472449B0F1FF3F088007DD224819498E
:108B7C000160224801780131017010E0D9F8004001
:108B8C0044B1DAF80800002100220023006C0068D0
:108B9C000C30A047012041F2883114F0E3FD384637
:108BAC0024F023F802E0E1200BF0E0FC0AB0BDE871
:108BBC00F08700BFA46D00200C010020BF26002010
:108BCC00BCEB0200F4230020FC6B00200C6D002099
:108BDC00156E0020E86A0020B026002018690020DD
:108BEC00801A0600706B00204C240020C825002041
:108BFC00D5A90000F86D0020F8230020F1230020F7
:108C0C002DE9F04F8DB044698246207800EB40008E
:108C1C00013024F024F9002800F0C0808146671C44
:108C2C0000260DF11C0800252078864226D2DAF8A1
:108C3C0000003A8843468188007D1CF0A8FE00287D
:108C4C0078D0B8789DF82210884275D19DF8231001
:108C5C008A0773D5890673D4099911B11FF062FD87
:108C6C0006E0DAF800003A888188007D20F038FAB6
:108C7C00ADF81A00054407370136D5E7002089F80E
:108C8C000000A8B224F0EBF8002800F08480CDF8A6
:108C9C0010904FF000094FF0000806460590207820
:108CAC0080456CD204EB0905DAF800002F46818868
:108CBC0037F8012F007D07AB1CF069FE00285ED051
:108CCC00B5F80100059921F8090001EB0900C0F87D
:108CDC000360099880B10DF11C0B30460DF11A029E
:108CEC00594620F0B8FBDAF800105A463B46087D8E
:108CFC0006311AF0E3FE13E0DAF80000B5F80120B3
:108D0C000DF11A038188007D009333461FF022FD7C
:108D1C00DAF800106B68087D063107AA1DF09CFB81
:108D2C00002840D1BDF81A0009F1070908F1010823
:108D3C000644B4E7862004E08D2002E0882000E0A1
:108D4C007E2089F801000121388889F80010A9F8E3
:108D5C000200DAF800109AF8043001259AF80A405B
:108D6C008A88087D25EAD30306310294CDE90035C3
:108D7C004B4613F07FF9484623F01BFF0FE0DDF85C
:108D8C001090002089F80100012089F80000059856
:108D9C0023F00FFFDDE7484623F00BFF00252846A4
:108DAC000DB0BDE8F08FDDF8109089F80100B5F832
:108DBC000100A9F8020005980AACC51CB8F1000F17
:108DCC00E2D0DAF8000035F8032C23468188007DC8
:108DDC001CF0DDFD0028D7D00C9F5FB12E689DF8EC
:108DEC002E0031461FF09EFC02463846314623F0D9
:108DFC00D7FA07E0DAF800102B682246087D063116
:108E0C001DF02AFB0735A8F10108D7E72DE9F04F33
:108E1C008BB0846906462588B4F8029028461DF06C
:108E2C006DFC01280DD1307C717C00228023CDE9B2
:108E3C000052CDE90220B21C48F2060018F070FC7A
:108E4C00D8E028461DF05AFC20B96D4800888542B0
:108E5C0040F0C78008962679651D5EB1700023F03E
:108E6C008CFF38B10246304629460A9223F0B7F8F7
:108E7C00054602E0002000260A9015F8017B57B148
:108E8C00780023F07AFF30B1024638462946099221
:108E9C0023F0A5F802E0002000270990B81914214E
:108EAC00DFF864B14FF6FF754FF0000801EB40009E
:108EBC00C0B207907800069070000590DBF800B007
:108ECC00BBF1000F69D0DBF8040001780029F5D064
:108EDC009BF80E20D207F1D0DBF808401CB1012022
:108EEC00A047824601E0D0F808A0BAF1000FE5D007
:108EFC00BAF80200814518BFA94526D1DAF8083026
:108F0C009AF807200A9930461FF0B0FC40B9DAF8FD
:108F1C0010309AF80C20099938461FF0A7FCA0B124
:108F2C00079820F021FF38B30546D2202870089806
:108F3C0040882F732E7168804EB10A99059A05F1FD
:108F4C001400A86023F064F903E014BBB6E700201A
:108F5C00A86047B105EB46000999069A14302861C0
:108F6C0023F056F901E000202861DBF804002946C3
:108F7C004068007818F0F8FA9AF80000234A5FFA73
:108F8C0088F108F10108002C4FF6FF7550543FF49E
:108F9C0095AF504623F0EFFE90E7089C0A9D5FEAE0
:108FAC00086011D016485FFA88F3227C617C008837
:108FBC00CDE9000315480023CDE90202A21C48F2BA
:108FCC00060018F0ADFB01E0207BB0B115B12846CE
:108FDC0023F0D1FE099868B10BB0BDE8F04F23F037
:108FEC00CABE08480078012804D8307C717C002265
:108FFC0081231CE70BB0BDE8F08F4FF00008D1E7E0
:10900C00D86C00201C2500207C6D0020AC66002054
:10901C002DE9F04F93B0DDF870A006461D46049282
:10902C008B4650461FF0D6FA044650461FF0BAFA4B
:10903C0000270790002C00F0E580002D18BF0125BB
:10904C00680100F14001BBF1000F4FF0000B08BFAD
:10905C00690103914FF6FE754FF00A0108BF082114
:10906C00029109A90431019100F108010C3006911B
:10907C0005909AF81000834580F0BF80200600F020
:10908C00BC800AEBCB0898F81C00C00740F0B280FB
:10909C0098F8160028B101200F97CDE90D770890AC
:1090AC001EE0B8F8180023F030FD88B1007940F0CC
:1090BC00020003280CD198F81C00002140F080001D
:1090CC0088F81C000798000603D10020079091E057
:1090DC00012198F81600CDE90D770F970891B8B1DA
:1090EC004A49B8F8180091F86810012908D1FF21F5
:1090FC00ADF83400069841F2080988F81A1023E0FC
:10910C00B080681C4FF00C09ADF8340005981BE0DA
:10911C00B8F81800A84213D104208DF8240098F850
:10912C001D00ADF8300009A819F04AFB0198002188
:10913C0000220023B580ADF8345017F037F901E068
:10914C00ADF83400DDE902908DF8360001208DF881
:10915C003900307D8DF838000DA808F0D1FB9DF852
:10916C00480090BB109804994176417DA0F8169068
:10917C0088F81B1098F8161019B1244991F868104A
:10918C000177BAF80A100185BAF8121041859AF8DD
:10919C00141080F82C109AF8051080F83A1098F8F2
:1091AC001A1080F83B103189A0F84010717D80F8BE
:1091BC00491072683169C263406C327D23F028F823
:1091CC000DA81BF027FF9DF8480098F81C1041F0E3
:1091DC00010288F81C2020B141F0090088F81C001D
:1091EC0006E008980799013C80F00100091A0791E4
:1091FC004FF6FE750BF1010B3BE75046002117F0C3
:10920C0004FC0746384613B0BDE8F08FC05E002062
:10921C002DE9F04F8DB00746C089144689460730BA
:10922C0086B2304611F084FA0546FF280AD1304642
:10923C00FAF774F8B04205DA70480778002F08BFC7
:10924C000527A3E06D4E3078C0B91CB1022C15D1A6
:10925C00FF2D13D1387A002203238DF81C00786877
:10926C00009206906648C188C07805AA02F0D6FD27
:10927C009DF824003874BDF82000B881DFF880B167
:10928C00002104239BF80340BBF806A00CAA20463F
:10929C0022F07EFF9DF830007E2805D120467C21EF
:1092AC001EF054F89DF830007C286BD1FD8905F137
:1092BC0007081AFA88F0B0F5005F65D8BB88C5F3CB
:1092CC0085120490F88849461FFA88F94FEA850CF4
:1092DC008DF82DC042EA83128DF82A00C0F30120CC
:1092EC008DF82C209A088DF82B203A7A05EB0A077A
:1092FC00B9F10D0F40EA82008DF829004AD23F489F
:10930C002A460197CDF80CC000F11C06304623F01C
:10931C00A9FDDDF829007119002200270291705176
:10932C009DF82D000871681D81B2304623F07EF93E
:10933C00DDF8291032464B46715196212F4D8DF890
:10934C002F10039923F066F802998DF82E000B98D4
:10935C00C1F80300204651461DF008FA04EB440105
:10936C00049A28700BEB81018A83BBF806104144E8
:10937C00ABF8061050B1019881B2204619F046FEA8
:10938C002F7803E0012700E00527377038460DB031
:10939C00BDE8F08F894608462946002223F046F99D
:1093AC000DF12901052221F0D5FE96214A462B46C6
:1093BC008DF82F109DF82D1023F02CF851468DF8B8
:1093CC002E0020461DF0D2F93070B9B220460DF1B6
:1093DC00290207231DF0CAF9317851EA00073770CA
:1093EC00D4D104EB4400049900270BEB800081835B
:1093FC00BBF806004044ABF80600C7E70822002083
:10940C00006600202DE9FE4F1D4614460F4681468E
:10941C0023F0D6F8DFF8C0A183464FF6FD78DAE9E1
:10942C000010494518BF084660B1B83023F077FCEE
:10943C0040B19AF82400CAF8209040F004008AF851
:10944C0024009FE021F0B4F9002868D00646634858
:10945C00CDF808B0DDE90CB823F0C4FB604908F086
:10946C00200EB1F8540001306FF31F30A1F85400F6
:10947C00B5605C480025C6E903792268D4F80C80F5
:10948C0086F83250C6E908550BEA000C207C726352
:10949C002279C6E906CEC6F8408086F8440086F8E4
:1094AC003820B1F8541086F83350D4E9055331867E
:1094BC00A168C6E91253F163A18BA6F8501028B924
:1094CC00B8F1000F1CBF012086F844004AB9387B64
:1094DC0000F00F00022804D1012086F83800B8688B
:1094EC007063DDF808B00822FF2353FA82F23C4681
:1094FC00D0B2851A18BF01257F680FB1002DF4D1A9
:10950C00208800F47C40B0F5305F0BD196F8330026
:10951C000022082340F0100086F8330004E008F124
:10952C0001082FE0002202234CEA03004EEA02015C
:10953C002B4DC6E90601DAF82000484507D19AF808
:10954C002400C1071CBF00F0FE008AF82400264846
:10955C00046854B1A96CEA6C05F1400005F13803BC
:10956C0000903046A047033013D1FD209AF8241008
:10957C00CAF820904FFA80F841F004018AF82410C0
:10958C0022F026FE584623F030FB0FFA88F0BDE897
:10959C00FE8FB6F83080B5F85410414501D022F05A
:1095AC0017FEC0B2012801D8FE20DFE7002089F8A1
:1095BC00FC0096F8330040F0800086F83300A86B6E
:1095CC00B04205D0F068007B00F00F000228D9D122
:1095DC0016F086F9D6E700BFE81E0020B063002025
:1095EC00A81F0020FFEFFF9F80250020F0B597B04B
:1095FC0004460A2048218DF80A004FF6FF70ADF89A
:10960C0008002068C0F3411201EA1011022A08BFB9
:10961C000131002A08BF1031202303EAD02503EAC8
:10962C00D00300F00700022A18BF29441844032A6B
:10963C000DF10F0508BF4030012A08BF803002220F
:10964C00022740EA012040F01800ADF80C0003A9F5
:10965C00284622F0A5FE206800F0070002280BD057
:10966C00C8B9A81D211D042222F09AFE00208DF8F5
:10967C005000606815900EE004F10806A81C082242
:10968C00314622F08DFE8DF8507014A83146082218
:10969C00043022F085FE05F10A0004F1100123F0DC
:1096AC00BFFAA17805F10B00C9070CBF02A904F1A0
:1096BC00340123F0BEFA2068434E0DF10B01012258
:1096CC00C0F344208DF80B0005F10D00B04705F1F7
:1096DC000E0004F120010422B04705F1120004F140
:1096EC0024011022B04705F1220004F111010822D7
:1096FC00B04705F12A0004F11A010222B04705F126
:10970C002C00FF21102222F0A0FC2068C0F3411194
:10971C000139012920D8BDF80C2000F06000D10BD4
:10972C00402808BFC2F3002105F13600012222F0C7
:10973C008CFC05F1370004F11C0123F07AFAA078B7
:10974C00C00716D114A81AF014FFADF8060005F1E5
:10975C0039000DF1060110E005F13600002101225F
:10976C0022F073FC05F13900FF21022222F06DFC7E
:10977C0005E005F1390004F1340123F05AFA05F142
:10978C003B00FF21042222F060FC05F13F0004F1B4
:10979C00360123F045FA9DF80F1005F1400011F049
:1097AC00180F04D0FF21012222F04FFC03E00DF131
:1097BC000A0123F035FA21680DF10F000122FAF7A6
:1097CC009DFE17B0F0BD00BFADC302002DE9FF41F7
:1097DC00DFF8BC81002003900290D8F83840B4B375
:1097EC00D8F84C0010B9D8F8480070B3D8F8480035
:1097FC0060B12069D8F848100969814206D194F803
:10980C003300C00602D5D8F84C0090B1002702A84E
:10981C0087F0010103AA11F0B3FE0546FFB9F5B1BB
:10982C000299002900F09D805A4821F009FF002779
:10983C0014E0D8F84800C06840880028F9D0D8F85F
:10984C004800C06840880128F3D00127DFE7524860
:10985C000221283023F0A5FA0027002500242CB380
:10986C004E48466816B30298B0FA80F0400928407A
:10987C0001281BD1D8F84800D8F84C10039A87F06F
:10988C000103CDE9003208F1380208F14003B0477A
:10989C00012868D0022809D1D8F8480001220123F8
:1098AC000069D8F84810B1F9301065E02046002C5A
:1098BC0018BF01203840012851D13948216940682E
:1098CC00814203D034484FF4806145E0029800286F
:1098DC0018BF01202840012806D1D8F8480018B933
:1098EC00D8F84C0000284DD0082021F029FB94F822
:1098FC0033004C25C00658BF482508F1380020F02D
:10990C004AFD48F80500274BD4E90601C2439A608A
:10991C00DA681043D860C843186058680843214679
:10992C0058600820E56820F063FF284620F0A0FE70
:10993C00288843F60601411A022906D3B0F5C15F07
:10994C0003D040F60201884203D10120294620F0C1
:10995C004FFF11484FF08041283023F022FABDE828
:10996C00FF8100277BE70398002818BF0446B4F951
:10997C0030102069012200230092002207F086F9A2
:10998C00BDE8FF8108201DF063FDBDE8FF8100BF2D
:10999C00A81F0020F4630020E81E00208025002072
:1099AC00481D0020081004402DE9F0478AB0684D8E
:1099BC002868416E02A88847664FF87918B1B879C3
:1099CC0008B10020C0E022F0FBFDDFF88CA180463E
:1099DC0000249AF8000080074FF0000005D47D2089
:1099EC0000210EF0BFFE8DF818408DF80C4002944B
:1099FC005A4C0790616911B19AF800008847E068E9
:109A0C0008B180470890387A98B1606A88B180476D
:109A1C005349544B8A1D002818BF0A1D12781A701E
:109A2C008DF82420CA1D002818BF4A1D10788DF807
:109A3C0025004D4EDFF8349100200590317BF27EED
:109A4C00B0607080D9F8080001F07001803131737A
:109A5C0002F08001D0F82824F4206331F176032140
:109A6C008DF8181006F11C019047387980B99AF8D6
:109A7C00000080060CD52868C06B8047317BB06035
:109A8C00029001F0F0010231317301218DF80C10BC
:109A9C0029683748344E384B0D6D4FF08071006893
:109AAC0001913449009102AA3146A8470546334832
:109ABC00B5F1FF3F058035DDB87900210024013078
:109ACC00B871787901307871FE60F8790130F871ED
:109ADC00022013F047FE3C712948D9F80820018870
:109AEC00D2F8AC30D2F8D4201C7841EAC411D48C12
:109AFC000180D2E9117193F800C0538D7486C48132
:109B0C00C0F80710C0F803708381508DC6E90A7144
:109B1C000CF001013086308B20F0800040EAC1103F
:109B2C00308309E0626812B10020002190470220C6
:109B3C0041F2883113F016FE404623F056F800200F
:109B4C00B5F1FF3FC8BF01200AB0BDE8F08700BFE8
:109B5C00A46D0020EC2300201C6E0020BCEB020046
:109B6C000C6D0020146E0020486500200C010020B4
:109B7C00C8250020200043000D310100F66D0020A7
:109B8C00506C0020F0B587B004466F48007878B16F
:109B9C00228B0020E57A01210390CDE901008DF89C
:109BAC000910500706D402F008030121002008E038
:109BBC00BA20AAE0402012F008038DF8060008BF76
:109BCC000321402606EA82064BB1C02093068DF88D
:109BDC0006004FF0010358BF02238DF807305309DC
:109BEC0003EA121202F00802324342EA0106217A19
:109BFC0003290AD8DFE801F00215112540F004070B
:109C0C0022F0FCFC8DF8067008E00F291DD140F005
:109C1C00080046F004068DF806002088ADF8040014
:109C2C0013E04A4991F86810002900F080802788D9
:109C3C0040F0080006F58056FF258DF806003846E2
:109C4C007EE001A920461EF08DF80027208BC0076E
:109C5C000ED09DF8060010F00C0F58D09DF80600A1
:109C6C0000F00C01042904BF40F020008DF8060020
:109C7C00A07C8DF8080001A807F042FE9DF81800A2
:109C8C00002842D10498C682B4F81B10A0F8191011
:109C9C00217A012903D12D4991F868100177A17E11
:109CAC00E37F0185228B80F82C301306428508D582
:109CBC00D20506D5417D94F820001FF024FBA17E2F
:109CCC000498878780F83B5080F84A10A17A80F876
:109CDC003A10D4F80E10C0F83E10A17F80F84B104B
:109CEC00617F80F84910406C6169628A22F090FAB9
:109CFC00208B400604D51648016809B101A8884795
:109D0C0001A81BF087F99DF8180007B0F0BD20885A
:109D1C0018F0EAF948B19DF8060040F020008DF8E3
:109D2C000600208BC00799D1A2E7BB20EDE740F0DD
:109D3C000C00278846F004068DF806004FF6FD70DF
:109D4C00ADF8040082E700BFE4220020C05E0020D2
:109D5C00702600202DE9F04F89B0714F14460A4649
:109D6C00064610460492B98C1EF0ECFB054610B169
:109D7C006878002866D0B06A4FF00E09B34690F8A8
:109D8C000180867890F805A05FEA886158BF4FF093
:109D9C000609B0F80300039004981CF057FD18F066
:109DAC00870F4CD108F01801182948D09BF81C10CB
:109DBC00894544D100EB0A020021BBF80C00B146E6
:109DCC000091D1B292460E46049B4946324610F0A1
:109DDC000BF8032836D008F07801B8BB18F0180F30
:109DEC0062D05FEAC86088464FF0030058BF01207C
:109DFC0040EA0108BBF80C00414612F081FB88B127
:109E0C00817911F0180F0DD0417901290AD14DB18A
:109E1C00B98C40881EF096FB20B1407810B169785F
:109E2C0088420FD322F0EFFA88B94FF0FF30208030
:109E3C009BF8080000286BD0DBF8181069E0D320E1
:109E4C000FF09BFB002009B0BDE8F08F88462088FE
:109E5C004FF6FF718842F5D10121BBF80C00324658
:109E6C0000914946049B0FF0BFFF0398414685B211
:109E7C0028461BF051FFF98A88420CD1284622F063
:109E8C0044FE20B300790138012820D805A92846C2
:109E9C001EF078FC21E0DBF8280080F805A009B062
:109EAC00BDE8F04F20F0A4BB787B884608B122F0C7
:109EBC00AAFA03984FF6FE710022434680B205F0D1
:109ECC0057F80028C3D14FF6FF702080C4E721F06B
:109EDC007DFE014605A822F0F1FE9BF80800012842
:109EEC0004D1DBF8181007A822F0E8FEDBF82810E4
:109EFC00BBF80C00497805AA07ABCDE9003200226B
:109F0C004B4641F030010291294609F09BFF99E73D
:109F1C000021BBF80C00324622F013FF97E700BF7C
:109F2C00C05E00202DE9F04F95B0064600201022AF
:109F3C008DF844001090CDE90E000BA822F03AFBEE
:109F4C0020B10124204615B0BDE8F08F96F826000C
:109F5C0003280DD196F8400022F00FFF0028F0D016
:109F6C0096F8402006F14101044622F051F900E038
:109F7C00002496F82500019402288DF8480003D09F
:109F8C0048B9F06A139006E012A806F118010822ED
:109F9C00043022F03DF93446002054F8342F12A935
:109FAC000EAB18F0BCFB14F80C0C14F80F7C6FF013
:109FBC00330814F80E9C14F80DAC002808BF6FF091
:109FCC0073080625022F08BF0725002F08BF0A2596
:109FDC0014F80BBCB9F1020F04D0B9F1030F21D165
:109FEC00284603E096F840000544E8B222F0C5FE8E
:109FFC00C0B147EAC90180F80080871C804641EA5D
:10A00C004A1141EA8B11417096F82510022910D0A3
:10A01C00B9B906F12C013846042222F0F9F808F1FE
:10A02C0006070EE0019800283FF48BAF22F0A3FE48
:10A03C0087E706F130013846012222F0E9F808F1F1
:10A04C00030738462146042222F0E2F896F826004F
:10A05C00022806D196F84020381D06F1410122F065
:10A06C00D7F802A822F05CFCE8B2CDF80C8008907E
:10A07C000BA802900EA8069040F20D40ADF82800F7
:10A08C0006F13C00079096F8260003280DD196F8AF
:10A09C004000019D09901548CDE90455006802A9BE
:10A0AC0022F08BFD18B1012409E001240CE096F894
:10A0BC00402006F14100294622F0AAF80024284647
:10A0CC0022F059FE96F8260002280BD100200990A8
:10A0DC00CDE904000548006802A922F06EFD0028B5
:10A0EC0008BF0446404622F046FE2BE7506D002088
:10A0FC0070B58AB000F11605044628461CF0BEFC6B
:10A10C0067480078013801282BD800201021012243
:10A11C0014238DF8110005AE0DF11100CDE90210DC
:10A12C00CDE900620DF11201042000221CF0F2FEB8
:10A13C0050B15C48006804A905AE324611F040FCF1
:10A14C000228ADF812000CD806F1080029460822A6
:10A15C0022F05EF8BDF812100420142233461EF0D3
:10A16C000FFF2846FF21082221F050FC10B14E4869
:10A17C000121017028461DF007FA207901380528C5
:10A18C0000F28B80DFE800F00389345C8903A01DAA
:10A19C000021102913D0425C0131002AF9D06179D9
:10A1AC001FF0BAFE4348424D90F8410008B12878A0
:10A1BC00D8B160790FF0A2F80020287015E03D4866
:10A1CC0090F8410088B905AC002062210025224698
:10A1DC0011F048FE204600211FF09EFE00200FF0DB
:10A1EC008DF8CDE90755CDE9055520F043FF54E036
:10A1FC000DF1120128461FF032F860B10DF1120278
:10A20C004FF6FE7029461EF0C1FC284600210022A4
:10A21C00002316F0CBF8BDF8126005A930461EF0ED
:10A22C0041F8059828B905A81BF0EEFD08B905986A
:10A23C000680A11D284611F0E3FF14F0A1FD2CE0CF
:10A24C001A4E307848B30DF1120105AA284611F0C8
:10A25C00B7FB01469DF81200F8B10025012014222D
:10A26C00ADF8240006958DF82650059505AB042015
:10A27C001EF086FE06344FF481701021224622F027
:10A28C0001FB28B94FF481701021224622F000FB0B
:10A29C0001200321357019F03FF90AB070BD00BFE1
:10A2AC001C250020386D0020076E0020592000204E
:10A2BC0058200020C05E00202DE9F04788B00446ED
:10A2CC004FF0FF3002214FF6FE79CDE90200E08914
:10A2DC00002808BF0821A66916F801A030B165480E
:10A2EC0035880088854208D1634E31E0624831469A
:10A2FC0020F0C8F8F0B15F4829E0284622F005FCB0
:10A30C00B0B301790026012933D140880DF1100832
:10A31C008DF81060ADF81C00404618F051FA064656
:10A32C00002818BF08F10406BAF1000F18BF4FF04F
:10A33C00FF3A0DE0304622F04CFCB0B10179013906
:10A34C00012912D8BAF1000F18BF4FF0FF3A058857
:10A35C004D4518BF002E05D1207B002848D1474819
:10A36C0040680EE04548406813E04FF6FE7500E08B
:10A37C000026207BE0BB414840684D4518BF002EAD
:10A38C0007D1E1894FF0810881B100F8018B02AE51
:10A39C0011E05FFA8AF1022902D24FF0000807E0BF
:10A3AC00217B012924D04FF0800801E009F101053F
:10A3BC0000F8018B0EB1314600E002A922F07EFCC0
:10A3CC00064605805FFA8AF00B27012808BFB8F112
:10A3DC00000F10D0E289294D1020A11CFBB2A870EF
:10A3EC0004F1110042F4004217F0CEFA0020A870DC
:10A3FC0008B0BDE8F0871F48A9B200888142E9D1B6
:10A40C0000250DF107008DF8075016F05DFB98B193
:10A41C00E1890322002908BF0922A1698B5C9DF800
:10A42C00072000EB43019A4209D9D21A0D258DF869
:10A43C00072005EB420706E00C27B570CAE700229F
:10A44C000D278DF80720F370331DB27012060DD056
:10A45C0011F8022B03F8022B11F8012C03F8012C34
:10A46C009DF80720013A8DF80720EFE722F083FCD6
:10A47C00B0E700BFD86C00202C6D002070250020A8
:10A48C002DE9F0478AB0002900F0D180149E0746D0
:10A49C00007A0D469946904631078DF8020012D489
:10A4AC00387A02240F2800F2C3800121814011F078
:10A4BC000B0F19D003288DF80C0024D101A83946B4
:10A4CC0022F0FCFB22E0022840F0B1803C8822F014
:10A4DC0095F88442E4D038880121032213F052F815
:10A4EC000028DDD0CD24A3E048F20400014200F0A6
:10A4FC009F8038881CF002F9002800F094800F200F
:10A50C0038728DF80C003888ADF80400B00714D4FC
:10A51C000020ADF814004848006888B14168A94291
:10A52C00FAD1826862B129780220904768B101881B
:10A53C00ADF8141022F01FFC07E04FF6FF7002E09C
:10A54C00A86810B14088ADF81400C6F380129DF8CD
:10A55C000C30DDE9121A15988DF8012010225C1EC2
:10A56C0002EAD60218BF01240F2B134618BF43EA88
:10A57C008403F40658BF134606F0400243EA9212D5
:10A58C007307ADF81C2044BF4032ADF81C20069177
:10A59C008DF82000ADF81690ADF81280797A002273
:10A5AC009AF800008DF800208DF80F10B1068DF888
:10A5BC001E00287821498DF80E00097848BF042127
:10A5CC008DF81F1021F0B4F818B1016909B101A878
:10A5DC008847684621F086FB484505D21848016833
:10A5EC00F9B101A8884702E001A8FFF7CBFA0446AD
:10A5FC009DF80C0002280CD1BDF8046021F0FEFF80
:10A60C00864206D19AF800102878424623461BF061
:10A61C0019FC6CB99AF80000002401308AF800008B
:10A62C0006E00224E4E7387A0F287FF443AF0224D3
:10A63C0020460AB0BDE8F0877C6D00205F1C00202E
:10A64C00E4250020F0B587B0674C054694F8370038
:10A65C0028B9664F042138781BF022FBF0B164480E
:10A66C004078C8B994F83A0005F0CE0668B1A8074E
:10A67C000BD594F83700C00607D420F043FB042018
:10A68C000121FAF70DFE86F0020694F8371006F059
:10A69C003F00084384F8370007B0F0BD94F837004A
:10A6AC0005F00E066178304384F8370059B1002864
:10A6BC0049D04F48002101703878042107B0BDE81B
:10A6CC00F04015F0E3BD0120607020F0E9FF012897
:10A6DC0007D1562022F065FA18B10146562022F017
:10A6EC0005FA02F05DF804F13A035520002101222D
:10A6FC0021F0ACFB94F83A0078B33E48007801386E
:10A70C00012809D83C4D00210822286821F07EF947
:10A71C0010B921F0D5FC30B335480721017094F8FD
:10A72C0037000021304340F0100084F8370000203F
:10A73C0006F062FCA0B100201FF048F807200021B1
:10A74C00FAF7AEFDA8E72A4807210170072000217F
:10A75C0007B0BDE8F040FAF7A3BD94F83700A6E7C0
:10A76C0011F062F898E728680DF11B0101AA11F0AD
:10A77C0027F90546214800780028CDD09DF8140013
:10A78C00FD28C9D00228C7D01D480088854217D2A1
:10A79C0001AE1421304621F0C3FBFF2029461422C0
:10A7AC0033468DF8140004201EF0EAFB154905EB26
:10A7BC004500002241F8202001EB800042724260EB
:10A7CC0000255520012104F83A5F224622F060F85A
:10A7DC00FF2003211BF0E8FD0548042105703878A3
:10A7EC0015F054FD58E700BF542000200A6E0020DD
:10A7FC00606D00201C250020386D0020C52600202F
:10A80C0054F00200AC68002070B58CB004460020F7
:10A81C008DF82C00CDE906000890A078411E052982
:10A82C0025D82220DFE801F00321212C23036248E4
:10A83C00007820BB22F0CDFA40B9604DA168082207
:10A84C0005F1180021F0E4FC208828805C48007891
:10A85C00022814D1A0680DF1030101AA11F0B0F87F
:10A86C009DF8140038B1B1206CE01B2008E0B32037
:10A87C008DF82C0059E09DF803000028F3D023201C
:10A88C008DF81C000120A17B8DF81A0020888DF812
:10A89C001D102169ADF81800607B0891012804BFD8
:10A8AC0021208DF81A0006A807F02AF89DF82C0034
:10A8BC00D8BB0998456C05202870A0786870A81C36
:10A8CC00616819B1102221F0A3FC04E00021C160E1
:10A8DC00816041600160A078062801D0012803D175
:10A8EC00E078A874133500E01235A168284621F0F1
:10A8FC0067FDA17805F1080006290AD8012202FAA1
:10A90C0001F111F0520F04D02E49096822F0D6F94A
:10A91C0001E0217B017020881BF0F0FE10B109983A
:10A92C000421C1829DF82C0070B12348007838B9FD
:10A93C0022F04FFA20B921480021C0E9061101800C
:10A94C009DF82C000CB070BDA078042814D1A06820
:10A95C0001AD0DF103012A4611F032F806469DF8BF
:10A96C00030018B94FF6FF708642DED0206968B13B
:10A97C0006A80FF0BDF80CE0206918B106A80FF07E
:10A98C00B7F8D2E706A81AF045FBCEE706A81AF0EE
:10A99C0041FBA16805F10800082221F039FC0120D7
:10A9AC00314614222B46ADF814000020CDE90100ED
:10A9BC0004201EF0E5FAB8E71C250020082300202F
:10A9CC00CD260020386D0020F8B5634E01211D46C0
:10A9DC001446F068C068017060480021017060483E
:10A9EC000170B068016C096811B9D0F84C0580474A
:10A9FC005C48076847B15C4822462B464188B068E2
:10AA0C00006C00680C30B84715F0E24F14D0574872
:10AA1C000178013901705448406818B15448C18913
:10AA2C000131C181B068006C006840680078800614
:10AA3C006FD41EF021FA6FE020070CD44A4840680E
:10AA4C0018B14B48C1890131C1814848017801399D
:10AA5C0001701D205EE0454C42F205422078013821
:10AA6C0020704448418841F00400904218D13E487F
:10AA7C00406818B13E48C2890132C2813C484289C3
:10AA8C000132428142F20542E120914208BF1C2072
:10AA9C0009F06CFD207800284AD094F9000040E0C1
:10AAAC00314842F606024188914212D0B1F5105F4E
:10AABC0049D14069334908601AF00CFE2E480078E1
:10AACC0050B32F480168013138BF0160002101816A
:10AADC0022E0406818B12648C1890131C18126485D
:10AAEC000078C8B12548042100780228204808BF06
:10AAFC000621425A0132425221484168013138BF85
:10AB0C0041600189428901318BB20181934288BF36
:10AB1C004181E92009F02AFD1448017841B190F9EE
:10AB2C00000000280ADCB068D0F84C05804705E02E
:10AB3C00B0680021D0F8582400209047F06800211C
:10AB4C00C0680170F8BD406800283FF482AF084827
:10AB5C00C1890131C1817CE70C010020EF23002069
:10AB6C00BF260020BCEB0200E86A0020F123002085
:10AB7C00FC6B002018690020F4230020156E0020C7
:10AB8C00A86C0020B86D00202DE9F04F8BB0064664
:10AB9C00007898468A460792022809D0002840F08F
:10ABAC00B1804FF6FF700424ADF82000022006E0BF
:10ABBC00311D08A80822082421F02AFB03208DF857
:10ABCC0028005E48DFF878B1351D002790F800901A
:10ABDC00B94500F097805BF82700B0B13178027965
:10ABEC008A4212D108302946224620F071F960B110
:10ABFC003078022801D040B909E0BAF1FF0F06D035
:10AC0C005BF82700007C504501D00137E0E7F8B233
:10AC1C00814577D05BF827A00025B8F1010F8AF8A1
:10AC2C0003500FBF4FF00D0848F08C08307840F0FF
:10AC3C00800515F010094FFA88F44FF00B0008BF8F
:10AC4C000320B4F1FF3FC8BF02209AF811209AF8F4
:10AC5C0010309AF8166018F00301CDF81090069297
:10AC6C00CDE902310BD19AF804C0BCF1000F04D02D
:10AC7C00BCF1020F08BF013001E040F00400304489
:10AC8C00C0B2059022F079F8E0B3B446064681468E
:10AC9C00B4F1FF3F0AF1170106F8018BDCBF89F80C
:10ACAC00015009F102060398049B70B300200022A6
:10ACBC00B3FA83F36546B4F1FF3FC8BF01225B09C9
:10ACCC0052EA030808BF46F8040B6246069806F8D9
:10ACDC00010B304621F09CFAB8F1000F04BF0020A4
:10ACEC0070514B465BF82710C878897C0091079906
:10ACFC00019108A9059A0FF0D3FC012802D148460E
:10AD0C0022F039F80BB0BDE8F08F9AF8040028B1A6
:10AD1C000228CBD1029806F8010BC7E7DAF8080035
:10AD2C003070DAF80800000A7070BAF80A00B070D7
:10AD3C009AF80B00F0700436B8E700BF67F0020019
:10AD4C00946D00202DE9F04395B0DFF8A081044606
:10AD5C0098F80200002800F0C680A07800F00700E8
:10AD6C0002288DF848000BD0002840F0BC80A06869
:10AD7C0004211FF05DFF1390A068002604300BE047
:10AD8C00A16812A8043021F0BDFFA16801F10800F0
:10AD9C00A06001F109000E7A411CA160811C0778AA
:10ADAC00A160457847F01000F32808D19DF84800C1
:10ADBC00002840F098801398002840F0948005F10A
:10ADCC0018001EF0D1FF002800F08D80814606741B
:10ADDC000120B5F1FF0689F8030009F1170018BF2F
:10ADEC002E46A168324621F0DBFA89F8166089F804
:10ADFC00117009F1040012A90C2221F0D1FA0120E2
:10AE0C001BF0B6F889F812000520A9F80000A0780C
:10AE1C00000705D599F8030040F0200089F80300DD
:10AE2C00334EA188F08A814241D1D8F8080010B184
:10AE3C008047002857D0D8F80C0010B18047002864
:10AE4C0051D001270DF105010DF1460288F8007073
:10AE5C0012A812F04BFC58B99DF80500810707D4D5
:10AE6C0040F00200BDF846100DF1050321F0F0FB97
:10AE7C0089F80270A179307E0B3188F80400814288
:10AE8C002CD01C4D286821F00BFB38B9286841F2F6
:10AE9C00883121F076FE184821F08DFFA0790B3017
:10AEAC0006F8180FE120314619F00EFE16E012A834
:10AEBC000DF105010DF1460212F018FC58B99DF880
:10AECC000500810707D500F0FD00BDF846100DF117
:10AEDC00050321F0BDFB002089F802000748494614
:10AEEC00007816F041FB15B0BDE8F0835823002024
:10AEFC00C05E0020906D0020C0640020136E002006
:10AF0C00FEB504462C2021F038FF002820614BD0E0
:10AF1C002C2121F005F8256920884FF6FF760DF1DC
:10AF2C000301AE8212F012F948B30DF10300694629
:10AF3C0020F052FABDF80020B24220D0584902EB62
:10AF4C004200AA8206226A82002251F820302A741A
:10AF5C004FF47A72AB6151F820300133B3FBF2F548
:10AF6C0041F8203005FB12324AB901EB8000012177
:10AF7C0001724C484FF40061007815F087F9216993
:10AF8C002088083112F0E2F821F09AF8256970B1A6
:10AF9C004FF4D000C5F81200022028744248016812
:10AFAC00A9610131016021E010202075FEBDA88A45
:10AFBC00B0421BD13D4F05F1080039681FF062FA11
:10AFCC0058B93D6820F002FE014628461FF05AFA97
:10AFDC0018B921F075F800285FD02169208803F09A
:10AFEC00CFFD256900B1AE8200202874A88AB0423A
:10AFFC0031D12F48C17A11BB90F8410001281ED1E4
:10B00C000DF10B02002001213A2301271FF01AFF3A
:10B01C0008B1AE8213E09DF80B002F74A8754FF4A5
:10B02C006810C5F81200234801684A1CA961026027
:10B03C0029B91C484FF40071007815F027F92569DF
:10B04C00A88AB04207D1A1202075284621F093FE92
:10B05C0000202061FEBD287C012801D10E210CE0CE
:10B06C00A06808B10D2108E021F02AF80D2118B9CB
:10B07C00A078C00708BF052125690D482977A1785C
:10B08C0001F00301007B012908BF05206870C0B2E4
:10B09C0021F0FEF821694877FEBD2569A6E700BFBF
:10B0AC0088680020046E0020F8250020386D0020F0
:10B0BC00C05E0020E02300202DE9FC4F83F000430C
:10B0CC0001E02DE9FC4F1F03FF0847EAD2574FEA76
:10B0DC0042284FEA43095FEA595906D147EA080A60
:10B0EC001CBF00210020BDE8FC8F57F000575FF417
:10B0FC00E06E1EF1FF0EF14505D14FF00000190D69
:10B10C000905BDE8FC8F002B05D55FF0000AD8F1CE
:10B11C0000086AEB07070C03E40844EAD0544FEA32
:10B12C0040254FEA4106760D08D144EA050A19BFBD
:10B13C000021002019461046BDE8FC8F44F0005455
:10B14C00764504D10020090D0905BDE8FC8F0029C6
:10B15C0004D55FF0000A6D426AEB0404B6EB090EED
:10B16C0008D5A2463C465746AA464546D046CEF19F
:10B17C00000E4E46BEF1360F5CBF4FF0000B23E0C5
:10B18C00BEF1000F04BF4FF0000B1AE0CEF1390AEC
:10B19C00BAF120092EBF08FA09FB07FA0AFB4BEAA1
:10B1AC00080BDEF1200A07FA0AFA38BFBA4647FA4A
:10B1BC000EF72DBF28FA0EF8AEF1200E4AFA0EF853
:10B1CC00D04415EB08057C4154EA050A02BF002166
:10B1DC000020BDE8FC8F002C58BF4FF0000A06D5AC
:10B1EC005FF0010A5FF0000E6D426EEB0404A6F1F5
:10B1FC0001066D006441FAD515F4806E11D005F48A
:10B20C0080794BEA090B15F5806554F1000428BFD1
:10B21C00761C0BD205F400795BEA090B08BF25F408
:10B22C00006525F4E0656D0044EB0404B61CDEBF3C
:10B23C0000210020BDE8FC8F5FF4E06E1EF1FF0ED4
:10B24C0076450AD34FF0000013F00043FF21C900EC
:10B25C00C91D09051943BDE8FC8F270547EA1530C0
:10B26C00210B41EA065141EACA71BDE8FC8F7047D7
:10B27C0010B5624C20780E2838D8DFE800F0B737CC
:10B28C0037460837373737374037080808005D48E6
:10B29C000078B0B1A078012845D1E0780130E07099
:10B2AC00C0B2032839D859484FF6FF71808C8842B8
:10B2BC0037D05748012101704FF44170A4F80100B8
:10B2CC0031E055480021E170017000201BF04AFB71
:10B2DC0018B120780D38012853D805201FF0D8FA62
:10B2EC0042F21070BDE810401EF04CBE1CF01AFF6C
:10B2FC004A4810210078BDE8104014F0C7BF404800
:10B30C00008800F007000128C1D13E480078F8B150
:10B31C000020BDE8104018F011BF3B480078012810
:10B32C0001D10020A07018F0E5FA1FF081F9344823
:10B33C008078000703D537480078012856D1A078CB
:10B34C00032853D108200121BDE8104002F078BA3F
:10B35C0032481021007814F099FF00201BF002FBFA
:10B36C0048B3207803282BD00A2836D124480088EB
:10B37C0000F00700022830D02448082180F826105D
:10B38C002BE006201FF084FA1D4CA078000704D592
:10B39C004FF40040012102F053FA208800F007001E
:10B3AC00022804D000200021002220F0D9FEBDE8A4
:10B3BC0010401CF0B7BE05201FF06AFA0120A8E768
:10B3CC001CF0B0FE16480078022806D101201EF0B1
:10B3DC00FDF902200121F9F763FF06201FF058FA4E
:10B3EC000748008800F00700022800D110BD00209B
:10B3FC0000210022BDE8104020F0B2BE0423002042
:10B40C00806C0020296E0020FF6D0020C05E0020A3
:10B41C00096E0020DA26002057200020046E002040
:10B42C00606D00202DE9F04788B00646109C002086
:10B43C00DD099A461746C3F3C308E060A06060605C
:10B44C002060E9B1E94621461022484620F0E0FE92
:10B45C0020463146102220F0DBFE484621F0DAFB74
:10B46C000020102805D0315C225C51402154013061
:10B47C00F7E70AF1800A1FFA8AF04FEA102901E077
:10B48C004FEA1A296E46280418D03046214610225D
:10B49C00013D20F0BDFE20463946102220F0B8FEBA
:10B4AC00304621F0B7FB0020102805D0395C225C17
:10B4BC00514021540130F7E70744E4E7B8F1000F9D
:10B4CC0025D068462146102220F0A2FEB8F10E0FBE
:10B4DC0040D30025204639464246E560A5606560AC
:10B4EC00256020F095FE80202146102204F80800EB
:10B4FC0004AE304620F08CFE684621F08BFB102DFC
:10B50C0048D0705D615D484060550135F7E76E4687
:10B51C0021461022304620F07BFE0027802021F0AF
:10B52C0040FA21461022C4F80170C4F80570C4F822
:10B53C0009706773207004AD284620F069FE304610
:10B54C0021F068FB102F42D0E85DE15D4840E055EA
:10B55C000137F7E70026204639464246A681A66009
:10B56C006660266020F054FE80202146102204F8EC
:10B57C00080021F016FA04AD284620F049FE684672
:10B58C0021F048FB102E22D0A85DA15D4840A055AB
:10B59C000136F7E76F4621461022384620F038FE78
:10B5AC00002530462146102221F0FBF9256065600C
:10B5BC00A560A58120F02CFE384621F02BFB102D28
:10B5CC0005D0705D615D484060550135F7E708B006
:10B5DC00BDE8F0872DE9F84FD0E90158D8F80010F4
:10B5EC00CA690A62D20740F0A480D8E9040105F1C7
:10B5FC00C8094FF0000A4FF0000B0843D5F8CC10E7
:10B60C0049680968C1F8040505F130000090BBF1E8
:10B61C00010F00F29780D5F8C000002800F092804E
:10B62C00D5F8E0C0D5F8CC70DC2224232024BCF162
:10B63C00000F08BFD82208BF1C2358F8033008BFDE
:10B64C0018247F68D8F8146058F804403F68D7F87D
:10B65C000415314211D0A16849070ED10168D5F803
:10B66C00D0408C4209D1416939B9D8F800104C6AE4
:10B67C0024F002044C62C7F804659968490702D0AB
:10B68C000BF1010BC3E7AB58002BF9D045F802A026
:10B69C00D5E934121A44BCFA8CF35B09C5F8D420F2
:10B6AC005B01C5F8E0300368994228BF9A420CD27E
:10B6BC002846414602F000FD95F8FE000028DFD038
:10B6CC0020F098FA18BF8862DAE7D9F800204B46C8
:10B6DC0080F810A02AB153690BB11A46FBE702F1AE
:10B6EC0014031860C5F8D4A0BCF1000F4169C0F870
:10B6FC0014A04FF0D800C5F8C01008BFDC202858A3
:10B70C00C5F8D00059B12846414602F0D5FC95F851
:10B71C00FE0050B120F06EFA18BF886205E0D8F830
:10B72C000000416A21F003014162009821F03BFBCB
:10B73C00A6E7D5F8C0203AB103211174BDE8F84F43
:10B74C0005F07EBDBDE8F88F486820F00200486027
:10B75C00486A20F003004862D8E904021043D5F887
:10B76C00CC2052681268D062C2F80405486920F0F7
:10B77C0001004861012008624046BDE8F84F1EF008
:10B78C0015BA70472DE9F04F8BB0DFF8A081044655
:10B79C00D8F80800D0F80001807AC00021F0EDFA4A
:10B7AC000028099000F0B5804FF0000920F008FF48
:10B7BC00009001AEFF270025D8F80800EAB2D0F8B7
:10B7CC000011CB7A9A422CD2D0F88824D020314662
:10B7DC008DF80650ADF80440904700BB9DF8100062
:10B7EC0020B101281BD19DF80F1001E09DF80B1022
:10B7FC00A9B100284FF0080008BF042000218142A5
:10B80C0003D272180131D770F9E73044314680F811
:10B81C000390D8F80800D0F89424D0209047013534
:10B82C00CAE74FF6FF7701AE0DF1140A4FF0FF3B5C
:10B83C004FF00009C9885FFA89F291426BD9ADF8D3
:10B84C000620D0F88824D1203146ADF8044090472A
:10B85C0030B1D8F8080009F10109D0F80011E9E776
:10B86C00BDF80800B842F4D0ADF81400D8F80800C0
:10B87C005146D0F88824D4209047002841D1002587
:10B88C00D8F80820D2F80001C1888D4216D2D2F81F
:10B89C008824D1203146ADF80650ADF804409047CD
:10B8AC0028B9BDF81400BDF80810814201D001354B
:10B8BC00E6E7D8F80800D0F80001C1888D42C8D15D
:10B8CC00CDE907BB099AADF81A70ADF81870807AFB
:10B8DC00C1000020814214D0131808309B88A34269
:10B8EC00F8D11118002241F8082C09990844514646
:10B8FC0020F8047CD8F80800D0F89424D420904781
:10B90C00A7E7009821F071F9099821F034FA192071
:10B91C0008E01A2006E0009821F067F9099821F058
:10B92C002AFA00200BB0BDE8F08F00BF0C010020FC
:10B93C0070B58EB0044680781FF066FF002800F0CA
:10B94C00BF8005466078A0F1E101E873102906D9A3
:10B95C001A2818BFCD2808D01D2806D05EE0012279
:10B96C0002FA01F1584A1142F2D06989090539D419
:10B97C002846002106F0A2FC00284ED05348807BBC
:10B98C00800727D52968086A20B3C97F01AA07F068
:10B99C0035FC6078E92808D12868E27B01234189CD
:10B9AC0000880093E92306F0D9F92868BDF80E1039
:10B9BC0001809DF80920BDF81010BDF80E00002A7A
:10B9CC0018BF012292010AF06DFA18B1688940F093
:10B9DC00200068816A89617828891FF0A9F828817C
:10B9EC00607801E005216973E92861D03848006866
:10B9FC0000B18047374E3068002859D03348807BDF
:10BA0C00800755D52868418900881CF09BFD0028CB
:10BA1C004ED06178326890474AE060788DF8080023
:10BA2C00A07B01958DF80900287C28B101A811F0A4
:10BA3C0027F89DF8083005E001A803F075FE9DF885
:10BA4C000830DBB1E92B00D03BB92868E27B01263A
:10BA5C0041890088009606F081F91C48807B80079C
:10BA6C0026D5687B022802D16889400712D46078F9
:10BA7C00E9281DD1284619F04DFE19E028680088E8
:10BA8C001AF03CFE0028D4D1114800680028D0D010
:10BA9C008047CEE7286800881AF030FE002811BFD6
:10BAAC00032028684FF6FF71018008BF05206873DA
:10BABC00687B022804BF06206873A07810F0A0FEF3
:10BACC001EF09AF80EB070BD01010100C05E00209E
:10BADC003422002038220020FEB50C4615F078FAEE
:10BAEC00A00600F18280200400F1AF80E00607D5AB
:10BAFC002E208DF80400604821F02FF801A888470B
:10BB0C00E00707D025208DF804005B4821F025F8CC
:10BB1C0001A88847A00707D526208DF804005648B1
:10BB2C0021F01BF801A88847600707D527208DF85E
:10BB3C000400514821F011F801A88847200707D5C7
:10BB4C0029208DF804004C4821F007F801A88847FB
:10BB5C00600607D52D20ADF80400474820F0FDFF06
:10BB6C0001A88847200607D53020ADF804004248CC
:10BB7C0020F0F3FF01A88847E00507D53520ADF884
:10BB8C0004003D4820F0E9FF01A88847200505D5B1
:10BB9C003720ADF8040001A821F066F9E00405D5C2
:10BBAC003820ADF8040001A821F05EF9324CA068F1
:10BBBC00D0F898000068B0B120F002FDA168D1F86F
:10BBCC0098100A68029200220A6021F00EF8A06810
:10BBDC00D0F8981002984860A168D1F840138847B3
:10BBEC00A06820F041FD0020FEBD234E02ADB068E0
:10BBFC00C06B04301DF0B4FF002802903FF473AF0B
:10BC0C0020F0DEFCB168C96B0A7B013A0A7320F0A4
:10BC1C00ECFFB1680298D1F89810077848608DF85D
:10BC2C000470417839B1162F0BD1B068D0F8541389
:10BC3C0028468847DBE7B168D1F840138847162FB0
:10BC4C00D5D0B06820F010FDD1E70B4DA868D0F826
:10BC5C009400007814F0F0FF002802903FF446AFF7
:10BC6C00A968D1F898104860A968D1F840138847A2
:10BC7C00A86820F0F9FCE9E70C0100202DE9F0415F
:10BC8C005A4E04465A4DB068D0F8D41091F88380BF
:10BC9C00297819B1D0F84C058047B068016C096857
:10BCAC0011B9D0F84C058047524F0120062C3C703E
:10BCBC0028701ED8DFE804F0040422252B51400024
:10BCCC004E4800214170B068026CD0F8D410106856
:10BCDC004B4AC08A40064FF04E0058BF2520085CE6
:10BCEC00107014BBC97801B3022828BF0220107051
:10BCFC001BE0B068D0F84C0580472EE019F0AAFC88
:10BD0C002BE03E480021417018F0EEFF25E03A4848
:10BD1C0000213A4A0170B068006C006890F8691014
:10BD2C0090F86A0051703649087009F02BFAB06827
:10BD3C00006C006888B940E0B068324A006C016859
:10BD4C0091F86D1011803049006890F86E00002851
:10BD5C0008BF012008701BF019F828480078A0B91A
:10BD6C00B268106C016829B9D2F84C058047B068EC
:10BD7C00006C01684968254A097801F020011170AE
:10BD8C00234900684068807808703878062814D8F1
:10BD9C00012101FA00F010F04C0F0ED020F010FC35
:10BDAC000446387802280AD183202870204620F0D7
:10BDBC001CFFBDE8F0411AF09DBABDE8F0811548B2
:10BDCC00017819B9144909780029EDD00221B8F18C
:10BDDC00010F297004D10078832808BF15F084FE68
:10BDEC002046BDE8F04120F000BF00BF0C01002050
:10BDFC00236E0020266E0020C12600202525002061
:10BE0C00246E0020F46D0020256E00202F6E002083
:10BE1C00306E00201B6E00201E6E00202DE9F04FAE
:10BE2C0089B08246129803F0F00403F00F0B00283F
:10BE3C0018BF01200392103C0025B4FA84F4640965
:10BE4C002040D4880290107A92886FF39F2400F0DF
:10BE5C003F0024036FF39F2244EA0060544C1044CB
:10BE6C0000905248007804AEC2B2ABB2934280F05C
:10BE7C009580A27801355FFA8AF7974273D08AB21F
:10BE8C000195172A6DD3A1F10709384632461FFADE
:10BE9C0089F421460FF018FE9DF81B8008F0030072
:10BEAC00022826D1BBF1030F00F27D800398007AA3
:10BEBC00DFE80BF0140205109DF8181007E09DF850
:10BECC001810884215D10398BDF81610C088884206
:10BEDC0004D00EE00498009981420AD102980028FF
:10BEEC0054D01298002183688289304616F0E7FE00
:10BEFC0060B15FEA48701CD5BDF81E0084421CD9A5
:10BF0C00A9EB000188B21728BDD228E012988088CE
:10BF1C00E0B3129BDA8819689B681A440B78157881
:10BF2C009D42E6D1013802F1010201F10101F5D186
:10BF3C002CE01F4C0120607104E03846214617F0BC
:10BF4C0065F81B4C00200025F7F7E8F91748E17855
:10BF5C0000780131B1FBF0F202FB101A03E0134838
:10BF6C000078134C019D5FFA8AF1C2B251FA80F14C
:10BF7C00013991FBF2F303FB121A5FFA8AF14900C3
:10BF8C0051FA8AF104EB8101898B6DE7039D96E8E8
:10BF9C001F001FC5002009B0BDE8F08F03990020D9
:10BFAC0088810A20F7E70420F5E700BF026E002025
:10BFBC00006600202DE9F04F87B00546087A0C4644
:10BFCC0040F0020103291ED10026EDB1FF2D1BD03C
:10BFDC00984617460AB9032815D003A821460A2209
:10BFEC0020F016F98DF8167014F010FA204616F0A1
:10BFFC006DFB8146207A4FF6FE71B0F1010A18BF35
:10C00C00BA46894504D10026304607B0BDE8F08F0A
:10C01C000138DDF840B0494FB0FA80F04409464889
:10C02C0001780020814240D03A78AA4208D17A782F
:10C03C00A24205D17A88914502D13A79924502D033
:10C04C000E370130EEE787B33D495FFA80FA4FF0C7
:10C05C0000093E4609880191B8F1000F65D0BBF884
:10C06C000040304621461FF067F8C8B930462146DB
:10C07C001EF03CF898B1019A022051463B461CF048
:10C08C007FFF3048BBF800100268ADF818101AB1E9
:10C09C0003A89047BBF8001020F0A7F900E0002699
:10C0AC000BF1020BA8F10108D6E70DF10B001CF007
:10C0BC00DBFD0646B8B32448224F86F804A0A6F848
:10C0CC000290747035704FF000090DF10C0A5C464B
:10C0DC000078404538BF8046C346BBF1000F0DD0F9
:10C0EC003A682188ADF8181012B150469047218853
:10C0FC0020F07BF90234ABF1010BEEE71099B01D87
:10C10C004FEA480286F8058020F082F89DF80B1063
:10C11C000A4AC1EBC10002EB400309480288022025
:10C12C001CF02EFF01E04FF00009B9F1010F08BF20
:10C13C0017F034F968E700BF7AF002003A66002085
:10C14C00D2E70200682600206AF002002DE9F04FC9
:10C15C008BB0D0F814A0044600260DF110090DF197
:10C16C000E080027BAF80000ADF80E009AF802008D
:10C17C00FDB2854211D22068227943468188007D28
:10C18C00C2F3C002CDF8009014F080FB28B1BDF8CA
:10C19C000E00013601370130E6E7E07A15282FD082
:10C1AC000C2840F09B80680050FA87F0023020F099
:10C1BC0056FE002800F09280804638064FF00109A8
:10C1CC0061D0BAF8000008F1020B0DF1200A0DF154
:10C1DC001E05002EADF81E0040D0206822792B469B
:10C1EC001FF0FEFFD0B3BDF82400013E2BF8030B6B
:10C1FC009DF826000BF8010CBDF81E000130E8E795
:10C20C00A800023020F02BFE002867D081463806AB
:10C21C004FF001054CD0BAF8000000250DF1200BB1
:10C22C000DF11E08AE42ADF81E0021D02068227917
:10C23C0043461FF0DDFFD8B1BDF8241009EB850093
:10C24C009DF82720013541809DF82610017102F0E0
:10C25C0007014171BDF81E000130E3E72068227927
:10C26C000DF11E031FF0BCFFB0FA80F040090BE08B
:10C27C00206822790DF11E031FF0BAFFB0FA80F08E
:10C28C000125400915E0012088F8017088F80000AC
:10C29C0021682379A47A8A88087D29EAD303063198
:10C2AC000294CDE9003943460FF068FF404613E095
:10C2BC00012089F8017089F8000021682379A47A9B
:10C2CC008A88087D25EAD30306310294CDE900352E
:10C2DC004B4610F055FB484620F06BFC01200BB090
:10C2EC00BDE8F08FB0B560480021604C016094F857
:10C2FC003A01032812D002282ED0012840F0AF803A
:10C30C0094F8400111F07CFC002084F8400159485D
:10C31C00817B0220002908BF06209EE0544801685A
:10C32C00B1F5C060C4F82C01B8BFC1F5C060D4F839
:10C33C001011002900D5494288422ADDD4F8140195
:10C34C001DF048FDD4F818011DF056FDD4F8280155
:10C35C001DF076FD01201DE0454805681FF070FFBB
:10C36C00C4F814011FF074FFC4F818011FF078FF13
:10C37C00B5F5C061C4F82801C4F8101109D094F8BF
:10C38C0030215AB1D4F81401D4F82021D4F82C114E
:10C39C000AE0002084F8300106205EE0C4F8240195
:10C3AC00D4E94502C4F82C110223C4F81C0100295D
:10C3BC0048BF6FF0010301EB41011944042391FBC9
:10C3CC00F3F111440029C4F820110FDD1F2931D3DA
:10C3DC00D4F824212AB33E28A8BF3E2001302929B5
:10C3EC0028BF2921C4F81C010B3909E0D4F82421F9
:10C3FC00032A09D111F1140FD8BF6FF013011531B5
:10C40C00C4F82011002113E00128D8BF0120013805
:10C41C0011F10A0FD8BF6FF00901C4F81C010B31E0
:10C42C0003E0332928BF33211539C4F82011032127
:10C43C00C4F824111DF0CEFC01201DF0EFFCD4F843
:10C44C0020011DF0D9FCD4F824011DF0F9FCA5F253
:10C45C00FF510420032938BF0620C4F83C01BDE875
:10C46C00B04006F039B800BF3C500C40501A0020C8
:10C47C0008400C40FCED02002DE9F84F584BDD1D37
:10C48C00584B93F800B000235B4505D215F8054CCA
:10C49C002CB108350133F7E74FF000099DE04FF060
:10C4AC0000095B4500F099804F4B0092504A4FF0C9
:10C4BC00000805F8019C1E1D4C4BB2F816A04FF657
:10C4CC00FE721F78012307B336F8044C8C4218BF58
:10C4DC00544503D12436013F5B00F4E73478042C37
:10C4EC0003D0012C06D0002CF4D109F1010905F878
:10C4FC00019CEFE702F1010CB0F80AE01FFA8CF492
:10C50C00A64508BF48EA0308E4E73B4CDFF8E0E047
:10C51C00384B2678BEF824700A33B6B133F80A4C7F
:10C52C008C4218BF944202D11C33013EF5E71C88A3
:10C53C00BC42F9D1DC79002CF6D01C7A002CF3D05B
:10C54C0009F1010905F8019CEEE72C495FFA89F322
:10C55C0009788B4284BF05F8011C8946009A5FEA72
:10C56C00096102D0817C012901D1002102E09EF8F1
:10C57C000210013105F8031C9EF801109EF80730DB
:10C58C00B8F1000F05F8022C05F8041C8189C07C59
:10C59C0005F8053C25F8071C287011D0184D194BCF
:10C5AC00BBF1000F0CD01E78284619462EB14B1C3F
:10C5BC00051DABF1010B9642F2D1C0F800800A7058
:10C5CC00114C4021207819F06BFB20B920784021C8
:10C5DC00642220F037FB4FF001094846BDE8F88F84
:10C5EC007A5A002069F00200B83E00207EF002006A
:10C5FC00C05E0020E44500206CF002006FF00200E9
:10C60C00485E0020B8690020036E00202DE9F04F31
:10C61C008FB0FF2806D15E485E49007809788842C1
:10C62C0080F0B3805C4900EB800001EB8004002CAF
:10C63C0000F0AB80E0884FF6FF71884200F0A580D7
:10C64C00254615F80C0F002800F09F80002122468B
:10C65C00C0EBC000ADF830108DF838104F490130E8
:10C66C00898CADF83A1012F8011F09928DF8391027
:10C67C0020F083FB82462878800020F07EFB064663
:10C68C00BAF1000F18BF002E75D02878CDF814A081
:10C69C0004F11009FF234FF0000BCDE906660AF8F0
:10C6AC00010BA01C4FF6FF740890287883454DD2DF
:10C6BC00CBEBCB0000212AF800405044064607463D
:10C6CC0046F8031F07F8023FD9F80080CAB2934519
:10C6DC0008D3B8F1000F36D0934588BFD8F8048042
:10C6EC000131F3E7B8F1000F2DD0D8F800100A880B
:10C6FC00028008980188099800780AAB0CF03EFF7C
:10C70C0001281FD107989DF82A40042230600B9E07
:10C71C003C7031461FF07CFD079020461DF0AAF9B5
:10C72C0070B1D8F800000021C0F802102046D8F8EB
:10C73C0000701FF0F9F80246B81C31461FF068FD76
:10C74C004FF6FF74FF230BF1010BAEE7089804883A
:10C75C000998067820F0D8F800210122CDE90021B3
:10C76C00CDE902010CA9DDF814A03046224653464F
:10C77C000AF0EEFA069EBAF1000F02D0504620F0F5
:10C78C00FAFA16B1304620F0F6FA0FB0BDE8F08F89
:10C79C000F6E00200E6E0020A05F0020C05E0020F7
:10C7AC002DE9F04F87B05C48002101705B480068B0
:10C7BC0008B11EF0FDF85A4D00242D689DB1686833
:10C7CC0000781FF061FB0028F7D0017C0029F4D021
:10C7DC00406907300029F0D010F80C2B0139C2F356
:10C7EC0080021444F6E7E0B21BF08CFD10B34E4D02
:10C7FC004A4F162128783A684143562020F042F8D7
:10C80C00092879D00A280ED01EF0D2F8562020F034
:10C81C00C8F94FF01608B0FBF8F6F4B220461BF03E
:10C82C0071FD012860D100F04FFF1EF0C1F807B078
:10C83C00BDE8F08F3B48DFF8E8A000F1040BDAF814
:10C84C0000A0BAF1000FD2D0DAF8040000781FF083
:10C85C001BFB0028F3D08146007C0028EFD04FF062
:10C86C0000088045EBD2D9F8141008EB480001EB16
:10C87C008003DA79520729D5DAF804C01D4631F85D
:10C88C0020105C4635F8042F9CF8000026685EB139
:10C89C0034682778874205D1A788974202D16788E8
:10C8AC00B94218D0341DF1E70020069019884FF6D4
:10C8BC00FF732A889CF800000A25009306ACCDE98A
:10C8CC0002530A23019404940BF0F6FE99F810001D
:10C8DC0008F10108C5E7E38825890A340494CDE9F9
:10C8EC000054CDE90235EFE73B6804FB08F2562013
:10C8FC0000211FF0ABFA2E700A4D6868002892D008
:10C90C00D0E90041696020F036FA287801382870A7
:10C91C00204620F030FAF0E70B6E0020646D00200A
:10C92C007C6D0020046D00200C6E00202DE9F84F6A
:10C93C000DF076F95E480024002690F800A05445CE
:10C94C0010D2E0B21CF0EEFD50B1017941F00401BF
:10C95C00042905D1807A1EF0DBF8002818BF0136B7
:10C96C000134ECE700241CF0DFFA05460027E0B2A6
:10C97C0085420AD91BF05EF828B1807C1EF0C8F8FD
:10C98C00002818BF01370134F1E707EB06085FEA0E
:10C99C00086032D04FF47F7000EA8809484620F0D6
:10C9AC00ECF950B34946FF2204461FF0B3FA0027B6
:10C9BC005FFA86F94FF0000B574529D25FFA8BF0DE
:10C9CC00484525D2F8B21CF0ADFDA0B10646007961
:10C9DC0040F0040004280ED1B07A1EF099F850B142
:10C9EC000146727A30885FFA88F30093234615F07B
:10C9FC00F5FC0BF1010B0137DEE700244FF00008CA
:10CA0C002C48007BE0B11FF043FCC0F1540018E04F
:10CA1C0000275FFA88F9F8B28542F1D91BF00AF8C1
:10CA2C0060B10646807C1EF073F838B10146727C0A
:10CA3C0030882346CDF8009015F0D0FC0137EAE79A
:10CA4C006220C1B20322A2462546B1FBF2F9B9F12C
:10CA5C001F0F28BF4FF01F09C0B25FFA88F1444680
:10CA6C00002818BF0120420102F1400749452A461F
:10CA7C0084BF47014C46E0B2394612F0A0FD0022BB
:10CA8C00064617F0400008BF621E40EA0601A8EBFC
:10CA9C0002080020D2B2002905EB8205DCD0BAF1E5
:10CAAC00000F02D0504620F066F93046BDE8F88FF2
:10CABC007EF00200C05E00202DE9F04706680446B7
:10CACC00307B02280ED1F07F6568D6E904A7914629
:10CADC00884668B1B16853481FF0AEFF28B16FF0BB
:10CAEC00010750E06FF006074DE0012086F82200A8
:10CAFC0000204E492246B0614B48C6F8008086F8AB
:10CB0C001D901EF04CFF297827201EF07FF950460F
:10CB1C003946062203F04AFA48B196F8220070B35F
:10CB2C00404820F03AF9002086F8220027E0404DDA
:10CB3C00404FD5F8800320F00200C5F88003307F09
:10CB4C00042804D157F84C0C41692720884702204F
:10CB5C00C5F8FC023868416806208847B0B140200F
:10CB6C0028608020286096F8220028B12D4820F0FB
:10CB7C0014F9002086F822000020C5F8FC024FF0C2
:10CB8C00FF30B061B7693846BDE8F0870220BA467D
:10CB9C001BF050FA0027B9F1020F0AD0B9F1040FBB
:10CBAC004FF0000006D0B9F1060018BF012080003C
:10CBBC0000E00020C5F84C010123D8F80C10D8E98E
:10CBCC000102C5F85011C5F8547186F82030DAF816
:10CBDC0000301D690B46A8472568287F02281AD00B
:10CBEC000428D0D1DAF80000816914488847B0F1E4
:10CBFC00FF3FDCBF4FF0FF30A8610020AF6985F824
:10CC0C002000697F0339022928BF85F821002046BE
:10CC1C0019F05CFCB7E708484FF0FF311FF00CFF30
:10CC2C00AF69B0E7786200202C6A0020BDF10100EA
:10CC3C0004440240FC010010C86200200100008086
:10CC4C002DE9FF47D0E901590E4604461FF0B8FC08
:10CC5C0095F8FD1021B97169102901D8032906D85E
:10CC6C001FF0C3FF0024204604B0BDE8F087012765
:10CC7C0085F8FD701FF0B9FF00204C4A85F8FC00C8
:10CC8C00C5E93000C5F8C80085F8FE003069C5F864
:10CC9C00E4007069C5F8E800307B85F8F9000028DD
:10CCAC00317885F8F8107168C5F8EC10B9F80E10E9
:10CCBC00A5F8F610317E52F8211085F8FA1008BF4D
:10CCCC001027C5F8F07099F80C000BF035F92046D8
:10CCDC0016F0E0FC99F83B0085F8FB00D4E90187DD
:10CCEC0098F8F91097F8380001291AD1F96ADFF889
:10CCFC00C0A0D047B96A97F83900D047396B97F87C
:10CD0C003A00D047796B98F8FB00D04798F8FB00B5
:10CD1C0028491EF05FF898F8FB0021461EF038FFFA
:10CD2C000FE0B96ADFF888A0D047F96A97F83900A4
:10CD3C00D047396B97F83A00D047796B98F8FB00DD
:10CD4C00D047E84640461FF0EBF999F805001A4A1F
:10CD5C004346CDE90040284699F8041018F0B0FE7F
:10CD6C0040461FF0A5FAD9F8080014494246009431
:10CD7C00029005F130001AF0B9FB12F047FE104A90
:10CD8C00C5F8CC0005F11C00042123461DF06AF8FF
:10CD9C0095F8F80008B1B06805E005F16C000021C9
:10CDAC001DF066FD0748C5F8BC005CE788ED020085
:10CDBC00FDAD020079040200E1B50000C391020050
:10CDCC00C1C8020097CB020070B5604D0446A8683C
:10CDDC004169497F002973D0D0F8D420B4F84210AF
:10CDEC00D28C91426CD1D0F86C1304F12800884796
:10CDFC00002865D0A868002241694A77D0F8D41081
:10CE0C0091F8291021B1E868816A02208847A86846
:10CE1C00006F90F82B0018B1E868816A01208847F0
:10CE2C00207CC00608D5E868816A10208847A8686D
:10CE3C00D0F8281380208847E868C16B20208847E9
:10CE4C00A868D0F8FC14C068103088476268A868DD
:10CE5C0013785278416902F00F064E76C2F3001136
:10CE6C004269917603F00F01426991771909D0F864
:10CE7C00D42082F82C10D0F8D410426991F84F309D
:10CE8C00927F0F2B05D09A4203D26668F67806B9CA
:10CE9C001A464A730022C16881F83020D0F8D410A9
:10CEAC00497B0F290DD14169C97E022908D1D0F8DF
:10CEBC0064018047A868D0F86C01BDE87040004759
:10CECC0070BDD0F80C2520469047A9684869C07EF3
:10CEDC00022814D1C868D1F8FC148847AA684FF40A
:10CEEC007076D2F8D430D2E90301D2F8F0245B7B0F
:10CEFC0031F8131006FA03F3591A9047A968D1F8C0
:10CF0C00D400D1F8B431228990F82C100220984723
:10CF1C00A968D1F8D400427B90F82C0090420FD035
:10CF2C004869D1F8FC148847A8684169D0F87C019D
:10CF3C008860A868D0F8F024406941699047A968D6
:10CF4C00D1F828131020BDE8704008470C010020D0
:10CF5C002DE9F04F89B00546C07A022840F08D804B
:10CF6C006C69207800EB400001301FF078FF00283E
:10CF7C0000F08380261D00F101084FF0000A0DF12E
:10CF8C00180B4FF0000904902078824580F08680C1
:10CF9C00286837465B4637F8032D8188007D18F0EA
:10CFAC00F6FCC0B328799DF81F10C0F3C000B0EB9D
:10CFBC00D11F64D116F8010C9DF81E1088422CD19B
:10CFCC000898296858B38888032803D136F8030CCD
:10CFDC0000283ED0087D06315A463B4616F06EFDC1
:10CFEC0007462868808808BB36F8030C41F23731B5
:10CFFC0088421BD131680DF1150001221FF008F990
:10D00C009DF915001EF044F8102001210DF11502B8
:10D01C001FF03EFC0AE0862709E08D2707E0087D1B
:10D02C00336806315A4619F017FA07466FB15FFAA2
:10D03C0089F036F8031C400050FA89F009F1010917
:10D04C0008F800704044A0F8011007360AF1010AF4
:10D05C009AE731680DF1160002221FF0D9F8286802
:10D06C00007D17F075FD17F08DF82868017DBDF86F
:10D07C00160014F031FC0027B3E7002528E05FFA16
:10D08C0089F08621400050FA89F009F1010908F86D
:10D09C00001036F8031C4044A0F80110049E5FEA0F
:10D0AC00096086F8009004BF0120308029682B7934
:10D0BC00AC7A01258A88087D25EAD30306310294CF
:10D0CC00CDE9003533460EF0D5FF30461FF071FD2B
:10D0DC00284609B0BDE8F08F2DE9F04F85B0044625
:10D0EC00C078C1070ED04FF0FF316175A4F8131052
:10D0FC00217902290ED029B900F0DF004FF0040B82
:10D10C00E07009E001200490049800F0010005B0E3
:10D11C00BDE8F08F4FF0080B4C484D4E04F108055C
:10D12C004FF00008CDE9015B90F8009001200490CD
:10D13C000020CA460390C14565D056F828005FFA16
:10D14C0088F7B8B1217902798A4213D1083029467F
:10D15C005A461DF0BDFE68B1A07878B156F828008B
:10D16C000179C1B1E178890644D401204FF0000B5C
:10D17C00039014E0BA4608F10108DCE72079022894
:10D18C000BD1E078800608D556F82800217C007C6D
:10D19C008142F0D101E0012003904FF0010B0420FB
:10D1AC001CF0E2FDF8B107460620294D388055F8F1
:10D1BC002800817CF9701DF087FD039E394616F01E
:10D1CC00010018BF204645F828004FF0040018BF96
:10D1DC000120B8701F48007814F0C6F9049986F045
:10D1EC00010001400491BBF1000FDDE9015B184E19
:10D1FC00C1D089E7007C217C012203928142BAD103
:10D20C004FF0000BCBE70398C0077FF47DAF0420F1
:10D21C001CF0AAFD00283FF477AF014606200880D9
:10D22C00A07CC870CA4507D2A07838B1002046F857
:10D23C002A400490022002E0002000E004208870C4
:10D24C000448007814F090F95EE700BF67F0020024
:10D25C00946D0020136E00202DE9FE4F07460078D8
:10D26C009B468A46029200F00C000C2802D1B8882A
:10D27C00FE2119E056480568B878FF2808D01FF041
:10D28C0037F840B1064600781EF052FA054603E026
:10D29C002DB16E6800E00026FE20019016E0FE2005
:10D2AC0000250026019011E01AF0BCF9FE28014679
:10D2BC00019000F0868001981FF01AF8002800F009
:10D2CC008080064600781EF033FA0546002E78D092
:10D2DC00AA684AB13178022090474FF6FE7440B1EB
:10D2EC0004881FF048FD04E0B0684FF6FE7400B1EE
:10D2FC00448839893078A1420BD010B909B9002083
:10D30C0007E000284AD04FF6FE72013292B29142E9
:10D31C0044D197F80290B870387DD7F8108030302F
:10D32C00C0B21CF021FDB8B304461A20514620703F
:10D33C007868C4F80200A01D1DF0C6FEBBF8010001
:10D34C00A4F817000C983A7D397B84F820000E98CD
:10D35C006175A284E0610D986076F878E07330789E
:10D36C0020759BF80000A075788BA0857889608269
:10D37C00029820820F9884F82E0032B104F130000C
:10D38C004146A0621EF044FF01E00020A0627068DC
:10D39C002146007814F0E8F887F80290387800F00D
:10D3AC000C000C280FD0B8780026FF287FF48EAF25
:10D3BC0028680025002600283FF488AF46680546FB
:10D3CC0084E7BDE8FE8F0199B888C9B26CE700BF4D
:10D3DC007C6D00202DE9F04F87B01D4691468846A4
:10D3EC0007461EF085FF002800F096800646109C2C
:10D3FC00384649461EF0C4FF8346400607D45348BE
:10D40C00406820B1407E012808BF4BF0400B05A8B6
:10D41C00002108221EF019FE002C18BF01249DF8D3
:10D42C00140000F0FC0020448DF81400B0680028B3
:10D43C0070D03846494622462B4617F0CAFD0028C4
:10D44C0068D011AFDDE914349DF8141085CF1FB1ED
:10D45C0041F00401ADF8187000288DF81B508DF8C0
:10D46C001A3018BF0120C3001033002A08BFC300B4
:10D47C0001F0E70018448DF8140048074FF0050040
:10D48C0058BF032020441FFA80FA50461FF0E7FCD7
:10D49C00002843D005469DF814002346DDE91614F8
:10D4AC0000F0030028709DF8142002F004021044D0
:10D4BC0028709DF8142002F00802104428709DF882
:10D4CC00142002F010020244284600F8012B9DF8AB
:10D4DC001420520706D59DF8180068709DF81900A5
:10D4EC00A870E81C9DF81A2000F8022B9DF81B2050
:10D4FC0000F8012C1A461EF053FF144F78787CB1BB
:10D50C000390404631464A4653468DE8A0080AF03F
:10D51C0023FF0EE0012415E0022413E0102411E097
:10D52C000390404631464A4653468DE8A008FCF726
:10D53C00A7FF044678780F281CBF0F207870284668
:10D54C001FF037FB204607B0BDE8F08FF824002011
:10D55C00F8B50446007D50B1594994F91700C968D3
:10D56C00D1F880108847013004BFE820F8BD544E34
:10D57C00E27BB568D5F80011E86B09780AB1807ABE
:10D58C0000E0C07A81429CBFF120F8BD236A94F878
:10D59C00352094F83410208DD5F88C52A78B009739
:10D5AC00A84700285DD00546002028806868616A7D
:10D5BC00228D1FF057FC04F12C0005F184010CC8DE
:10D5CC000CC1028880788870B0680A802146D0F837
:10D5DC00442505F1900090476089B268A5F89A003F
:10D5EC00207B85F89C00607B85F89D00D4F80E00AC
:10D5FC00D4F81210D2F848259047A5F89E00A07DCB
:10D60C0085F8A000E07D85F8A10094F8380085F835
:10D61C006C00A28BA5F8A8202AB3A169D5F8A400A8
:10D62C001FF020FC1EF019FFB5F8A800E8B1D5F8E2
:10D63C00A400D0B16868411E6960F82100F8011C93
:10D64C006868411E6960002100F8011CB5F8A8004B
:10D65C006968091A6960A96529890844023028811A
:10D66C0003E01A20F8BD1EF0F8FEB5F89E10C805B0
:10D67C001DD594F83720E8202AB111F0040208BF18
:10D68C0011F0010100D0F8BDB168486ED1F8FC145E
:10D69C00884794F837004FF47A71B26848430949C7
:10D6AC000978B0FBF1F1506ED2F8F4249047B068D1
:10D6BC002946D0F89400007813F056FF0020F8BDEE
:10D6CC000C0100201F6E00202DE9FE4FDFF8609149
:10D6DC00D9F80000002800F0A8804FF016084FF091
:10D6EC00000B54480478A34580F09F80D9F800A023
:10D6FC000BFB08A045880BFB08F01AF800602946C4
:10D70C00304619F0DDFFFF2824D1BAF1000F00F0EC
:10D71C0089800AF1080300224FF6FF704FF6FF7C58
:10D72C004FF6FF77E4B313F8081CB1420FD133F86E
:10D73C00061CA9420BD133F8021C81423CBF674640
:10D74C00084619880132B9423CBF8C460F46163345
:10D75C00013CE7E707460A201FF00FFB002864D0C6
:10D76C0004461DF0F1FF1EF063FE218000F10E0156
:10D77C00A01D1EF04DFD22883046294601AB0BF052
:10D78C00FDFE012804D10299A01C04221EF040FDCC
:10D79C00294907EB870001EB800021460C303DE066
:10D7AC0011063FD02549097804293ED8224F234C35
:10D7BC0001EB810201310023217007EB820107F894
:10D7CC00223088800A200B610B81A1F806C04D80A5
:10D7DC004E700B731FF0D1FA38B307461DF0B4FF2F
:10D7EC001EF026FE398000F10E01B81D1EF010FD52
:10D7FC003A883046294601AB0BF0C0FE012804D113
:10D80C000299B81C04221EF003FD0C480A4900784A
:10D81C0000EB800001EB80003946083817F07AFEE7
:10D82C00012802D00BF1010B5BE7BDE8FE8F00BFB6
:10D83C00646D00200C6E0020A05F00200E6E002096
:10D84C007CB5584D584E4CF6C0722B78347883F01A
:10D85C00010384F00204234308BF1040534C0029F9
:10D86C005249898C0CBF21EA00000843A08401B204
:10D87C00B1F1FF3F08DC01200DF103018DF803002D
:10D88C00522017F021F9A08C810400F1828081B222
:10D89C000A042AD401047CD04FF0FF310191317875
:10D8AC00022976D12978002973D1216823460131C8
:10D8BC0001A908BF0B46C207224608BF0B461D68CC
:10D8CC0052F8046FB54298BF1A46050758BF1A465E
:10D8DC00C30606D52546136855F8086FB34288BFB2
:10D8EC002A4683061ED4134623E0480451D504F17E
:10D8FC001000226A016812B11268914211D02C4DAD
:10D90C0020620129287803D1012112F0BFFC7CBDD3
:10D91C00012113F063F9216A28780A6801211FF0AC
:10D92C0091F97CBD2346156853F80C6FB54298BF2E
:10D93C001346420401D41A4606E022461D6852F8EA
:10D94C00106FB54298BF1A46C30401D4134606E0C3
:10D95C002346156853F8146FB54298BF13468207D7
:10D96C0001D41A4606E022461D6852F8186FB542DB
:10D97C0098BF1A46400701D4104606E020461368AB
:10D98C0050F81C5FAB4298BF1046884218BF002865
:10D99C00AFD10020012120620548007813F01EF958
:10D9AC007CBD00BFF32600201C25002060680020F1
:10D9BC00036E00202DE9F047814608688A469046A0
:10D9CC00D9E90045476806894E48E1681FF034F8EC
:10D9DC0018B16FF00100BDE8F08700204B494A46B2
:10D9EC00C4F814A084F809806060A07046481DF04B
:10D9FC00D6FF297827201DF009FA38463146062231
:10DA0C0002F0D4FA90B9424F57F84C0C41692720D8
:10DA1C008847404E0220C6F8FC0238684168062050
:10DA2C00884750B1402030608020306035481FF06E
:10DA3C00B4F94FF0FF30BDE8F08702201AF0FAFA83
:10DA4C003A68DAF810009AF82010D26990473A68D0
:10DA5C009AF820009AF821101368A8F10102B2FA82
:10DA6C0082F252099847DAE90610C6F850010020F4
:10DA7C00C6F85401C6F8581159B13A68DAF80400DE
:10DA8C00002315690022A8473868816922480130B3
:10DA9C008847207A042804D057F84C0C01692720B9
:10DAAC0088473B68DAF81C10DAE902021C690B465D
:10DABC00A047D9F8004001206070207A022815D0C8
:10DACC0004281BD13868144D816928468847B0F169
:10DADC00FF3FDCBF4FF0FF30606000206070A81C7F
:10DAEC00C6F88403484610F0CDFA04E00B484FF01A
:10DAFC00FF311EF0A1FF6068BDE8F0870020BDE893
:10DB0C00F08700BF786200202C6A002031F60100FB
:10DB1C00FC0100100444024001000080C862002097
:10DB2C002DE9FF4715460F46814639B138461FF09F
:10DB3C0050F818B10446A5F1010A4EE04A48A0F18C
:10DB4C0024014A480678701C01386DD001F1240478
:10DB5C0091F82810FF292146F6D1002C64D0E81E3C
:10DB6C00C0B201280DD84248B0F80080B8F1000FBF
:10DB7C0007D00320042118F0FDFCA6EB080181421C
:10DB8C006FDDA5F1010A5FFA8AF001280DD839483A
:10DB9C00B0F80080B8F1000F07D00120022118F076
:10DBAC00E9FCA6EB080181425BDD0120E846394621
:10DBBC00ADF802908DF8000008F104001EF000FC96
:10DBCC00404605F069FF0020A071BDF80C00608094
:10DBDC002948818C48461AF077FE4AF6012100202C
:10DBEC002571A4F80090A4F8091080212082E0602F
:10DBFC00E072E07184F8211020490978013149085C
:10DC0C0021725FFA8AF1042938BF012080000129B2
:10DC1C0060710BD81A48007858B11A4951F8200095
:10DC2C00C0EB0010800006E0002409E06FF001005A
:10DC3C0004E014480068012184F82010A061E06120
:10DC4C0000200421002518F095FC08490978884229
:10DC5C0024BF0D48057008F05BFF204604B0BDE8FA
:10DC6C00F0870024F9E700BFB83E00207EF00200E8
:10DC7C004EF0020050F00200C05E002068F002007E
:10DC8C00E6260020C8EA0200A82600202DE9F04173
:10DC9C008CB0534F05463878022804D14F48007891
:10DCAC00002800F09780DFF83C8198F826000828BF
:10DCBC0002D0042840F08E8009AC284621461DF085
:10DCCC00A1F91EF06AFF0234BDF8240021460AF0C7
:10DCDC00F5FD01287ED002AE30461EF01AFF30460C
:10DCEC0021461CF0CFFB68B1BDF824601EF074FC1B
:10DCFC00864207D0BDF82400414621F81A0F4B206C
:10DD0C0016F0E2FEAD8A1EF079FC854214D0204656
:10DD1C001EF05FFF30B100790138012802D820468F
:10DD2C0013F0C2FA3148016831B12F48007801284C
:10DD3C0002D1BDF824008847BDF82400002100263C
:10DD4C001BF021FFB8F82410BDF824001AF0BCFD1C
:10DD5C00BDF824008DF81460ADF8160005AD28460A
:10DD6C000DF042FB70B1CDE902662E1D02A83146C2
:10DD7C001CF088FB30B1304621461EF021FB05A873
:10DD8C0005F08AFE281D21461EF01AFB28460FF0CE
:10DD9C0089FE50B1BDF82400BDF81610814204D0A4
:10DDAC00ADF8160005A805F077FE3878012811D8D3
:10DDBC000F4D4FF0FF30CDE90000286850B1694697
:10DDCC00204608221DF084F820B92A68BDF82410DA
:10DDDC00204690470CB0BDE8F08100BFF326002030
:10DDEC001C250020C05E0020DA26002050220020D6
:10DDFC00B8250020F8B5514F514E524D3888316836
:10DE0C00EC880844224600F10801A868806D1FF0D8
:10DE1C0029F8A96838884C4B8A6D204438802244F4
:10DE2C008A65326881B20832565C811C398089B2AD
:10DE3C00515C1970C11C0730398089B25158388037
:10DE4C006846009104211BF0A1F900901DF0ACF97B
:10DE5C00A968C86300981CF00BFEA968A1F84000E3
:10DE6C00EA2019F0AFFC3948426812B1A8680121C8
:10DE7C00904737480221374C0170E06840690078C0
:10DE8C0030B1A87B800917F039FE08B10120A870C9
:10DE9C00A878A96800280A7C70B218BF42F0040266
:10DEAC000A74002100271EF0B0FF0146A86880F814
:10DEBC00461000F17401B0F85C2080F8486080F8DE
:10DECC00477081650189511A426811444160417B58
:10DEDC00890709D5A168D1F808138847A868416E4D
:10DEEC0011B1B0F86810F1B190F8601049B1A168A7
:10DEFC00D1F80C138847A868C16C11B1B0F8501058
:10DF0C0089B1A168D1F8B820137823B1926C12B101
:10DF1C009047A868A168D1F8581288470020A860DB
:10DF2C001DF0A4F9F8BDA068D0F8541205F1080052
:10DF3C0088470020A86010F00DFBF8BDF26D0020A2
:10DF4C00246D0020FC230020206E0020BCEB02007E
:10DF5C001B6E00200C0100202DE9F04F89B0064605
:10DF6C005048DFF844B1CDE904120125006806AF32
:10DF7C00002800F094800321D0F804808DF8201044
:10DF8C001EB1049839461AF0FDFB4FF0000A4FF011
:10DF9C000009D8F80800017B8A451CD200699BF85F
:10DFAC000040DBF808309BF8072030F81A1098F87E
:10DFBC000000CDE9007401240296039414F03CF99E
:10DFCC00054610B1B22D03D108E04FF001093EB166
:10DFDC000AF1010ADDE7B22D03D1B225314A2DE059
:10DFEC0000254FF0000A2EB9B9F1000F02D02D4ACE
:10DFFC0006AF26E00024D8F80800C1798C421BD269
:10E00C008068DBF810309BF800509BF80C2030F83F
:10E01C00141098F8000006AFCDE9026ACDE900753E
:10E02C0014F00AF9054610B1B22D03D104E05EB12B
:10E03C004FF001090134DEE71A4A06AFB9F1010FBE
:10E04C0000D126B1FF2003E0164A002506AF802040
:10E05C000599B22D096808730FD014480078FF2871
:10E06C001DD110680068002810603FF481AF416832
:10E07C0009780139F029F5D27AE70D480D4C0021C9
:10E08C0001702078402112F0A9FD1CF01DF82078B9
:10E09C004FF4804112F0A2FD0C201EF039F909B0AA
:10E0AC00BDE8F08F60200020846B0020AE2600209D
:10E0BC00542000200A6E00202DE9FC4FD0F8C090AF
:10E0CC00D0F8D0C0D0F8E820D9F80030CB46E646DE
:10E0DC009C450CD3D9F814B0BBF1000F00F0848030
:10E0EC0001234FF0000E8BF81030DBF80030A3EB5F
:10E0FC000E05A2F1080AB5F5806F28BF4FF48065B4
:10E10C00D0F8D82032B101F1200301F12402C0F87B
:10E11C00DC5005E0C0F8D85001F1180301F11C02E5
:10E12C000026BAF1000FC8BF0126DBF804401268C4
:10E13C001F68CDF800E07CB1344B53F82630BB603F
:10E14C0005FA06F30126BAF1000FC8BF02260EFB32
:10E15C0006332344013B05E02D4B53F82630BB60BE
:10E16C0000F1F6033B6043F6F0730191D1F80080A7
:10E17C0003EB0514234008F1080EC7F804E0BC6853
:10E18C001C43BC600024BAF1000FC8BF0124DBF8AB
:10E19C0008709FB16146DFF87CC05CF824608C4647
:10E1AC0005FA04F496600126BAF1000FC8BF0226E6
:10E1BC00009901FB064139444C1E05E0144951F805
:10E1CC00241000F1F40491605460C2F800E09168EE
:10E1DC0019439160CB4504BF05EB0C01C0F8D0107E
:10E1EC0090F8FE10019A09B1BDE8FC8FD8F8241004
:10E1FC0041F00301C8F82410D0F8CC00D2E9041285
:10E20C004068114300688162BDE8FC8F70ED02002C
:10E21C0078ED020080ED02002DE9F04F85B0074645
:10E22C008A465818D7F80880D8F80410884202D9C2
:10E23C006FF003057BE04E4D7C68DDF838904FF0B5
:10E24C00FF319B46164628681EF0F6FB6068B8F84E
:10E25C002010C5E901015FEAC97014D15FEA897029
:10E26C0023D5D8F80C0000287AD0D8F81010002943
:10E27C0076D001228DE80700384651465B4632467F
:10E28C0013F056FB0EE0A068C14300EA0B0211EA42
:10E29C000B0F1CBFD8F808100A4400EA0A013846D4
:10E2AC0006F052FD08B105463DE0D8F800005C468A
:10E2BC003546039600EB0A09ECB3384612F0D0FD54
:10E2CC0078BB38461AF036F858BB02208DF81390FC
:10E2DC008DF810004FEA19208DF812004FEA194002
:10E2EC008DF811002248018938461DF030FE5FFA86
:10E2FC0089F0C0F58076B44238BF264604A80421C4
:10E30C0013F0EEFF68B92846314613F0E9FF40B927
:10E31C001748A41BB144018938461DF021FE354431
:10E32C00CAE74FF0FF35124800681EF036FD28464C
:10E33C0005B0BDE8F08F0E98400701D40025F2E738
:10E34C00D8F80C0060B1D8F8101049B100228DE853
:10E35C000700384651465B46039A13F0E9FAA2E7E8
:10E36C00034800681EF019FD6FF00705DFE700BFDA
:10E37C00C42200202DE9F04F89B08246807E1CF02B
:10E38C00D7FAA0B3DAF81CB0054600270DF118082F
:10E39C0000260BF102049BF80000874215D207EB14
:10E3AC004700BAF80C104346225A287817F0EFFAB7
:10E3BC0048B19DF81E001BF05DFB20B19DF81E00BE
:10E3CC001DF0B2FA06440137E5E7C0EB001001304E
:10E3DC00C0B250FA86F01EF0D0FC049028B115F0B3
:10E3EC0065FE30B104981EF0C6FC10266AE00226C9
:10E3FC0068E004984FF00008002180F800809BF83A
:10E40C0000009AF81A70814246D20BEB0809BAF850
:10E41C000C4005913846B9F8025021462A4617F0AF
:10E42C006BFD0646384621462A4606AB17F0AFFA76
:10E43C008621FF2E18BF002813D1049C08EB8800FE
:10E44C00B9F8022008F1030820442378417099F8A8
:10E45C000110A0F80320013381700599237001315C
:10E46C00CDE79DF81F00400701D48C21E5E7049906
:10E47C0008EB8800162208449DF81E1041711349C0
:10E48C00096816FB021101F10E02C260D1F80610E8
:10E49C00C0F806100021D0E7049C9AF80A00BAF8DC
:10E4AC000C2000260121CDE900110AF10E01CDE965
:10E4BC0002063846234602F055FB20461EF05BFC54
:10E4CC001CF076FA304609B0BDE8F08F646D002080
:10E4DC002DE9F047012816D1DFF830A1DAF8340124
:10E4EC00012813D10220CAF834011AF0CBFA01200A
:10E4FC00012419F0DFFF60B1CAF834411CF038F97F
:10E50C004FF0FF347FE06FF001047CE06FF0040407
:10E51C0079E09AF85A419AF859119AF85801002C56
:10E52C0018BF0124002918BF0234002818BF043476
:10E53C0001201EF0C3F8013818BF01209AF83811D9
:10E54C00B1FA81F1490910EA010902D1002007F062
:10E55C00A3FADAF808002E4D10F0010807D12D4F60
:10E56C00286A8168384688470428F9D00646404610
:10E57C001EF053FAB8F1000F08D1012E04D1286A0D
:10E58C0001214268234890471DF052FE28684169DA
:10E59C00204688479AF8540118B14FF480601EF059
:10E5AC0093F89AF8530118B14FF481601EF08CF86F
:10E5BC0019480121016003200021CAF834011748D1
:10E5CC000160204616F04EF90128FAD1144E30683D
:10E5DC00042019F06FFF044612480125B9F1000F11
:10E5EC000560306802D1012007F056FA1EF018F8C9
:10E5FC00082019F05FFF0443CAF8345118BF4FF0DC
:10E60C00FF341CF0B5F82046BDE8F087501A002006
:10E61C00B801001000400340282008600C2008407E
:10E62C002C2009400C4009407CB54B4EB068016C65
:10E63C00D0F8D420096892F8835019B9D0F84C0559
:10E64C008047B068D0F8B800007800B316F04CFBE7
:10E65C004349424809680068096C884705461DF023
:10E66C00AFFF04463F48017811B93F49097821B3FF
:10E67C003E4902220A700078832808BF13F034FA4E
:10E68C001EF0CBFA1EF092F90420884757E01DF0DB
:10E69C0097FF04463348017811B933490978C9B357
:10E6AC0002223249012D0A7004D10078832808BF58
:10E6BC0013F01AFA1EF0B1FA41E01EF077F90020BF
:10E6CC008847B0680DF10701D0F82824F420904752
:10E6DC009DF90700854223DB254D287800BB1EF0F1
:10E6EC009CFA25480078042803D0B068D0F84C0573
:10E6FC0080471E48042101702878013028701EF0D4
:10E70C0055F909B1032088471C48032101801EF0EC
:10E71C0086FB14E01548832101701EF07EFA0CE094
:10E72C00124883210170002018F068FB1EF075FA66
:10E73C001048F16880780969087017F0DBFDF06803
:10E74C00C068007800B17CBDB0680021D0F85824B6
:10E75C00002090477CBD00BF0C010020C825002084
:10E76C00A46D00201B6E00201E6E0020236E002066
:10E77C00C126002025250020266E0020F46D0020E7
:10E78C002DE9F84F89460188904607460B209A469A
:10E79C0001F00702022A08BF1420002A08BF0F202C
:10E7AC0011F4007118BF043004D1397EE22904BF82
:10E7BC0000217976797E451828461EF050FB0028FA
:10E7CC0059D03946022206461DF0EAFD3888B41CA1
:10E7DC0000F00700022807D080B9391D204604221A
:10E7EC001DF0DEFDB41D09E007F1080120460822EA
:10E7FC001DF0D6FD387C06F10B04B07207F1140144
:10E80C00204604221DF0CCFD387E2071787E60718C
:10E81C0006347A7E52B1F96969B320461DF0C0FD09
:10E82C00F86997F819B01EF0C4F95C4407F120019F
:10E83C00204602221DF0B4FD97F82200A0707878D3
:10E84C00800705D5E01C07F1240104221DF0A8FD6A
:10E85C001B4CF2206072A9F10C002661E573A073C9
:10E86C001848808C60811848007838B102202072DA
:10E87C001648008806E01020BDE8F88F0F202072A3
:10E88C004FF6FD70BAF1000F208003D09AF801000A
:10E89C00800604D4404615F06CFEA08105E004F11E
:10E8AC000C000AF10B011DF059FA094832210068DD
:10E8BC001EF067F907481EF07EFA0020BDE8F88FBD
:10E8CC00986B0020C05E00205B2300205E2300209C
:10E8DC00846D0020386400202DE9F84F494C10213C
:10E8EC00207817F0DDF928B9207810214FF47A72CE
:10E8FC001EF0A8F9444801780139017009065AD074
:10E90C0043484FF000084FF6FE790026041D41489D
:10E91C000578AE421DD22078C0B1FF2816D0013840
:10E92C002070000612D16078032807D134F8041C3B
:10E93C0034F8020C022211F037F8607801281EBF5F
:10E94C00A4F8018024F8029C24F8049C08340136B5
:10E95C00DFE73148DFF8C4A0314C4FF00008002746
:10E96C0090F800B05F4519D007EB87000AEB400523
:10E97C00287A0138287200060ED12046294619F053
:10E98C00C9FD064610B130461AF0A2FA002EF4D199
:10E99C0085F80080A5F802900137E3E72148224969
:10E9AC00007830B10A780AB1013A0A70083101389E
:10E9BC00F7E7BDE8F88F15490022097801700020AF
:10E9CC0005211AF08FFF04460626002C98D020460D
:10E9DC000521002225461AF085FF044628890028C7
:10E9EC00F3D0013828810004EFD16889400702D5A3
:10E9FC00287B19F067FB2868F0216E73407B15F0BB
:10EA0C002DFCE2E7036E00207F6C002077F0020003
:10EA1C005C4B002071F0020070F0020018630020C3
:10EA2C00C545020072F00200046000202DE9FE438F
:10EA3C000C46080426D4E0074CD1A00700F18B80CB
:10EA4C0020074FF000001BD54B4FDFF828814FF00B
:10EA5C00FF3100220123CDE90011694698F800909E
:10EA6C003D7888F8000038704448FE8A0088F882A7
:10EA7C0017F0E8FF84F0080088F80090FE823D70E3
:10EA8C00BDE8FE833848007812F0D6F800285ED036
:10EA9C000546007820B96878A9781EF0A0F8287887
:10EAAC00012803D128460AF09FF92878022803D1BF
:10EABC002846F8F7C1FF2878082803D1284604F027
:10EACC0027F9287805280BD12846FEF705FB0646C2
:10EADC00287806E018F006F984F00100BDE8FE8302
:10EAEC000126042821D1DFF88480D8F80800C0B1B1
:10EAFC0095F8400044301EF040F990B1074695F867
:10EB0C004000294600F1440238461DF081FB0020EC
:10EB1C001749B86038461DF06BFAD8F8081028462B
:10EB2C008847284619F01EFC2878104F062804D177
:10EB3C00396811B1284688472878072803D1F96825
:10EB4C0009B12846884716B128461CF0BDF884F454
:10EB5C000040BDE8FE830548406800B1804784F062
:10EB6C000200BDE8FE8300BF136E0020BC23002012
:10EB7C0004260020006E0020C05E00207E5700207E
:10EB8C00F0B58BB0ADF80A00002001F108070C4677
:10EB9C008DF8080038461CF06AF808B306AE0DF183
:10EBAC000701384632460CF00BFF05464FF6FF7056
:10EBBC0085421FD09DF8070000B39DF8280000285F
:10EBCC004ED0FF280AD0022840D0FD2806D00128BC
:10EBDC0055D13B480078013801283CD939483CE0F4
:10EBEC0002A80CF001FC012802D102A818F060FB6D
:10EBFC00A12062E03348C4F812005DE006F1080081
:10EC0C00394608221DF004FB40F2FF10ADF8280035
:10EC1C001DF0FEFE00F00F0000272946142233469B
:10EC2C008DF82A000420CDE906771AF0A9F92649B7
:10EC3C0005EB450041F8207001EB80002149C0E94B
:10EC4C000177C4F812100121417218E01C480078B9
:10EC5C00013801280CD84FF08170C4F812000EE076
:10EC6C00052060829DF82B0000F07F00A08206E05A
:10EC7C0004F11E0006F1080108221DF0C9FA124A1F
:10EC8C0005EB4501002052F821305D1C42F8215063
:10EC9C00A3610A232074B5FBF3F303EB8303A5EB09
:10ECAC00430353B902EB81000121017207484FF471
:10ECBC008061007811F0EAFA00200BB0F0BD00BFC3
:10ECCC001C25002000000301AC680020046E00200D
:10ECDC002DE9F04192B006462C201EF0C0F8D0B3BE
:10ECEC000446082008222080307C317FE17020749B
:10ECFC0004F1140006F114011DF052FB251D311D09
:10ED0C000C2228461DF04CFB317D307F14F050FC5A
:10ED1C0020B30020A0708DF80400E0788DF8050079
:10ED2C0001AE95E80E00301D0EC0207C6169A26911
:10ED3C00079206918DF8140006F11C0004F11C01D9
:10ED4C0010221DF02DFB3348314600781DF0BFFE1C
:10ED5C0020461DF02EFF12B0BDE8F0810DF14301ED
:10ED6C000DF13302304601F0B9F90428A070D0D06F
:10ED7C00012802D00028CCD0CDE7707D9DF84380CF
:10ED8C0098B1254801A9B8F1070F90E8CC00CCC187
:10ED9C0002D0B8F1040FBCD10DF1330001A910223F
:10EDAC001CF00CFB0028B4D12AE000208DF84700A1
:10EDBC00194801A990E8CC00CCC111A80DF147036A
:10EDCC0020220090F220212117F063FB9DF84700D0
:10EDDC00404505D1114901A810221CF0EFFA48B1A9
:10EDEC00B8F1010F0CD10DF13302002062210DF0AE
:10EDFC0039F805E009490DF1330010221DF0D0FA65
:10EE0C0004F11C000DF1330110221DF0C9FAA07899
:10EE1C0081E700BF126E0020C0EE020010EF02006E
:10EE2C002DE9F843DFF830810C469146074622461F
:10EE3C00B8F8241013F054FE002879D00689054642
:10EE4C004FF6FE70864204BFC320BDE8F8831DF068
:10EE5C00D5FB864204BFC220BDE8F8832988B8F8E8
:10EE6C00240088421CBFA8F82410084615F05EFF49
:10EE7C00E87A3946013088F8380008F139001DF07D
:10EE8C001DFF02208DF8010068461AF09BFB00283C
:10EE9C0051D00746006906210126017098F80E1022
:10EEAC004170BE771CF092FE78624020BE7687F8E7
:10EEBC001890F88228897880384611F033FE0028A3
:10EECC0045D1092008F11A0188F826002889A8F8EC
:10EEDC001A0098F81800A04218BF88F818401F4C68
:10EEEC004B20A04708F124015020A04708F118013D
:10EEFC00E120A04708F116015320A047082001216A
:10EF0C00FEF79EFC4FF400500021FEF799FC144CC8
:10EF1C004FF48061207811F061FE134800780228CC
:10EF2C000BD110480078012807D14FF4DC6208E0BF
:10EF3C00CA20BDE8F883102009E0082010F0C4FEB8
:10EF4C00820020784FF480611DF07FFE002007497D
:10EF5C0000220A70BDE8F883C05E0020D54A02008A
:10EF6C00036E0020F32600201C250020096E0020D3
:10EF7C002DE9F0474FF6FC76B04201D100240FE0AA
:10EF8C00884600211D469246002416F0C5FEDFF887
:10EF9C0014910746680606D4B9F81600874202D1C8
:10EFAC002046BDE8F087384629460DF0A9FA30B95D
:10EFBC00B01C002180B20DF0A3FA002860D0B11C67
:10EFCC00078089B2884505F0010118BFA0F80280BE
:10EFDC0045EA8101BAF1010F817142D101214171E0
:10EFEC00334915F0180F99F81420097818BF0A4600
:10EFFC0002714046B9F8241019F0A4FA0028BDD1CA
:10F00C002A482C49DFF8B0A0274B0022007891F851
:10F01C0000C06245B2D0C2EBC20600270AEB8604E0
:10F02C00B8420BD003EBC70521886D888D4201D007
:10F03C000137F5E70132F9B28842EAD120461C21AA
:10F04C001CF06EFF4AF601202AF82680A4F8110065
:10F05C001A480078013040082074B9F82400608107
:10F06C008CE7417901293FF489AF114915F0180F4C
:10F07C0008BF09F11301097880F805A001717DE73B
:10F08C0015F0180F0CD0094907480978063039B12A
:10F09C0010F8082B013912F0180FF8D10E388EE742
:10F0AC0002247DE7C05E00205C4B002071F0020062
:10F0BC0074F002006CF00200E445002068F00200DD
:10F0CC00F0B58DB00546007C0F2873D36E68686967
:10F0DC0008AC0021224613F0ABF99DF82000002863
:10F0EC0068D1287C0B2865D3307A022862D1B1898B
:10F0FC00C8B2FF285ED19DF8220010F0FD0F59D147
:10F10C00404F97F8263043F00402062A04D13E4AB9
:10F11C001268AAB1C90B1FE03B4A126812B195796B
:10F12C00012DF4D0082B01D0042B43D17589002A72
:10F13C0042D0917902293FD1284619F0B3FE39E02B
:10F14C00727C7189308800230093002302F006FE44
:10F15C00B089C10B9DF8220032888DF80D10B17B5F
:10F16C009DF824308DF810009DF825509DF8320044
:10F17C00ADF8082072898DF80C109DF821108DF8CF
:10F18C000E308DF813508DF81400ADF80A20727CF7
:10F19C009DF826608DF81110E11D8DF812208DF868
:10F1AC000F6002AD082205F10D001DF031F8284664
:10F1BC001DF0DBFD0DB0F0BDB98CA942FAD10128D0
:10F1CC0006D0E11D07F139001BF05CF90028F1D1E4
:10F1DC000E484FF40071007816F062FD0028E9D15A
:10F1EC0040F20120ADF80D00B86A029097F82E009D
:10F1FC008DF80C0002A812F033F900289CD01BF0FB
:10F20C0017FAD7E7C05E0020C0250020036E00204F
:10F21C002DE9F047DFF83091D9F840A0BAF1000F92
:10F22C0000F086800AF10C020820FF2151FA80F0D0
:10F23C00C3B21B1A18BF012312686AB163B11388D9
:10F24C00A3F60303012B01D90432EFE7DAF810001F
:10F25C0092E8FA003830FAC0DAF808200025DAE92A
:10F26C000A10CAE90A55B2B110F0E2440CD021F0F0
:10F27C000F0220F0E2434FF0000852EA030005D0E1
:10F28C001DF0F2F8B04701E0884604461DF0ECF89A
:10F29C0042462346B0471DF093F90446B9F8560090
:10F2AC0001306FF31F30A9F856004FF6FD70AAF825
:10F2BC00300009F140008AF833501BF06CF82046FE
:10F2CC001DF093FCB9F85600B9F8541088422FD1B0
:10F2DC001E48406890F8FC10072000291C4908BF04
:10F2EC000520D1E900540FF0A9FC55B195F8FC00AC
:10F2FC00002100284FF0000008BF286885F8FC109A
:10F30C0000E0002044B194F8FC200021002502B953
:10F31C00256884F8FC1000E00025A84288BF05464B
:10F32C00681C05D035B90020BDE8F0471BF0ECBDDA
:10F33C00BDE8F0871DF0EDFCB5FBF0F10548BDE82C
:10F34C00F0471CF07DB900BFA81F0020481D00200D
:10F35C00E81E0020B063002070B588B00179044627
:10F36C0001F00700012824D14B48021D2068037DC1
:10F37C001268F2B115799D42FAD19668CEB18288A5
:10F38C00212A16D1090718D4812101228DF81510D4
:10F39C00E17A0024CDE9004221228DF814103F4976
:10F3AC000978CDE90241811D05ABF22017F0FDFE75
:10F3BC0000E00124204608B070BDE07A0B281DD077
:10F3CC00022830D0062844D0012863D130680028A8
:10F3DC0060D0A07A3149032208702068417D063044
:10F3EC0005908DF81810E16805AD681D1CF0D8FF6C
:10F3FC00E0680330E0600790316849E070680028ED
:10F40C0048D0A07A254901220870E16820680630AE
:10F41C00059005AD281D1CF0C3FFE0680130E060CD
:10F42C000790716834E0B068A0B3E16805A80122C8
:10F43C0002301CF0B5FFE16820680131E1600691F3
:10F44C00817B022904BFC088ADF81400B16805A8FF
:10F45C001FE0F068F0B1E16805AD0122A81C1CF0BA
:10F46C009FFFE0680130E0601DF083FCE168ADF8BF
:10F47C001800A81D01220231E1601CF091FFE16827
:10F48C0020680131E1600791408AF168ADF8140001
:10F49C002846884700248DE71C240020CC26002019
:10F4AC002DE9F04F8BB00C460690C9881F46079289
:10F4BC00E07816F03FFD00287ED0217D0546C0B2D5
:10F4CC001AF0ADFB002879D00646E188E078059764
:10F4DC00DDE9177900224FF0000816F03BF883465F
:10F4EC00E0787071E188A07D86F80880227DF1803B
:10F4FC007081F06821691CF08BFE86F8149077827D
:10F50C004FF000090027BBF1000F4AD05FFA89F0D9
:10F51C00854246D906EBC00A9BF80110504600F80C
:10F52C00168F012904D101270770BBF8020005E0F2
:10F53C00BBF802008AF81D001BF082FFAAF8180025
:10F54C0022789BF8041052068AF81A1005D59AF8FE
:10F55C001C2042F002028AF81C20C7B9204AD28A29
:10F56C00904214D11E48A170DDE90613CDF800803D
:10F57C00828C159801901698CDE90208204608F067
:10F58C002BFC9AF81C0040F005008AF81C0009F1CD
:10F59C000109E188E0785FFA89F215F0DBFF834618
:10F5AC00B1E7304619F002FD0599DDE91423204638
:10F5BC000096F9F72DFD10E0B92000E010208DF831
:10F5CC002800E078A17D8DF82300E0888DF82410C8
:10F5DC00ADF8260008A81CF0BDFA0BB0BDE8F08F02
:10F5EC00C05E00202DE9F84F816A91F90120002AB4
:10F5FC002AD4824602F01F0000EB40049AF81C301B
:10F60C000234A34220D18B1CD2B24FF6FE784FF6B7
:10F61C00FE7C08B1B1F802C0DFF804914FF0000B8A
:10F62C004FF6FE770021B9F81650814211D29C7822
:10F63C0014F0880F08D133F8037BBEB2AE4208BF7A
:10F64C0004F0070B0131F0E7D320BDE8F84F09F0C7
:10F65C0094BF5FEA0B6006D11FFA8CF0B9B216F0BA
:10F66C0079F800284FD0BAF80C001DF04EFA98B17A
:10F67C000021027AC1712B4909788A4208D30131E1
:10F68C00490801725FFA8BF1072938BF0BF1010BA6
:10F69C0080F809B0BDE8F88F08F10101BAF80C0048
:10F6AC0089B218F0ADF920B105461E48297C0078C6
:10F6BC0015E016F0F3FC30B31C2105461CF030FCB1
:10F6CC004AF60120A5F81100BAF80C002880B9F808
:10F6DC002400688113480078411C49082974814230
:10F6EC0008D30130400828745FFA8BF0072838BF24
:10F6FC000BF1010B002085F811B028730235284658
:10F70C001BF0B5FA08B1BDE8F88F9AF8080000288C
:10F71C00F9D0DAF818102846BDE8F84F1DF0CEBA2B
:10F72C00C05E002068F002007CB50568002D6DD02D
:10F73C0004464748026842B121792846904701287F
:10F74C0003D1688920F001006881687B02282DD1E3
:10F75C00688980072ED52079CD282BD0F02829D088
:10F76C00688A00060CD5A87E50B1A873286800885A
:10F77C0016F0C4FF40B94FF4987009F0FEFE03E098
:10F78C00344800780130A8732079002856D0042022
:10F79C0020216873304800882881A87B0138A8761E
:10F7AC00A8732E48007810F071FD687B40F00400BF
:10F7BC0006282BD12B49288BC98A884214D028497A
:10F7CC00097889B129680988ADF8000001208DF805
:10F7DC000500287BADF802108DF8040020798DF817
:10F7EC00060068461CF028FB6889C0070ED02179FA
:10F7FC0028461BF04CFE688920F0010068812868BF
:10F80C00008816F07BFF217908B121B17CBD39B19C
:10F81C0040F2311001E040F22D1009F0AEFE7CBD3B
:10F82C0040F22F1009F0A9FE002560798542EDD237
:10F83C004FF49B7009F0A1FE0135F6E700266079C4
:10F84C008642A4D24FF49B7009F097FE0136F6E77E
:10F85C00F0220020D62600209E260020036E0020D9
:10F86C00ED240020C05E00202DE9F04F85B0064647
:10F87C00484893460D464FF0000E4FF6FE774FF674
:10F88C00FE730078039044480078049001200190A6
:10F89C00424800F1110A4248043002904FF0000C2B
:10F8AC000020C0076FD10499504601B330F8118C79
:10F8BC00B84518BFB04502D11C300139F5E7A84551
:10F8CC0018BFD845F8D00278541E062CF4D8072A55
:10F8DC0001D14346F0E7019A0CF1010CD207EBD1B0
:10F8EC005FFA8EF25FFA8CF49442E5D34DE0DDE9D9
:10F8FC000201994621B330F8048CB84518BFB045C5
:10F90C0002D124300139F5E7A84518BFD845F8D005
:10F91C0043795A1E062AF4D80278013A022AF0D307
:10F92C00072B01D1C146ECE7019A0CF1010CD2076F
:10F93C00E7D15FFA8EF25FFA8CF39342E1D324E0C5
:10F94C005FEA0C6002D05FEA0E6006D001204FF631
:10F95C00FE73C846B945A4D017E000205FFA8CF8B6
:10F96C004FF0010E4B46B8F1010F01903FF496AFEA
:10F97C001DF04EF8C0B24B46B0FBF8F101FB180E6F
:10F98C00002001908AE74FF6FE781FFA88F005B048
:10F99C00BDE8F08F7EF002006CF00200E445002020
:10F9AC00B83E0020F0B58DB0044603200D468DF80E
:10F9BC0030000AAE30461DF081F91CF007F9014603
:10F9CC0030461AF05FFD50B1287D40F0020103294A
:10F9DC0005D1297A09B1FF2914D1822000E08420B5
:10F9EC008DF82700E289207C0DF127010123CDE958
:10F9FC00001004F11100A11C42F4004214F0A2FA10
:10FA0C000DB0F0BD032804D1A87DFF28E5D0002857
:10FA1C00E3D0304F4FF0FF300822CDE9060006A9A5
:10FA2C003E1D30461BF054FA18BB2B486188C08A27
:10FA3C0081421ED03878FF280AD0297A814207D01B
:10FA4C0078884FF6FF71884202D06989884210D1BC
:10FA5C000020314608228DF8080002AF381D1CF03A
:10FA6C00D7FB38460EF01EF86088BDF80A108142AC
:10FA7C002DD1E08905F10C0621281CD18C20698937
:10FA8C00AB7D32468DF82700287A18F03BF9002818
:10FA9C00A8D11CF072FF287D0328A3D102A93046FF
:10FAAC0018F060F900289DD1304600210022002377
:10FABC0010F07CFC96E76989287AAB7D32461BF006
:10FACC006DF908B188208BE71CF057FF8AE78D2071
:10FADC0086E700BF04250020C05E00202DE9F04F12
:10FAEC008BB04B4FB868D0F80001807AC0001DF085
:10FAFC0044F9002809907ED00DF1040B00264FF636
:10FB0C00FF7A0BF103051CF05BFD0DF1140900905D
:10FB1C00B868B2B2D0F800110B899A4263D20124B2
:10FB2C004FF00008C97A5FFA88F28A4221D2D0F8E5
:10FB3C008824D02059468DF80680ADF80460904793
:10FB4C0028B1B86808F10108D0F80011EAE79DF86F
:10FB5C00100000240128F4D19DF80F000028F0D1EA
:10FB6C000020082806D0295C0130FF29F9D0002498
:10FB7C00E7E70CB10136CBE70024B868E1B2D0F866
:10FB8C000021D2888A42F5D9D0F88824ADF8061025
:10FB9C00D1205946ADF80460904710BBBDF8080061
:10FBAC0050451ED0ADF81400B8684946D0F88824EA
:10FBBC00D420904708BB4FF0FF304946ADF81AA04F
:10FBCC00ADF818A0CDE90700B868D0F89424D4207B
:10FBDC009047B8685946ADF808A0D0F89424D120C5
:10FBEC0090470134C9E700981CF0FFFF09981DF0FD
:10FBFC00C2F8002008E01A2006E000981CF0F5FF7F
:10FC0C0009981DF0B8F819200BB0BDE8F08F00BFB3
:10FC1C000C0100202DE9F84F1D4600928B468146C1
:10FC2C001CF0CEFC444A824600214FF4A060012710
:10FC3C0005F1010C002392F86040602935D007FAD9
:10FC4C0003FE1EEA040F0AD0BCF1000F18BF9D4240
:10FC5C0005D1561896F80A80B8F1000F04D000F5BB
:10FC6C00807020310133E8E724EA0E040125737219
:10FC7C0082F8604092F86240B572013482F86240BA
:10FC8C009EB142F801902D49BBF1020F86F808B0E5
:10FC9C00716011D0BBF1010F34D1591DB1740A211F
:10FCAC0031820A99896871612CE0FE2450461CF05F
:10FCBC009CFF60B2BDE8F88F718A5A1D0A9B02F056
:10FCCC000F0221F4706141EA0221718221F0F801E6
:10FCDC005A7902F01F0241EAC201718221F4C0413B
:10FCEC009A7902F0030241EA423140F20362328215
:10FCFC0071824EF6FF721140DA7902F0010241EA8C
:10FD0C00023171820B9A42B111785278920042EA18
:10FD1C00411108430A49084300E000200099B061F2
:10FD2C0001B171600748416809B9C0F804900FF03F
:10FD3C00D7FD747ABAE700BF385F00201B6E010054
:10FD4C0001000406481D00202DE9F04F95B00DF17F
:10FD5C00110A80464FF0000BADF852100AF1340036
:10FD6C000AF12C060AF12A070AF122050AF13704D6
:10FD7C0001900AF13B0002900AF10B000390BBF1D9
:10FD8C00040F76D85FFA8BF0514617F070FF0D28F0
:10FD9C006CD00A286DD003990DF152001CF037FF7E
:10FDAC00B8B90DF1520021461CF031FF88B9029907
:10FDBC000DF152001CF02BFF58B90DF152002146E9
:10FDCC001CF025FF28B902990DF152001CF01FFF01
:10FDDC00E8B10C201DF043F8C8B100210C2281467B
:10FDEC001CF033F9BDF85200FF210822A9F80000DD
:10FDFC0009F102001CF029F90020494689F80A0093
:10FE0C001D4800781CF05EFE48461CF0D2FEB8F18E
:10FE1C00000F2BD04046294608221BF0CFFA40B1E8
:10FE2C000DF1520039461CF0F2FE002838461DD167
:10FE3C0017E04046314608221BF0C0FAB0B1A1468B
:10FE4C002C463D463746019E0DF1520002223146AA
:10FE5C001BF0B4FA002830463E462F4625464C4649
:10FE6C0004D10DF1520102221CF09AFA0BF1010B94
:10FE7C0085E715B0BDE8F08F126E0020F8B50D4681
:10FE8C00417F0446827F1020002908BF0820607043
:10FE9C000AB108306070217F09B101306070A1791E
:10FEAC0021B1217A00EB4100023060700021267EE6
:10FEBC0084F83410217D002E18BF0E2631440844DE
:10FECC002870217E31B13848007B1CF0E1F929788B
:10FEDC0008442870C0B274283DD81CF04EFFD0B333
:10FEEC00054631482178677E237F94F818E094F812
:10FEFC0006C0627F807C002B41EA800007F0030182
:10FF0C00A77F40EA811094F83410287018BF0123A1
:10FF1C0040EA032040EA4E2040EAC22040EA073083
:10FF2C0040EA8C2040EA4130000A6870A078A87042
:10FF3C00E078E8702079287160796871A07EA871EA
:10FF4C00E07EE871607F40B1216A05F108001CF089
:10FF5C00B5FE102702E0002523E00827A07F20B182
:10FF6C00616AE8191CF0AAFE0837A07970B1207AF2
:10FF7C00E855E8190237617A4170E819227AE1688C
:10FF8C0052001CF045F9207A07EB4007207F08B19E
:10FF9C00F9B268546078227D2169284430441CF001
:10FFAC0037F92846F8BD00BFC05E00202DE9F04FA0
:10FFBC0089B00E46834601A8202114461BF0B0FFE1
:10FFCC00202E08D0182E04D0102E0CBF012700278D
:10FFDC0002E0022700E0032744F2040A4FF0010874
:10FFEC00C4F2020A40F2B01908FA04F5C1F2000991
:04FFFC000094CAF8AB
:020000021000EC
:100000000054D9F8000044F2007441692720C4F27A
:10001000020488470320C4F88080C4F88400C4F830
:100020000080C4F888004FF60850CFF6FF702158C2
:100030008F4218BF2750182ECAF8FC5315D101A8BB
:10004000594618221CF014FF0320C4F8880000BF92
:10005000D4F890008007FBD10020C4F24820012191
:10006000016020260DF1040B11E0BBF1000F18BF59
:10007000002E10D00320C4F8880000BFD4F89000F0
:100080008007FBD10020C4F2482001210160CAF89A
:1000900000B0CAF808600325CCF2000501201CF06E
:1000A00042FDD4F890002842F8D0D4F890000540E2
:1000B000C4F88850D9F80000016A27208847D9F889
:1000C00000000169272088470020B0EB957F07D109
:1000D000DAF800040099C043C84000F0010000E0D5
:1000E000012009B0BDE8F08FF0B597B006460020BA
:1000F0000590ADF81200B1B11446A2B19EB1002036
:100100000D4610220870204600211BF0A4FF307914
:100110008DF8040050B101A806F10801082204304E
:100120001CF044F904E0042017B0F0BDB068029060
:100130000DF11B0701A80DF1120239460DF0DCFA92
:10014000012855D0022808D13148807800284FD0A6
:10015000307D01283BD90320E6E79DF80400022802
:1001600006D1307C9DF82510884218BFFF283DD16C
:100170009DF82810307D01F00301084334D007F1C9
:100180000E0105A804221CF011F9B06905998142FD
:1001900016D29DF82800317D00F003028A420FD16B
:1001A000C10602D4717D01290AD0C0F3820007285C
:1001B00001D0042801D1717D11B10538012819D869
:1001C00013488078002818BF01204000ACE7707DFC
:1001D00050B91049204610221BF0F6F820B90D49FD
:1001E000204610221CF0E2F802209DE70028BFD034
:1001F000002099E707F11201204610221CF0D6F8E2
:100200009DF82800C0F38200287001208CE700BF11
:100210005823002010EF02002DE9F04F8BB0424828
:10022000DFF80CB100240DF11C0A4FF000084FF06C
:10023000000900270078019000EBC00086003B48D1
:10024000007801304008029046455CD01FFA89F1E1
:10025000032000221023CDF800A018F081FE002812
:100260004CD19DF821300BEB0801BDF81C009DF826
:1002700020200C82CC60CC724B714AF601232BF803
:100280000800BDF81E000A71A1F80930029B4880E1
:100290000B72BDF82230CB800A9B5D1C04D081F824
:1002A0002040C1E9063315E0013A012A09D8214A64
:1002B00012784AB1204B53F82220C2EB021292006E
:1002C00004E06FF0010203E01B4A126881F820404D
:1002D0008A61CA614FF6FF7188420FD0ADF81800ED
:1002E00001208DF80C0003A812F070FA28B1134811
:1002F000818CBDF81C0018F0EDFA013708F12408D4
:1003000009F10109A0E700200421002416F038F9C2
:100310000199884224BF0A48047006F0FFFBF8B236
:100320000BB0BDE8F08F00BF7EF0020068F0020065
:10033000B83E0020E6260020C8EA0200C05E002089
:10034000A82600202DE9F041414F04467878C8B135
:10035000DFF80081B8F85400B8F8561088421ED073
:1003600008F1380120461AF02DF880B9D8F8480075
:1003700010B10069A04207D008F1400120461AF0F0
:1003800021F803E0BDE8F081D8F8480038B1B0F9B1
:10039000301020460A224FF0E04308F091F81CF09C
:1003A00015F92D4D0646284602C8A14208BF284629
:1003B00000210160787801387870000636D17C60C1
:1003C000387E02280ED1082017F048F830461CF07D
:1003D00012FC04F150004FF0FF311CF033FB1CF015
:1003E000F5F8064605F128001CF0DFFC40461CF03D
:1003F000A4FC1A481CF0D9FC08F11C001CF09DFC60
:1004000017481CF08AFC17481CF087FC1648416806
:1004100011B107F15000884707F128001AF0BEF922
:100420001248807810B10D2007F0C0FA7868A04219
:1004300004BF0020786030461CF0DDFB04F1500062
:100440001CF0AFFC04F1B800BDE8F0411CF065BC45
:10045000481D0020A81F0020E81E002088650020FD
:10046000F4630020B06300206025002058EF0200F4
:100470002DE9F0410546880058BFBDE8F081002015
:10048000002411F0A3F83E493E483F4FCC6108607C
:1004900040F60A008846B887FC8797F8480000F0C5
:1004A000F00087F848003C6497F8490000F0F0003D
:1004B000013087F84900284608F0A6FBAC68012007
:1004C00021460E46496849B10A88A2F60302072A66
:1004D000F7D800FA02F212F0830FF2D0707B00F02E
:1004E000F000707307F13C0070602848806B28B101
:1004F000C0680088A0F6030002281AD3284630F806
:10050000381FB1B10021E9636987386495F8440068
:1005100095F8451000F0F00085F8440001F0F00077
:10052000013085F8450097F8490000F0F00087F8A1
:1005300049001BF079FB1648F86197F8250030B1A7
:1005400019F096F80028FBD013F072FC0DE011486A
:100550000068016801208847012806D0707B00F000
:10056000F000013070730C48F86100202146C8F893
:100570001C00C8F800400120BDE8F0411AF03EB967
:100580000010044001010E04481D0020A81F002097
:1005900055380000E0010010A51F02002DE9F047CA
:1005A0008EB080460E2016468A468DF81A308DF899
:1005B00018208DF8190001208DF81C003E48B8F174
:1005C000000F077B8DF81B7021D00AEB0605687BB6
:1005D00012F0C4F9002403463A2802D03B2B0BD179
:1005E0003B230DF10409002011214A461AF030FC8A
:1005F000002808BF09F1010428780994384305F858
:10060000050B0DF12B0029461CF05EFB36E001AD19
:10061000002011213A2300242A461AF019FC08B1BF
:1006200009942BE0DFF894906C1C012101220994BD
:10063000D9F80430581CC9F804000AEB06000090F1
:10064000384612F069FB1BF0C7FA01460DF12B008A
:100650001CF03AFBB9F80000194901300968A9F803
:10066000000080B2814203D3D9F80400012805D1EB
:1006700014484FF4007100780FF00EFE0DF12B00BE
:100680000AEB06050422691C08301BF0C7FD1AF8A6
:1006900006008DF837005CB106A90DF12B0240462B
:1006A000534605F08FFF297801F0F801297000E02A
:1006B000A1200EB0BDE8F087C05E0020DC23002042
:1006C00034F00200046E00202DE9FE431BF07EFF93
:1006D000DFF80C91804699F80100B8B14148032237
:1006E00001688260C80711D03F4C20684168022031
:1006F00088470190206841680120884702903B4864
:1007000001A91C3011F0A6FA18F004FAD9F8045027
:10071000EDB13649686A01AF01F11C06A96A884249
:1007200019D23046394612F00FFD013011D0D5E90B
:100730000912E869541A08443946082C28BF0824CD
:1007400022461CF095FB686A20446862E6E70024B4
:100750000CE0D5E909010024884207D309F104001F
:10076000294618F00DFF85F83240012499F8010060
:1007700088B9D9F8040018B180681BF063F90AE061
:100780001A481C301BF084FE28B9194A4FF0FF307C
:10079000012110F0B3FA40461CF02DFAF4B1A8681C
:1007A00000220168CA628A690AB10223137091F8B3
:1007B0003030012B07D0022B10D101F134001CF096
:1007C000F2FABDE8FE8322B1CB6800219847BDE86C
:1007D000FE830C69CA698B6A0021A047BDE8FE83CD
:1007E000A821002008800240CC010010D020002069
:1007F00080A9030070B586B0454D0446A868D0F8BE
:10080000F41091F84420B2F1820318BF531C81F810
:100810004430D0F8F40090F8441000EBD10090F888
:100820002C104A0880F82C20C807A86809D1D0F8F5
:10083000F41091F94420531C12F1020F81F8443056
:10084000E7DCD0F8F420114611F8443F802B25D87E
:10085000D0F83024E1209047AA6802208DF81400D7
:100860004FF0FF30D2F8F430ADF80C009878022841
:1008700023D0012824D030BB1CF051FA4FF47A71F8
:10088000244B0022B1FBF0F023490BF0FFFDE0B355
:10089000A8681A21D0F8F400417004E0907810B9EB
:1008A0001C4814F0DDFC2A202070A868D0F8401302
:1008B000204606B0BDE870400847D2F86814F7E754
:1008C0000820802101E007208321D2F8786303F11A
:1008D00049020023CDE9003203AA4FF6FF73B04767
:1008E000A0F1DB01182910D8012202FA01F10B4A0C
:1008F00011420AD0A968D1F8F41048702A2020705B
:10090000A868D0F840132046884706B070BD00BFE5
:100910000C010020C06D0020DD4901001124000100
:100920002DE9F04F85B0054691460E46C80731D1F6
:100930002846314615F0F6F9404FF98A884242D0F0
:100940002846022132460CF023FEE0B328464FF63B
:10095000FE7102223346FEF711FB90BB4FEA1528C9
:1009600006F0DF0A70061ED402A9284617F010FF11
:1009700068B9B98C284617F049F8A0B1871C3846E9
:100980001AF07BF978B102A839461CF09DF946F0BF
:10099000200A08E0B0074CBF46F0100A46F0080AEB
:1009A0004FF0FF08FC25264800220778791C0170CB
:1009B0002248012100913946C08A034609F01AFAFB
:1009C00018B1C72036E0002034E00E201AF02004D1
:1009D00008BF06208DF8110004A818F0F9FD40B3F7
:1009E0004FF0010B064680F81EB01BF0F5F8706260
:1009F0003069002141710AF078018770C57080F874
:100A0000048080F800B041701CB1063002A91CF0CF
:100A10005BF96FF00300B9F1000F708005D0094851
:100A20000078484588BF86F81A90304610F080F864
:100A300000E0102005B0BDE8F08F00BFC05E0020D0
:100A40002A6E002065F002002DE9F0438FB015F00A
:100A5000D3F83F4F97F82600082806D00120C7E9B1
:100A60000C003C480078F87078710DF114082421CE
:100A700040461BF05BFA39480F25374EDFF8E0900F
:100A80000DF13B018DF83B5000783570013818BFEF
:100A900001208DF81E004620C847324800248DF8FA
:100AA000004000788DF801001BF0A8FD8DF80200D1
:100AB00097F838008DF80640ADF8034007F139018A
:100AC0000F2838BF05468DF805506D46E81D1CF00F
:100AD000FBF84FF0FF303278234EADF80F008DF861
:100AE000110097F8720031468DF81200284611F077
:100AF00032F945203146C84706F010F8B88D97F80E
:100B00002F108DF820408DF834408DF82940ADF835
:100B10001C00387E8DF81F1007F116018DF81A00A1
:100B2000B88CADF818005320C84707F11A014B20C4
:100B3000C847F879642100FB01F20C4808210078CD
:100B40001CF089F8404606F057FC0FB0BDE8F08372
:100B5000C05E00207EF00200C42600201C2500207C
:100B6000D54A0200F6260020706C0020036E00209B
:100B70002DE9F04F8BB01E46984691468A460025D7
:100B80000A9016F8027BAFB116F8010C08B10435D3
:100B90000DE0307808B1063509E0F47809352046D3
:100BA00018F06EFF18B120461AF0C4FE05440F3647
:100BB000013FE8E71FFA85FB58461CF056F900286C
:100BC00066D05746CDF82490064608F106094FF046
:100BD000000A044698F8000082453DD219F8050C39
:100BE000207019F8040C607019F8030CA07019F843
:100BF000020CE07019F8050C08B1043427E019F86C
:100C0000040C38B199F80400207199F8050060715E
:100C100006341CE019F8010C207199F8000060718D
:100C200099F80100A07199F80200E07199F80300A9
:100C30002072093419F8015C284618F021FF30B100
:100C4000D9F806102846224604F00EFB044609F1A6
:100C50000F090AF1010ABDE71799149A002918BF74
:100C600001210192159ACDE9066100203946092338
:100C7000CDE9022000901698099ACDE9040B0A9854
:100C8000FCF7AEFB044630461BF099FF204600E01F
:100C900010200BB0BDE8F08F2DE9F84F4FF0005653
:100CA000002A984617460C46824618BF4FF08046E9
:100CB0004D1C1BF08BFC814635B15046214600226D
:100CC00013F01AFE04460FE03748816C11B1096930
:100CD000514506D0C16C11B10969514503D0846BEF
:100CE00002E0846C00E0C46C34B194F93300B0F1DC
:100CF000FF3F03DD042451E003244FE0DFF8A8B0F8
:100D00000A9DDBF84800844218D0DBF84C0084428E
:100D100014D05046214642462B460AF07BFC002860
:100D2000E8D02248017E012937D0007E042834D043
:100D30001F48204928301CF03AF82EE0DBF8480024
:100D40000022334618F0A8FCDBF84C0000223346A2
:100D500018F0A2FC1848002F18BF00F5803019F0D9
:100D60008DFC85B1DBF848001BF049FEDBF84C0038
:100D70001BF045FE20690E49086291F8240040F0FE
:100D8000010081F82400B8F1000F06D0DBF838101C
:100D9000504601222B460AF03DFC832448461BF0B6
:100DA0002AFF2046BDE8F88FA81F0020481D00201C
:100DB000E81E002002000040010001042DE9F04778
:100DC00088B0434D0A4604461046A98C17F0C0FB74
:100DD00040B1417831B9072141703E49097801316C
:100DE00049080170A06A10224778F90658BF082206
:100DF00017F08F0F13D1BB0648BF0832237F9342F1
:100E00000DD190F8029090F80780B0F805A0B0F8E6
:100E10000360002909D407F0700708200DE0D320F3
:100E200008B0BDE8F04708F0AEBB00F1080106A825
:100E30001BF04AFF07F060071020B90606D5A16A2B
:100E4000014404A81BF040FF07F05007B6B2494622
:100E5000304616F037FB2049097888421ED21F49D8
:100E600000EB800001EB400010F8061F41452CD933
:100E700080F80080E88A864213D0A1891FFA8AF49C
:100E800001223B462046FEF779F8F0B904A806A9EE
:100E90000297CDE900103046214612E0E88A8642EA
:100EA00007D1A1891FFA8AF001223B46FEF766F8B6
:100EB0000BE004A806A90297CDE900101FFA8AF1F9
:100EC000304642464B4602F0C3FF08B0BDE8F0870B
:100ED000C05E002068F0020070F00200186300207D
:100EE00070B50C46080418D4E00725D1A00733D408
:100EF000A00636D4600448D4E0064BD4200744BF93
:100F000084F0080070BDE00556D4600760D400206E
:100F10002146BDE8704009F02FB9324E30780FF00D
:100F200091FE30B1054607F077FB284619F0D2FE56
:100F3000F4E784F4004070BD012019F0AFFC2A48AA
:100F40000F220F2381782948008800F0070001F064
:100F5000E1FF84F0010070BD0AF0C4FE84F00200DD
:100F600070BD2348007840B91F480078062802D198
:100F7000072019F093FC19F01DF81A481021007889
:100F80000FF08AF984F0200070BD13F03DFD84F469
:100F9000804070BD1448007811F008FD15480078B5
:100FA000012806D114484FF40061642200781BF038
:100FB00052FE84F0100070BD104890F826000828FA
:100FC00001D0042801D11AF057FE84F4807070BD5E
:100FD000FF20032115F0EEF91BF022FB0848012148
:100FE0000160FEE7046E002004230020806C0020D6
:100FF000296E0020DC260020036E0020C05E002049
:101000007C0520432DE9FE4F8A4683461AF03EFEBA
:10101000424FDFF80081404E397898F80200B073F3
:1010200039B1000713D501200DF10A018DF80A002E
:101030000AE00020002410F05BF8B07B000706D522
:101040008DF80B400DF10B01522013F043FD0EF013
:1010500073FE1AF02BFB38B1054610F0DBF916F0E1
:1010600061F90CF081FE08E00AF07EFE0546307E54
:10107000012101FA00F02A4908604FF6FE74012DA3
:1010800031D10FF039F91BF0C9FC07462548244936
:1010900000680860FF20022115F08CF9012013F090
:1010A0009BF8601C7483F4824FF00009B084002028
:1010B00013F09AFB07F07F00BAF1010F584400F1DA
:1010C00064061ABFCDE900996846002015F0DCFCE3
:1010D000114A124F212074211BF0E0FB0020022155
:1010E00015F068F900E00026284619F0F7FB601CAF
:1010F00080B2834506D00120387018F0E1FAB0B212
:101100001AF0C8FA98F8020019F0BEFE2846BDE8A9
:10111000FE8F00BF806C0020C05E002004230020F2
:10112000D86D0020882600202DE9F843804600680D
:101130003B4BD8E9012118603A4802603A48202226
:101140001BF096FED8F80C003849DFF8E89090E8DC
:10115000FC00FCC1D8F80C00354990E8FC00FCC14B
:10116000D8F81000494690E8FC00FCC1324D4022FE
:1011700099F80C00D8F8141040F0800089F80C00A1
:1011800028461BF075FEE87BD8F81810202240F0A6
:10119000A500E873294D28461BF06AFE40F2054081
:1011A000697BAA7CEB7DC5F8049028820320287512
:1011B000287B40F08000287301F0F00020490230C5
:1011C000687302F0E0000A460130A87403F0F000F2
:1011D0000130E875D8F81C0090E8F800F8C2087BE8
:1011E000CB7B4A7B40F08000087303F070008430B2
:1011F000C87302F0F000013048734FF45860086182
:10120000D8F820000F4908600F48C068406900788E
:1012100008B111F08FFEBDE8F84316F05BBB00BFCC
:10122000CC6D0020D06D002038690020B86A002005
:10123000D06A0020E86A0020486500201869002074
:10124000706B0020C86D00200C0100202DE9F041DA
:10125000D0E9016705461BF0B9F98046D6F8C00011
:10126000002867D096F8F81019B9007C03380128D7
:1012700065D838791BF063FDD6F8CC2079693868D9
:1012800052681268D16296F8F93013B9C368DB0668
:10129000FCD4436823F0020343603B69D3621943E3
:1012A000446A24F003044462C2F80415416921F041
:1012B0000101416101210162D6E93512D6F8C00071
:1012C00001604AB1FB699B68C3F309139A4203D9D1
:1012D0001144DA4311440160D6F8DC204AB17B6A3C
:1012E0009B68C3F309139A4203D9DB431A441144A0
:1012F0000160284612F0D4F9387919F06FF938797D
:101300001BF01FFDD6F8C00000220223016805462D
:101310003DB12C7C033C022C28BF2B742A606D69E4
:10132000F6E73246016052F8C81F79B14A695AB1EE
:101330001146FBE73868416821F0020141604046F0
:10134000BDE8F0411BF057BC01F114021060002011
:10135000C6E93000C6E93400C6E9360040461BF055
:101360004AFC06F13000BDE8F0411BF022BD704799
:10137000F0B589B00546002001F108060C468DF84D
:101380000F00304619F079FC18B9284631460BF0A9
:10139000E3FE04AD0DF10F0130462A460AF016FBBC
:1013A000374E4FF6FF7731784A1E9DF80F10012A0D
:1013B00010D879B900200DF10F01CDE90000684681
:1013C00004AA0AF003FBB8421ABF01218DF80F10DE
:1013D0009DF80F10B1B1B84214D09DF8201099B308
:1013E000FF2926D0022918BFFD2912D1264900EB7A
:1013F000400001EB8000A16950F8042F91420FD208
:10140000A2203AE0307810B91BF0E9FCC0B1A1206D
:1014100033E0012930D130780138012806D90FE0B6
:10142000013101603078013801281ED84FF08170F9
:1014300007E03078013801289CBF012084F826009D
:101440001048C4F8120017E0052060829DF82300C0
:1014500000F07F00A0820D480078002818BF01200E
:1014600084F8270084F8260006E004F11E0005F148
:10147000080108221AF0D2FE002009B0F0BD00BF1A
:101480001C25002000000301AC680020B2260020CB
:10149000F8B5D0E90067044638781AF075FB7A7819
:1014A000317990420ED1481E0A2807D8DFE800F0B3
:1014B00006060606414E064406065800072030710F
:1014C000002552E0481E0A2810D8DFE800F0170F68
:1014D000260F06060F0F2C0F0600307C10F0120F9F
:1014E00004D01AF063FE30681BF023FC02200025B4
:1014F00030717878E8B301283ED042E01BF011FC4F
:10150000B060307C00F0010510F0120F4ED01AF0E0
:101510004DFE30681BF00DFCEBE704203071307C91
:1015200000F00205E5E70A203071307C00F020056C
:10153000DFE7307C80062DD4B0681AF0A1FCF060A3
:1015400007203071307C00F00C050EE0B0681AF016
:1015500097FCF06007203071307C00F0140504E047
:1015600007203071307C00F00405787820B1012824
:1015700007D14FF4A02101E04FF4C021387816F0D4
:101580009FFC35B1726922B120462946BDE8F8407A
:101590001047F8BD0820B169326A30713068511ABD
:1015A0001BF0C5FB30681BF0C4FB89E702209FE7F6
:1015B0002DE9F04387B0DFF8FC8081462025EFF36A
:1015C000118085F31188D8F830501DB180F311884F
:1015D00000256AE0C8F83090374F80F3118800206A
:1015E000C9F80C104FF48031C9F81C20C9E9120069
:1015F000C9E90801002B18BF1F46D7E90116C9F831
:101600001810397B012905D1C9E91060C9F81460A7
:1016100030460DE0294A00203146002300251AF00B
:1016200089FCC9E910012649C9F814008E423CD84A
:101630000021DFF890E0C9E9160197F800C0C9F869
:101640005410BCF1020F08BF0146C9F8501001AB9D
:101650009EE8F5001946BCF1000FF5C108F11C0029
:101660001A4ACDF808900090174808BF0246142186
:1016700009F1280018F018FE05462020EFF311812B
:1016800080F3118881F3118899F8100010B9484649
:1016900012F0C2FE35B108F12800494619F032FEB9
:1016A0004D4602E00025C8F83050284607B0BDE896
:1016B000F08300BF181E0020F4EC020040420F002F
:1016C0003F420F00B8ED02005D6102004DC3020011
:1016D0002DE9FE4F8146408800274FF0050B4FF063
:1016E00002084FF0000AD9F8045001902E1800208B
:1016F0000290B5421ED2297801370AF1030019B1D0
:1017000018FA80FA0535F4E7EC781BFA80FA083508
:10171000204618F0B5F90028EBD020461AF00AF957
:10172000019910FA8AFA8A455FD802990544014462
:101730000291DEE7C7EBC7004000441C029850FA54
:1017400084F080B21BF091FB00284ED050FA84F553
:10175000D9F8044081465FFA87F84FF0000A0290FA
:1017600009F8017BC2453DD0CAEBCA0700210E2211
:1017700009EB470630461AF06EFC207809F817008E
:10178000B4F80110A6F8011020B1B4F80300053434
:10179000308124E094F803B04746B04608F803BF10
:1017A000A088A8F80100E0880834A8F8030058468B
:1017B00018F066F990B15846294616F0B9FF002195
:1017C000884203D0625C6A540131F9E798F800005E
:1017D000C6F80A501AF0AEF805440444B8460AF1B7
:1017E000010ABFE70298BDE8FE8F0020BDE8FE8F2A
:1017F0001EF0040F14BFEFF3098169468869A1F157
:10180000480214BF82F30988954621ED100BF1EED2
:10181000102A41F8082DEFF3118102B400B5DFF86A
:10182000D8E0F047374A1268116801EA00001060FA
:101830005DF804EB1EF0080F09D101BC80F311889C
:101840005DF8080BE1EE100ABDEC100B704704BC0C
:101850001EF0040F14BFEFF309816946A1F12001C6
:1018600014BF81F309888D464A604FF08070C861CB
:1018700025488861234B1B681868086040F20110F6
:101880001860704702B401B4EFF3148100291CBF43
:10189000002282F3148802B402B4DFF860E0F0475B
:1018A00001BC01BC00281CBF022181F3148801BCCB
:1018B000DFF84CE0F0470F484FF08051016001BC69
:1018C00080F3118800BF00BFFFF7FEBF1EF0040FBA
:1018D00014BFEFF30981694601F1200151F8080BAB
:1018E000E1EE100AB1EC100B14BF81F309888D46AC
:1018F000704700BF04ED00E03DEF0100D5CC0200D1
:10190000DBCC020040F0020084180100F8B5044668
:101910000020A5782075C4E9030045F0020000F01E
:10192000030002280CD115F00C0005F0030218BFCB
:10193000042809D1022A05D1E90601D402210FE0C9
:10194000012619E0022106E00C2803D00828F1D076
:10195000012100E00321022A02D1EA060E460BD43F
:1019600048B10E1D0C2807D8012202FA00F041F2FE
:101970001012104200D04E1D28060AD5E0788007CC
:1019800006D0A8074FF0030058BF0220064400E02D
:10199000013627881AF038FE87420BD0A80609D5F1
:1019A0001F48416920468847206918B9A07800F08F
:1019B000DF00A070207D00B1F8BD61795020751C5A
:1019C0008DF8000020798DF80210216928448DF8E7
:1019D000010029B10A7F497F104408448DF80100B5
:1019E000684613F07DFFA0B1012180F84850417690
:1019F00021884180618801872179226980F842101D
:101A000001692944416412B1127F11444164E060CC
:101A1000F8BD20461AF08FFF10202075F8BD00BFDA
:101A2000082300202DE9FF413B4E96F84201002893
:101A30006AD1012086F842011AF052FE374F86F82B
:101A40007001374D7868C6F86C01387B86F8410123
:101A5000A86810F4402F13D1386988B12868642130
:101A6000C0F3066000FB01F41BF059F9B4FBF0F27F
:101A70002C4906F19400002316F00AFA1AF0D6FB5E
:101A800001AC20461AF061FF2749A846002506F15F
:101A90000C0000221AF0B6FC20461AF056FF23492B
:101AA00006F1500008221AF0ADFC214A06F1D800D8
:101AB0003221002314F00AF81E4C1F4A06F1F400EC
:101AC0002C2100232560454614F000F8D8F80800C2
:101AD000797BC0F3815021B1032804BF012186F82E
:101AE0003911032803D040F00200022810D12068E9
:101AF00040F040002060022016F0A2FA686840071B
:101B000002D4002016F09CFA002004B0BDE8F08159
:101B100014F086FEF2E700BF501A0020FCED020030
:101B2000AC4F00502BC502000BC20100E152020075
:101B30009DFD010090220840F1C200002DE9F8430C
:101B40001D46434BDDF8208043F606061C680388DB
:101B500014F0007411D0B34227D0B3F5C15F33D075
:101B600040F60206B3423ED100F112030B60416918
:101B7000116081692960C1692EE0B3420AD0B3F5D2
:101B8000C15F03D040F60206B34203D100F1120355
:101B9000143002E000F11A031C300B600068106082
:101BA00000202860C8F800004BE000F11A034FF055
:101BB00000090B60C1691160016A2960416AC8F8B7
:101BC000001000F118011CE000F112030B604169E4
:101BD0001160416A2960816AC8F8001000F11001A3
:101BE00090F80F900DE000F11A030B60C1691160CD
:101BF000816A2960C16AC8F8001000F1180190F8E4
